:100000000C943E050C9484050C9484050C94840592
:100010000C9484050C9484050C9484050C9484053C
:100020000C9484050C9439180C9484050C94840564
:100030000C94D0310C9484050C9484050C948405A4
:100040000C9484050C9484050C94A3140C948405DE
:100050000C94D10A0C9484050C949B0A0C9484058E
:100060000C94F51A0C9484050C94562D0C9484056C
:100070000C94B6750C9484050C9435701C1B211BD4
:10008000261B2F1B461B5D1B6D1B7D1B9A1B831D97
:100090005D1B451C561C851CA31CC01C1A1D751D10
:1000A000901F3A20C9204921812124222B24952404
:1000B0000F255825A225D025FD256026AA26F42641
:1000C000ED27752DA92DEC2D5C2E742EB52E6C2FE1
:1000D0003330333033303330333033303330333008
:1000E000333033303330E82FEA2FEF2F0730093029
:1000F0000A0D3D3D3D3D3D3D3D3D3D3D3D3D3D3D93
:100100003D3D3D3D3D3D3D3D3D3D3D3D3D3D3D3D1F
:100110003D3D3D3D3D000A0D426174743A0020258D
:10012000642043656C6C732000204C6F77207761EE
:10013000726E696E673A2025642E2564000A0D46AA
:100140006F756E6420424C2D4374726C3A2000250A
:1001500064000A0D0A0D2121204D495353494E4791
:1001600020424C2D4354524C3A202564202121003A
:100170000A0D43616C6962726174696E6720707206
:100180006573737572652073656E736F722E2E00C2
:100190004F4B0A0D000A0D466C696768742D74692F
:1001A0006D65202575206D696E20546F74616C3A01
:1001B0002575206D696E00416E676C654E69636BD5
:1001C00020202020202020416E676C65526F6C6CCF
:1001D000202020202020204163634E69636B202073
:1001E00020202020202020416363526F6C6C20204F
:1001F000202020202020205961774779726F20200D
:1002000020202020202020486569676874205661DE
:100210006C7565202020204163635A202020202017
:100220002020202020202047617320202020202013
:1002300020202020202020436F6D70617373205692
:10024000616C7565202020566F6C74616765205B5A
:10025000302E31565D2020526563656976657220C7
:100260004C6576656C20204779726F20436F6D7006
:10027000617373202020204D6F746F722031202015
:10028000202020202020204D6F746F7220322020EB
:10029000202020202020204D6F746F7220332020DA
:1002A000202020202020204D6F746F7220342020C9
:1002B0002020202020202031362020202020202017
:1002C0002020202020202031372020202020202006
:1002D00020202020202020313820202020202020F5
:1002E00020202020202020313920202020202020E4
:1002F00020202020202020536572766F202020208F
:1003000020202020202020486F76657267617320AE
:100310002020202020202043757272656E74205B9F
:10032000302E31415D202043617061636974792012
:100330005B6D41685D20204865696768742053657E
:1003400074706F696E7420323520202020202020A8
:100350002020202020202032362020202020202075
:1003600020202020202020436F6D70617373205364
:100370006574706F696E744932432D4572726F7285
:1003800020202020202020424C204C696D697420C0
:10039000202020202020204750535F4E69636B208F
:1003A000202020202020204750535F526F6C6C206B
:1003B0002020202020202021212120494E434F4D64
:1003C00050415449424C4520212121002E000A0D64
:1003D00020444143206F7220493243204552524FFE
:1003E000522120436865636B204932432C203356E9
:1003F0007265662C2044414320616E6420424C2D7E
:100400004374726C005B25695D005B25695D002BA0
:10041000204D696B726F4B6F70746572202B0048B2
:10042000573A5625642E25642053573A25642E25C5
:100430006425630053657474696E673A25642025EA
:1004400073004D69786572204572726F72210048A1
:1004500061726477617265204572726F7220313A01
:100460002564202121004D697373696E6720424C19
:100470002D4374726C3A256421210021204E432DB6
:100480004552523A2025326420212000493243202F
:100490004552524F52212121004865696768743ADC
:1004A000202025356900536574706F696E743A2594
:1004B00035690050726573737572653A2535690048
:1004C0004F66667365743A20202535690048656972
:1004D00067687420636F6E74726F6C004449534197
:1004E000424C4544006163742E2062656172696EFE
:1004F00067004E69636B3A20202020202025356953
:1005000000526F6C6C3A2020202020202535690095
:10051000436F6D706173733A202020253569004B5D
:1005200025693A25346920204B25693A253469200C
:10053000004E693A2534692020526F3A25346920EB
:100540000047733A253469202047693A25346920E9
:100550000050313A253469202050323A2534692040
:100560000050333A253469202050343A253469202C
:10057000004779726F202D2053656E736F72004EA5
:1005800069636B25346920282533692E2569290084
:10059000526F6C6C25346920282533692E25692912
:1005A0000047696572253469202825336929004E82
:1005B00069636B2025346920282533692E25782925
:1005C00000526F6C6C2025346920282533692E2554
:1005D000782900596177202025346920282533693E
:1005E00029004E69636B2025346920282533692949
:1005F000282533692900526F6C6C20253469202826
:100600002533692928253369290059617720202558
:100610003469202825336929282533692900414375
:1006200043202D2053656E736F72004E69636B20FB
:1006300025346920282533692900526F6C6C2025E8
:100640003469202825336929005A202020202534A8
:100650006920282533692900566F6C746167653AF3
:100660002020202533692E2531695600437572728A
:10067000656E743A2020202533692E2531694100AA
:10068000506F7765723A202020202025346957006A
:100690004469736368617267653A202535696D4105
:1006A000680052656365697665720052432D525346
:1006B00053493A202020202534690052432D51759A
:1006C000616C6974793A202534690052432D43687E
:1006D000616E6E656C733A25346900436F6D7061AD
:1006E0007373004D61676E65743A2020202535696B
:1006F000004779726F3A2020202020253569005369
:100700006574706F696E743A2025356900506F7496
:100710006925693A202025336900506F746925697D
:100720003A202025336900536572766F20200053EC
:100730006574706F696E74202025336900506F7383
:100740006974696F6E3A202533690052616E67657E
:100750003A2533692D25336900424C2D4374726C60
:10076000204572726F727320002533642025336434
:1007700020253364202533642000424C2054656DCD
:100780007065726174757265002533642025336469
:1007900020253364202533642000424C2D4374729D
:1007A0006C20666F756E6420002025632020202554
:1007B000632020202563202020256320002025633E
:1007C0002020202563202020256320202025632051
:1007D000002025632020202D2020202D2020202DCA
:1007E0002000313000313100313200466C696768D9
:1007F000742D54696D65202000546F74616C3A2526
:1008000035756D696E004163743A20202535756D2C
:10081000696E0028726573657429000A0D47656E5C
:1008200065726174696E672064656661756C7420B9
:10083000506172616D657465722053657420256422
:10084000000A0D5573696E6720506172616D6574A1
:10085000657220536574202564000A0D47656E6536
:10086000726174696E672064656661756C74204D91
:1008700069786572205461626C65000A0D4D697873
:1008800065722D436F6E6669673A202725732720AE
:10089000282575204D6F746F727329000A0D41432E
:1008A00043206E6F742063616C6962726174656469
:1008B000210D0A0000008F001E01AD013B02CA029B
:1008C0005803E603740402058F051B06A7063307C9
:1008D000BE074808D2085B09E3096B0AF20A780BE5
:1008E000FD0B810C040D860D070E870E060F840F7D
:1008F00000107B10F5106E11E5115B12CF12421340
:10090000B31323149214FE146A15D3153B16A116C3
:1009100005176717C81727188318DE1837198E1997
:10092000E319361A871AD61A231B6E1BB61BFD1B3A
:10093000411C831CC31C001D3C1D751DAB1DE01D0F
:10094000121E421E6F1E9A1EC31EE91E0D1F2E1F71
:100950004D1F691F841F9B1FB01FC31FD31FE11FA3
:10096000EC1FF51FFB1FFF1F00200A0D7777772E66
:100970004D696B726F4B6F707465722E64652028C1
:10098000632920486953797374656D7320476D62DC
:1009900048000A0D74686520757365206F662074C1
:1009A00068697320736F667477617265206973205C
:1009B0006F6E6C79207065726D6974746564200A5D
:1009C0000D6F6E206F726967696E616C204D696B87
:1009D000726F4B6F707465722D48617264776172CB
:1009E00065005573657200486F54542056330041BA
:1009F00043542044534C004A657469005370656B3E
:100A00007472756D0050504D000A0D526563656932
:100A10007665723A2000756E6B6E6F776E2E20557C
:100A200073696E672050504D2E2E2E006E6F74200D
:100A3000737570706F72746564206279206861727A
:100A4000647761726521000A0D466C6967687443BA
:100A50006F6E74726F6C0A0D4861726477617265B3
:100A60003A25642E25640A0D536F667477617265AA
:100A70003A5625642E2564256320000011241FBEEC
:100A8000CFEFD0E1DEBFCDBF11E0A0E0B1E0E2E109
:100A9000F1EF02C005900D92A63AB107D9F718E020
:100AA000A6EAB1E001C01D92AA3EB107E1F76AEAE9
:100AB000E2E0F0E081E2809357007491AE014F5F75
:100AC0005F4F20EF37EFDA019FE0F9012F5F3F4FD3
:100AD00084918D93915097FFF8CF773911F40000EE
:100AE000FECFFA019EE0819168276095915097FFB3
:100AF000FACF8889681721F0773911F40000FECF0A
:100B00000E9457060C9488780C94000080EF90E0C7
:100B10009F938F9387E891E19F938F93E091E403F4
:100B2000F091E50309950F900F900F900F900895A5
:100B300080912B06E82FFF27EE0FFF1FE35AF84F97
:100B4000808191818D5E9F4F14F01092020180810F
:100B500091818A5B9F4FCCF4809102018823A9F494
:100B600081E080930201809118048F5F80931804C4
:100B7000853038F088EE93E09093DB018093DA01C2
:100B800004C066E970E00E946A35809118049927D4
:100B90009093B0058093AF0508951F93CF93DF9393
:100BA000182F882389F086E191E09F938F9387E83F
:100BB00091E19F938F93E091E403F091E503099510
:100BC0000F900F900F900F9080914E06823308F097
:100BD00044C084EF91E00E949615EC01112329F0A6
:100BE000CE010E949F158823D9F3C2E0D0E026E50C
:100BF00030E080911D0190911E018217930730F023
:100C00002196255D3F4FC730D10598F380914E0660
:100C10009927C89F9001C99F300DD89F300D11248E
:100C2000209300011123D9F068EC70E08C2F0E9412
:100C30006A35DF93CF938EE191E09F938F9387E89E
:100C400091E19F938F93E091E403F091E50309957F
:100C50008DB79EB706968DBF02C080930001112309
:100C600011F1809100016AE00E94DB77892F9927BA
:100C70009F938F93809100010E94DB7799279F9328
:100C80008F9389E291E09F938F9387E891E19F93FF
:100C90008F93E091E403F091E50309952DB73EB7FA
:100CA000285F3F4F2DBFDF91CF911F910895CFEF68
:100CB000D0E1DEBFCDBF8824992414B815B8B7EEB3
:100CC000EB2EB3E0FB2E2EEC3FEFE20EF31EF7FE11
:100CD000FACF189B06C0199B02C08DE007C08BE0BD
:100CE00005C0199B02C084E101C08AE08093010124
:100CF00081E887B93E9A8FEF88B98BE184B981E0AA
:100D000085B98EE38AB987E48BB9469A84B7877F21
:100D100084BF8091600088618093600010926000C1
:100D200084EC99E09093DB018093DA011092E60263
:100D30001092E50210926207109261071092E80289
:100D40001092E7021092EA021092E902209101014A
:100D5000243128F084EC94E0A0E0B0E004C08BE003
:100D600095E0A0E0B0E08093420190934301A0930E
:100D70004401B09345012A3011F0243110F0289835
:100D800001C0289A0E94FF150E94D0150E948F1161
:100D90000E94A7310E94AD1981E00E940A2D0E9495
:100DA00021630E94526C0E948474809101018C30F6
:100DB00010F4299A01C0299878940E94292C8091D6
:100DC0002102826080932102109224020E949A40A4
:100DD00084EF91E00E9496157C018091210280FDB4
:100DE00005C0C7010E949F158823B9F38DE391E0E8
:100DF0009F938F93A7E8AA2EA1E1BA2EBF92AF923C
:100E0000E091E403F091E503099580EA9FE00E94F8
:100E100096157C01C0E0D0E00F900F900F900F90DE
:100E20000FEF16E0F3EBCF2EF6E0DF2E0E949A4094
:100E30008091210280FD05C0C7010E949F15882373
:100E4000B9F3F60180811816ACF40BC00E949A40E9
:100E50008091210280FD05C0C7010E949F15882353
:100E6000B9F3C7010E949F15882321F4F8018081FE
:100E7000882364F7F801808187FF19C02196DF93EA
:100E8000CF9321978FE491E09F938F93BF92AF927E
:100E9000E091E403F091E50309958091A7018F5F4C
:100EA0008093A7012DB73EB72A5F3F4F2DBF2196F4
:100EB00084E090E0C80ED91E085F1F4FCC30D105EA
:100EC00008F4B4CFC0E0D0E00CEF16E0E3EBEE2E78
:100ED000E6E0FE2EF801838187FD1DC0F7018081C9
:100EE0001816CCF42196DF93CF93219782E591E0F9
:100EF0009F938F9387E891E19F938F93E091E40311
:100F0000F091E503099582E08093D8012DB73EB7B3
:100F10002A5F3F4F2DBFF80183818078838321961C
:100F200024E030E0E20EF31E085F1F4FCC30D10505
:100F300088F20E948605909129068091A701981752
:100F400028F48091FE0380618093FE0380E791E0A6
:100F50009F938F93C7E8D1E1DF93CF93E091E403B0
:100F6000F091E503099588EE93E00E9496157C01C7
:100F70000E94B3190F900F900F900F90C7010E941D
:100F80009F158823D9F380E991E09F938F93DF9396
:100F9000CF93E091E403F091E503099580E00E948E
:100FA0003936809101010F900F900F900F908A3089
:100FB00011F0843110F0289801C0289A80ED97E054
:100FC0009093DB018093DA0185E580931A048EE02B
:100FD00090E00E94512A9927182F00278FE090E077
:100FE0000E94512A080F111D1093AD010093AC010E
:100FF0008AE090E00E94512A9927182F00278BE061
:1010000090E00E94512A080F111D1093AB0100932C
:10101000AA010F5F1F4F39F08091AC019091AD0193
:101020008F5F9F4F41F41092AD011092AC0110926E
:10103000AB011092AA018091AA019091AB019F93FC
:101040008F938091AC019091AD019F938F9385E92F
:1010500091E09F938F93DF93CF93E091E403F0911E
:10106000E50309950E94021F88E893E190933D01F2
:1010700080933C01C1E0C09319048C2F0E94CD05E0
:10108000809151060E94D2730E94860580ED97E000
:101090000E9496157C018AEF90E00E94961583E0ED
:1010A000809387051092A601809197062DB73EB7D1
:1010B000285F3F4F2DBF84FF02C0C093AE018091D7
:1010C000B001882311F04798FECF8091DE0188237C
:1010D00009F429C280910F01882309F424C21092D7
:1010E000DE0180911804882319F00E94980502C03F
:1010F0000E94CA430E949A40209101012A3011F0B7
:10110000243110F0289801C0289A8091D9028823B0
:1011100031F08091D90281508093D9020EC0809124
:101120006F00806280936F0010925E0710925D07DF
:101130008091FE0388608093FE0380913C01909132
:101140003D01019790933D0180933C0180913C01CA
:1011500090913D01892B21F0809122028823C9F1D1
:1011600080913C0190913D01892BD9F40E94342D4E
:1011700085E090E090933D0180933C018091C10512
:101180009091C20501969093C2058093C10580910C
:10119000FE0381608093FE038091880582608093C6
:1011A000880580910701909108018F5F9F4FC1F4DE
:1011B0008091D8028823A1F088EA91E69093DB0120
:1011C0008093DA0180E890E0909308018093070112
:1011D00007C02A3011F0243110F0289801C0289A55
:1011E0000E943C758091DE01882309F09CC18091AA
:1011F0000D01882311F00E9416160E94D3110E943F
:10120000210DC7010E949F15882309F488C184E13C
:1012100090E0E80EF91E80912202882349F0809127
:10122000FE0382608093FE038091880582600FC078
:101230008091DA019091DB01892B59F480913C0176
:1012400090913D01079728F0809188058D7F8093CC
:1012500088058091AE01882361F08091D902873999
:1012600040F01092AE0188E893E19093DB01809307
:10127000DA0180910401882321F0815080930401D8
:101280002EC0809324041092AD021092AC021092F2
:10129000AB021092AA021092A9021092A8028091A9
:1012A000D9028823E1F480910701909108018F5FB2
:1012B0009F4FA9F42091AE01223089F088E99AE38A
:1012C0009093DB018093DA0180E09CE09093080129
:1012D00080930701222319F082E08093AE01809170
:1012E0009B01893C48F0815080939B018091FE03D3
:1012F0008B7F8093FE033FC080913E088823F9F0E6
:101300008091FE0384608093FE0389E08093B303A1
:1013100080910701909108018F5F9F4F81F4809128
:10132000D802882361F088E99AE39093DB018093E7
:10133000DA0180E098EA9093080180930701109207
:10134000A5031092A4031092A3031092A20310927B
:10135000A103109231081092700810926F08109239
:101360007208109271088FEF9FEF90936E08809330
:101370006D0810929B0180910001282F33278091E6
:101380001D0190911E0182179307CCF48091A10258
:1013900080628093A10280910701909108018F5F84
:1013A0009F4FC1F480E797E19093DB018093DA01CE
:1013B00080E093E090930801809307010BC0809137
:1013C000DA019091DB01892B29F48091A1028F7DB4
:1013D0008093A1020E94D86784E08093D901809114
:1013E000AF018F5F8093AF01813309F04FC010923E
:1013F000AF018091A10281FF0AC08091A801909164
:10140000A90101969093A9018093A8013FC05AEACF
:10141000852E55E0952E8091CE059091CF059C01AB
:10142000442737FD4095542F809115019091160166
:10143000A0911701B0911801281739074A075B07D7
:1014400034F48091CE059091CF0501961BC0809118
:10145000CE059091CF059C01442737FD4095542F30
:101460008091150190911601A0911701B09118017A
:1014700082179307A407B5074CF48091CE0590918D
:10148000CF0501979093CF058093CE050894811CDA
:10149000911C32E783163BE0930609F040C0882494
:1014A00099242091AC013091AD012F5F3F4F3093D3
:1014B000AD012093AC018091AA019091AB010196FE
:1014C0009093AB018093AA01832F9927682F8EE018
:1014D00090E00E94592A8091AC019091AD019070EA
:1014E000682F8FE090E00E94592A8091AA01909184
:1014F000AB01892F9927682F8AE090E00E94592A32
:101500008091AA019091AB019070682F8BE090E0E0
:101510000E94592A84E190E00E9496157C010E9465
:1015200028680E94696C8091D901882309F0C7CD91
:101530000E944263C4CD1F920F920FB60F921124E6
:101540008F939F93EF93FF93809106018823E1F49B
:101550008091CA019091CB0101969093CB01809329
:10156000CA01FC01E852FB4FE081ED3019F08F3ADF
:10157000910539F41092CB011092CA0181E0809359
:101580000601E093C60004C01092CB011092CA017C
:10159000FF91EF919F918F910F900FBE0F901F9031
:1015A00018951F920F920FB60F9211242F933F930D
:1015B0004F935F936F937F938F939F93AF93BF935B
:1015C000CF93EF93FF9390E08091B001813029F4A5
:1015D0008091C6008093CE00CCC08091B001823053
:1015E00029F48091C60080932704C3C08091C6006F
:1015F0008093C2015091D0015F3A10F09093D101D5
:101600008091C2018D3009F065C08091D101823096
:1016100009F060C09093D101852F9927895D9B4F78
:10162000FC01329740812091CC013091CD01241BE7
:101630003109DC0111978C91281B3109C9019F7078
:101640009093CD018093CC0146E0969587954A957D
:10165000E1F7982F935C9093CE012F733070235C49
:101660002093CF018081981729F48C91281711F4C9
:1016700091E006C090E08091BF018F5F8093BF0131
:10168000C091C101CC2309F074C0992309F471C041
:1016900081E08093C101580F5093BE015150E52F56
:1016A000FF27E95DFB4F8DE080838091290482351F
:1016B00009F05FC00E94021F88E190E02CE00FB6A5
:1016C000F894A895809360000FBE20936000C093AB
:1016D000D8014FC02091D101822F992781309105E7
:1016E000F9F0823091051CF4892B21F040C002975B
:1016F00011F13DC08091C201833239F48091C10162
:10170000882319F481E08093D1018091C2018093F4
:10171000270481E08093D0018091C201992722C0E3
:101720002F5F2093D101E52FFF27E95DFB4F8091CB
:10173000C201808309C0E52FFF27E95DFB4F80913F
:10174000C20180835F3A20F45F5F5093D00102C0F2
:101750001092D1012091C2018091CC019091CD01D4
:10176000820F911D9093CD018093CC0102C0109205
:10177000D101FF91EF91CF91BF91AF919F918F9147
:101780007F916F915F914F913F912F910F900FBE7D
:101790000F901F901895AC01A0E0B0E09D01A81734
:1017A000B90748F4E8EDF4E08191280F311D119656
:1017B000A417B507C8F33F70FD01E852FB4FC901FC
:1017C00056E0969587955A95E1F7835C808311964C
:1017D000FD01E852FB4F2F733070822F835C8083B2
:1017E000A752BB4F8DE08C93109206018091D804D4
:1017F0008093C6000895A0E0B0E0E1E0FCE00C9426
:1018000054782C859D850E85BB2483E28093D80473
:101810009F599093D9042093DA0433E0E32EF12CFE
:10182000002309F49EC0CF84D888BE016D5E7F4F2F
:10183000A989BA890150109709F493C01097B9F09B
:10184000F601EB0DF11DB3949081119791F40023F3
:1018500049F1FB016E5F7F4FDB01C080D1806E5F7D
:101860007F4F0D90BC91A02DBB24015002C090E091
:1018700019C01097B9F0F601EB0DF11DB39440813A
:10188000119791F4002341F1FB016E5F7F4FDB0163
:10189000C080D1806E5F7F4F0D90BC91A02DBB2486
:1018A000015002C040E018C01097B1F0F601EB0DF6
:1018B000F11DB3941081119781F4002371F0FB01A5
:1018C0003296DB01CD90DC90BF016E5F7F4FA0812F
:1018D000B181BB24015001C010E0F701E852FB4F79
:1018E000892F86958695835C80830894E11CF11C82
:1018F000F701E852FB4F892F99278370907024E0FD
:10190000880F991F2A95E1F755279A0194E036959B
:1019100027959A95E1F7822B835C80830894E11CDC
:10192000F11CF701E852FB4F4F705070440F551FE8
:10193000440F551F812F992726E0969587952A9564
:10194000E1F7842B835C80830894E11CF11CF70190
:10195000E852FB4F1F73135C10830894E11CF11CC9
:101960006ACFC7010E94CB0BE9E00C947078A3E02A
:101970007A2F4091BE014650442309F458C0E72F06
:10198000FF27E95DFB4F80818D537F5FE72FFF27A6
:10199000E95DFB4F20812D537F5FE72FFF27E95D36
:1019A000FB4F30813D537F5FE72FFF27E95DFB4F02
:1019B00060816D537F5F9927880F991F880F991F4A
:1019C000522F52955F70582B822F99278F709070ED
:1019D000F4E0880F991FFA95E1F7232F26952695B5
:1019E000282B832F992783709070E6E0880F991F2A
:1019F000EA95E1F7682B41504F3FC9F0EA2FFF27E6
:101A0000E95DFB4F5083AF5F41504F3F81F0EA2FBC
:101A1000FF27E95DFB4F2083AF5F41504F3F39F017
:101A2000EA2FFF27E95DFB4F6083AF5FA5CF8AE216
:101A300094E09093BD018093BC01A350A093BB019F
:101A40000895A2E0B0E0E7E2FDE00C945A788091BE
:101A5000C101882309F457C40E94B70C809128045F
:101A6000823609F023C38091290499278037910594
:101A700009F4AFC081379105C4F48A36910509F4A1
:101A800080C28B36910544F48B34910571F1863612
:101A9000910509F45FC10AC38D36910509F469C047
:101AA0008E36910509F44DC001C38437910541F18B
:101AB000853791054CF48137910509F491C083373E
:101AC000910509F4DFC0F2C28737910509F41BC202
:101AD000883791052CF48537910509F4D7C1E6C202
:101AE0008937910509F46DC1E1C2E091BC01F09123
:101AF000BD018081918190938F0180938E01D6C228
:101B00008091BE01A091BC01B091BD01853140F032
:101B100080E1E2E0F4E00D9001928A95E1F70DC0DA
:101B20008D919D910D90BC91A02D80930204909376
:101B30000304A0930404B093050480EF8093B901DB
:101B40004BC0809106018823E1F38DE490E09F93E0
:101B50008F9386EA96E09F938F9381E08F938F9384
:101B60008EE48F930E94FB0B8DB79EB707968DBFB7
:101B70009DC2A091BC01B091BD011C91113081F4B6
:101B80008DE4E6EAF6E00D9001928A95E1F70E9475
:101B9000662B19838091FE038F7E8093FE0301C024
:101BA0001982809106018823E1F381E090E09F9300
:101BB0008F93CE0101969F938F9381E08F938F93A4
:101BC0008DE48F930E94FB0BADB7BEB71796ADBFE8
:101BD0006DC281E08093C4018FEF8093040166C2DF
:101BE000E091BC01F091BD01E0818E2F8A508A30D6
:101BF00058F48983882311F481E003C0863010F003
:101C000085E0898361E00EC08E2F84518A3070F4A4
:101C10008983882311F481E003C0863010F085E0C9
:101C2000898360E089810E94E62B12C0E983EF3F3F
:101C300019F40E94C92B89838981882311F481E0DA
:101C400003C0863010F085E0898389810E946F2A65
:101C5000809106018823E1F38BE790E09F938F93B7
:101C60008AE296E09F938F9381E090E09F938F9319
:101C7000CE0101969F938F9382E08F9381E08F93A3
:101C800081E577C12091BC013091BD01D9018C91D2
:101C90008150853008F045C0F90181818A3509F00D
:101CA00040C08091D8028823E1F52F5F3F4F8BE73A
:101CB000EAE2F6E0D9010D9001928A95E1F7F90187
:101CC00082910E94D82A80916B069927AA27BB2768
:101CD000BC01CD0124EC39E040E050E00E94BC772B
:101CE000DC01CB018093860190938701A09388014A
:101CF000B093890180916C069927AA27BB27BC0164
:101D0000CD010E94BC77DC01CB01809382019093CE
:101D10008301A0938401B09385010E94C92B89831C
:101D200001C01982809106018823E1F381E090E0EF
:101D30009F938F93CE0101969F938F9381E08F9312
:101D40008F9383E58F930E94FB0B8DB79EB7079609
:101D50008DBF26C0E091BC01F091BD01E0818E2FC6
:101D60008150853018F48E2F0E946F2A0E94C92B53
:101D70008983809106018823E1F381E090E09F93BD
:101D80008F93CE0101969F938F9381E08F938F93D2
:101D900086E48F930E94FB0BADB7BEB71796ADBF1D
:101DA0008091D802882329F46EE670E089810E9430
:101DB0006A3580E00E94CD05809151060E94D27361
:101DC00075C1E091BC01F091BD018081992787FD2B
:101DD000909590937807809377078181992787FD65
:101DE000909590937A07809379078281992787FD50
:101DF000909590937C0780937B078381992787FD3B
:101E0000909590937E0780937D078481992787FD25
:101E100090959093800780937F078581992787FD10
:101E2000909590938207809381078681992787FDFB
:101E3000909590938407809383078781992787FDE6
:101E4000909590938607809385078085992787FDD5
:101E5000909590938807809387078185992787FDC0
:101E6000909590938A07809389078285992787FDAB
:101E7000909590938C0780938B078385992787FD96
:101E8000909590938E0780938D0710C1E091BC01CF
:101E9000F091BD0180810E9400318A83882319F46A
:101EA00081E0898301C01982809106018823E1F3D2
:101EB00088E090E09F938F9384EF96E09F938F93B9
:101EC00021E030E03F932F938091BC019091BD01C0
:101ED0009F938F933F932F93CE0102969F938F935F
:101EE0003F932F93CE01820F931F9F938F9384E094
:101EF0008F9381E08F9385E58F930E94FB0BEDB765
:101F0000FEB773963CC08091BB01893008F4CEC007
:101F10002091BC013091BD012F5F3F4F88E0A4EFBD
:101F2000B6E0F90101900D928A95E1F7D9018E9101
:101F30000E9456308A83882319F481E0898301C086
:101F40001982809106018823E1F321E030E03F937C
:101F50002F93CE0102969F938F933F932F93CE01A1
:101F6000820F931F9F938F9382E08F9381E08F93D3
:101F700087E58F930E94FB0BEDB7FEB73B96EDBF55
:101F800095C08091D802882309F090C00E94857383
:101F90008983823019F0843009F088C020E430E071
:101FA000F8948091C1008F738093C1008091C90023
:101FB0008F738093C9008091C100877E8093C10098
:101FC0008091C900877E8093C9008091C80087FFF7
:101FD00003C08091CE00F9CF8091C00087FF03C07D
:101FE0008091C600F9CFE091BC01F091BD01E08184
:101FF000E13021F482E08093B0012EC0E43611F488
:1020000021E830E081E08093B001832F992780930D
:10201000CD002093CC008091CD008093C5008091AD
:10202000CC008093C4008091CA008F7D8093CA0049
:102030008091CA008F7E8093CA008091C9008B7FF7
:102040008093C9008091CA0084608093CA00809107
:10205000CA0082608093CA008091CA00877F809303
:10206000CA008091C200877F8093C2008091C9001E
:102070008E7F8093C9008091C10088618093C100E8
:102080008091C90088618093C9008091C1008068F7
:102090008093C1008091C90080688093C90010922C
:1020A0006E0010926F001092700078948091290455
:1020B00099278436910509F4BBC085369105ACF4A7
:1020C0008136910509F46FC0823691052CF48B346A
:1020D000910509F45DC00FC18236910509F470C005
:1020E0008336910509F47FC006C18C36910509F449
:1020F000EDC08D3691054CF48736910509F4F8C092
:102100008836910509F4B2C0F6C08437910529F0EC
:102110008637910509F4E8C0EEC08091BE01A09118
:10212000BC01B091BD01803140F080E1E2E0F4E01B
:102130000D9001928A95E1F70DC08D919D910D90C2
:10214000BC91A02D8093020490930304A0930404F7
:10215000B0930504809106018823E1F31F928091DA
:1021600003018F9384E58F930E94FB0B8AEF80938A
:10217000B9018FEF8093040180EA9FE00E949615D9
:102180009093B2018093B1010F900F900F90B3C064
:10219000E091BC01F091BD018081918190938F010C
:1021A00080938E01A8C0E091BC01F091BD018081B7
:1021B00080930501803298F08FE1809305010FC074
:1021C000A091BC01B091BD018BE0EAE1F4E00D907B
:1021D00001928A95E1F7809123048093C9058FEFDE
:1021E0008093040188C08091B5019091B601892B3C
:1021F00089F4E091BC01F091BD01E081EE2351F042
:102200008AE0E89FC00111240E9496159093F5037F
:102210008093F403E091BC01F091BD0190818AE0CC
:10222000989FC00111249093B6018093B50115C009
:102230008FEF80930401E091BC01F091BD0190818A
:102240008AE0989FC00111249093B8018093B70150
:10225000892B19F081E08093C60180EA9FE00E94FB
:1022600096159093B2018093B10145C08FEF809392
:102270000401E091BC01F091BD01908197FD08C07F
:1022800082E08093C3011092B4011092B3011AC08E
:10229000909580911A02892B80931A0291818AE08D
:1022A000989FC00111249093B4018093B30184E0FE
:1022B0008093C30180EA9FE00E9496159093B2013B
:1022C0008093B10181E08093C70115C08FEF8093A7
:1022D0000401E091BC01F091BD01808180931B025B
:1022E00081E08093C80107C081E08093C50103C0ED
:1022F00081E08093C9011092C1011092BD0110923A
:10230000BC011092BB01E3E0CE5F0C947678982F6D
:102310008091C00085FFFCCF9093C60008950F9375
:102320001F9388E18093C1008091C00082608093F8
:10233000C0008091C10080688093C1008091C1007D
:1023400080648093C10000E010E00093C5008AE241
:1023500090E08093C4008091B7019091B8010E94F1
:1023600096159093F7038093F6038CED90E00E940E
:10237000961590932604809325041092F80388E51F
:102380008093F90384E08093FC038BE08093FA034D
:102390001092FB031093BD010093BC011092BB018E
:1023A0001F910F910895A0E1B0E0E9EDF1E10C94E7
:1023B000577880910601882309F4C1C28091B10148
:1023C0009091B2010E949F15882361F01092B40190
:1023D0001092B3011092B8011092B7011092B60199
:1023E0001092B5018091B3019091B401892B41F015
:1023F0008091D6049091D7040E949F15882329F4D8
:102400008091C701882309F460C080910601882368
:1024100009F45BC08091C30109ED15E08430A8F098
:102420000E94181F80E590E09F938F931F930F9356
:1024300081E08F938F9388E48F930E94FB0B2DB7DD
:102440003EB7295F3F4F2DBF34C010921C0287EB6F
:1024500093E09F938F938BE09FE19F938F93E09105
:10246000E403F091E503099584E190E09F938F9355
:102470001F930F9381E090E09F938F9383EC91E003
:102480009F938F9382E08F9381E08F9388E48F9363
:102490000E94FB0B8091C301982F8F5F8093C30133
:1024A0002DB73EB7215F3F4F2DBF943010F01092F3
:1024B000C3018091B3019091B4010E94961590934D
:1024C000D7048093D6041092C7018091C801882355
:1024D00051F180910601882331F10E94181F80E597
:1024E00090E09F938F9389ED95E09F938F9321E0E8
:1024F00030E03F932F938FE191E09F938F933F9331
:102500002F938BE192E09F938F9383E08F9381E0F1
:102510008F938CE48F930E94FB0B1092C8018DB7B0
:102520009EB70F968DBF8091C5018823D1F0809111
:1025300006018823B1F08AE090E09F938F9388EFA3
:1025400093E09F938F9381E08F938F9386E58F9392
:102550000E94FB0B1092C5012DB73EB7295F3F4F7C
:102560002DBF8091C9018823D9F08091060188236D
:10257000B9F08BE090E09F938F938AE194E09F9372
:102580008F9381E08F93809103018F9387E48F93E2
:102590000E94FB0B1092C9018DB79EB707968DBFA5
:1025A00080912504909126040E949F15882309F4A8
:1025B00061C080910601882309F45CC080914606C1
:1025C0009927880F991F880F991F7C010027F7FC16
:1025D0000095102F8091330390913403A09135031F
:1025E000B0913603BC01CD01A80197010E9430785B
:1025F000309313042093120480912B0390912C03A9
:10260000A0912D03B0912E03BC01CD01A80197012B
:102610000E94307830931504209314048091B60200
:10262000809316048091B5028093170488E090E0AF
:102630009F938F9382E194E09F938F9381E08F9398
:1026400083E08F938BE68F930E94FB0B809118049D
:102650002DB73EB7295F3F4F2DBF853018F086E07C
:102660008093180483E690E00E94961590932604C8
:10267000809325048091B7019091B801892B41F096
:102680008091F6039091F7030E949F15882321F40F
:102690008091C601882339F180910601882319F1C0
:1026A0000E94543482E490E09F938F9387E895E0F2
:1026B0009F938F9381E08F938F9384E48F930E94F5
:1026C000FB0B1092C6018DB79EB707968DBF809108
:1026D000B7019091B801009731F00E949615909340
:1026E000F7038093F6038091B5019091B601892B91
:1026F00009F4B8C08091F4039091F5030E949F15EE
:10270000882309F4AFC080910601882309F4AAC088
:10271000809146069927880F991F880F991F7C0181
:102720000027F7FC0095102F80913303909134031C
:10273000A0913503B0913603BC01CD01A8019701EA
:102740000E9430783093E7032093E60380912B03B7
:1027500090912C03A0912D03B0912E03BC01CD01CB
:10276000A80197010E9430783093E9032093E80391
:102770002091260830912708409128085091290877
:10278000DA01C90163E0880F991FAA1FBB1F6A9570
:10279000D1F7820F931FA41FB51F820F931FA41F91
:1027A000B51F209142013091430140914401509165
:1027B0004501BC01CD010E9430783093EB0320939A
:1027C000EA038091FB029091FC02A091FD02B0917E
:1027D000FE0249E0B595A795979587954A95D1F75B
:1027E0008093EC038091F7029091F802A091F90296
:1027F000B091FA0239E0B595A795979587953A95E6
:10280000D1F78093ED038091030390910403A0918D
:102810000503B091060329E0B595A795979587958F
:102820002A95D1F78093EE038EE090E09F938F93EB
:1028300086EE93E09F938F9381E08F938F9383E451
:102840008F930E94FB0B8091B5019091B6010E947D
:1028500096159093F5038093F4032DB73EB7295F47
:102860003F4F2DBF809105018F3F71F1992704E003
:10287000880F991F0A95E1F789549E4F40E150E077
:10288000BC01CE0101960E940F7680E190E09F93FB
:102890008F93CE0101969F938F9381E090E09F9359
:1028A0008F9385E091E09F938F9382E08F9381E0F7
:1028B0008F9381E48F930E94FB0B8FEF8093050130
:1028C0008DB79EB70B968DBF8091C9058823D1F037
:1028D000809106018823B1F081E090E09F938F936F
:1028E00089EC95E09F938F9381E08F938F9382E49F
:1028F0008F930E94FB0B1092C9052DB73EB7295F3D
:102900003F4F2DBF8091C4018823C9F080910601FB
:102910008823A9F084E390E09F938F938DE597E05F
:102920009F938F9381E08F938F9380E58F930E9485
:10293000FB0B1092C4018DB79EB707968DBFE6E0E2
:10294000C05F0C9473781F920F920FB60F921124F0
:102950002F933F935F936F937F938F939F93AF9347
:10296000BF93EF93FF9320E08091D901882329F052
:102970008091D90181508093D9018091C603882329
:1029800019F081508093C6038091E10181508093BA
:10299000E1018F3F09F05BC089E08093E101809104
:1029A000DF019091E00101969093E0018093DF01B7
:1029B00080910E018F5F817080930E01882319F43E
:1029C00081E08093DE01349903C081E08093E201CD
:1029D0008091DA019091DB01892B21F18091DA015C
:1029E0009091DB010B9750F08091DA019091DB011F
:1029F0000A979093DB018093DA0104C01092DB0107
:102A00001092DA018091DA019091DB0120910701A7
:102A10003091080182239323892B11F021E008C013
:102A200020E006C08FEF9FEF90930801809307018D
:102A300080910101222331F08A3011F45A9A07C0A3
:102A4000479A05C08A3011F45A9801C0479880917E
:102A5000E201882309F45AC020919B01222309F046
:102A600055C08091160883FF51C086B19927FC019B
:102A7000E071F07084FF13C08091DC019091DD0162
:102A800001969093DD018093DC018091DC019091AF
:102A9000DD01895E9340D0F12093E20137C080913F
:102AA000DC019091DD01892B69F18091DC0190912D
:102AB000DD018A56914030F58091DC019091DD0175
:102AC00069E270E00E94E7778091DC019091DD017E
:102AD000860F971F9093DD018093DC018091DC01CC
:102AE0009091DD010B9750F08091DC019091DD0118
:102AF0000A9790938F0180938E0104C0F0938F0109
:102B0000E0938E011092DD011092DC01FF91EF91B4
:102B1000BF91AF919F918F917F916F915F913F9105
:102B20002F910F900FBE0F901F9018952091DF01ED
:102B30003091E001280F391FC901019608952091B5
:102B4000DF013091E001821B930B892F9927869535
:102B5000807490700895CF93DF930E949615EC01D6
:102B6000CE010E949F158823D9F3DF91CF9108955C
:102B7000CF93DF930E949615EC0109C080910F015D
:102B8000882329F090930F018FEC80937A00CE0177
:102B90000E949F15982F882389F3DF91CF91089584
:102BA0009FB7F8945F983E9A469A8091B0008F70D4
:102BB0008093B0008091B00083608093B0008091DA
:102BC000B1008B738093B1008091B1008B608093D2
:102BD000B1001092B2008FEF8093B3008091B000EB
:102BE00080688093B000809170008A7F809370002D
:102BF000809170008260809370009FBF08958AE08A
:102C000090E00E9496159093E8018093E70182E09E
:102C100085BD83EA84BD17BC84EB88BD86E086BD94
:102C200080916E00816080936E000895A0E0B0E016
:102C3000ECE1F6E10C94567880916106E82FFF27CD
:102C4000E85BFE4F9681D08080910D01A92FBB27B4
:102C5000A7FDB095CB2FDB2F813009F012C1209159
:102C60003303309134034091350350913603BD0155
:102C7000CE010E94BC7797FF04C061587F4F8F4FF1
:102C80009F4F7B018C0187E015950795F794E7949A
:102C90008A95D1F78D2D992787FD9095A92FB92F6A
:102CA00020912B0330912C0340912D0350912E0342
:102CB000BC01CD010E94BC7797FF04C061587F4FD3
:102CC0008F4F9F4FC7E09595879577956795CA95E4
:102CD000D1F7F801E701C61BD70BE80BF90B2091E0
:102CE000AC033091AD03C901B3E0880F991FBA95C9
:102CF000E1F7821B930BAA2797FDA095BA2FC81B5B
:102D0000D90BEA0BFB0B809158069927AA27BB2702
:102D1000BC01CD019E01AF010E94BC7797FF04C0AA
:102D200061507E4F8F4F9F4FFC01EB01A9E0F5955D
:102D3000E795D795C795AA95D1F780916D01992709
:102D400076E0880F991F7A95E1F740910B01509139
:102D50000C01209160063327841B950BB9010E945A
:102D6000FB7780910B0190910C01860F971F909338
:102D70000C0180930B018091960680FF14C0809116
:102D80000B0190910C0197FD0F9664E09595879546
:102D90006A95E1F7AA2797FDA095BA2FC80FD91F0A
:102DA000EA1FFB1F15C080910B0190910C0197FD4C
:102DB0000F9654E0959587955A95E1F7AA2797FDC8
:102DC000A095BA2F8C1B9D0BAE0BBF0BFD01EC0128
:102DD00020919306222321F133278091D4019091F1
:102DE000D501829FA001839F500D929F500D112409
:102DF000CA01AA2797FDA095BA2F8C0F9D1FAE1F61
:102E0000BF1F2F5F3F4F442737FD4095542FBC0114
:102E1000CD010E9430783093D5012093D40104C0B5
:102E2000D093D501C093D40180915906282F332720
:102E3000220F331F220F331F8091D4019091D501AF
:102E4000821793077CF080915A06282F3327220F90
:102E5000331F220F331F8091D4019091D501281781
:102E6000390724F43093D5012093D40180910101D6
:102E7000843108F4F7C080910D018F5F80930D01BC
:102E8000F3C020912B0330912C0340912D035091DE
:102E90002E03BD01CE010E94BC7797FF04C061588C
:102EA0007F4F8F4F9F4F7B018C0187E015950795D2
:102EB000F794E7948A95D1F78D2D992787FD909502
:102EC000A92FB92F2091330330913403409135035A
:102ED00050913603BC01CD010E94BC779B01AC012F
:102EE00097FF04C021583F4F4F4F5F4FC7E05595A4
:102EF000479537952795CA95D1F72E0D3F1D401F51
:102F0000511F80915C069927AA27BB27BC01CD01E0
:102F10000E94BC7797FF04C061507E4F8F4F9F4F38
:102F2000FC01EB01B9E0F595E795D795C795BA9502
:102F3000D1F780916C019927A6E0880F991FAA9577
:102F4000E1F74091090150910A0120916006332771
:102F5000841B950BB9010E94FB7780910901909128
:102F60000A01860F971F90930A01809309018091AF
:102F7000960681FF14C08091090190910A0197FD86
:102F80000F9674E0959587957A95E1F7AA2797FDB6
:102F9000A095BA2FC80FD91FEA1FFB1F15C080913B
:102FA000090190910A0197FD0F9664E09595879528
:102FB0006A95E1F7AA2797FDA095BA2F8C1B9D0B68
:102FC000AE0BBF0BFD01EC0120919406222321F1F1
:102FD00033278091D2019091D301829FA001839FDA
:102FE000500D929F500D1124CA01AA2797FDA0955C
:102FF000BA2F8C0F9D1FAE1FBF1F2F5F3F4F44275F
:1030000037FD4095542FBC01CD010E94307830939C
:10301000D3012093D20104C0D093D301C093D20135
:1030200080915D06282F3327220F331F220F331F75
:103030008091D2019091D301821793077CF0809107
:103040005E06282F3327220F331F220F331F809154
:10305000D2019091D3012817390724F43093D3017A
:103060002093D20110920D01E7E0CDB7DEB70C94AA
:1030700072781F920F920FB60F9211242F933F93E5
:103080004F935F938F939F93EF93FF9380910101F1
:103090009091E301843108F04CC0992309F01CC1E0
:1030A0008091B00086FF24C08091B0008F7B809318
:1030B000B0008091D4019091D50187559E4F909397
:1030C000D7018093D60125E08D3D920718F08CED55
:1030D00095E005C08757914030F487E791E09093E1
:1030E000D7018093D6018091D6019091D701BAC0C3
:1030F0008091B00080648093B00080915F06282F9B
:1031000033278DED96E0289FA001299F500D389F11
:10311000500D1124CA012091E4013091E501821B78
:10312000930B9093D7018093D60181E080930D019A
:10313000D0C0992309F0D0C08091B00086FF97C01D
:103140008091B0008F7B8093B000E091E601EE2388
:10315000F1F480915F06282F33278DED96E0289FAC
:10316000A001299F500D389F500D1124CA012091B4
:10317000E4013091E501821B930B9093D70180937A
:10318000D6011092E5011092E401469AA2C089EAA4
:1031900093E09093D7018093D6018E2F99278330A7
:1031A0009105D9F08430910534F48130910549F0CE
:1031B000029761F020C08430910591F0059799F055
:1031C0001AC08091D4019091D50104C08091D201A0
:1031D0009091D30187559E4F1DC08091F20705C085
:1031E0008091CB0702C08091FB079927880F991F18
:1031F000880F991FEFCFFF27EE0FFF1FE35AF84FFD
:1032000020813181220F331F8091D6019091D70107
:10321000820F931F9093D7018093D6018091D6019E
:103220009091D70155E08D3D950718F08CED95E014
:1032300005C08757914030F487E791E09093D7011C
:103240008093D6012091D6013091D7012C5B30407C
:103250003093D7012093D6018091E4019091E5014C
:10326000820F931F9093E5018093E40132C0809117
:10327000B00080648093B0008CEB90E09093D70115
:103280008093D6018091E4019091E50184549F4F91
:103290009093E5018093E4018091D801882321F087
:1032A0008091D902882321F48091D801823011F4D1
:1032B000469801C0469A8091E6018F5F8093E601AF
:1032C00090915F06981728F481E080930D01109289
:1032D000E60181E08093E3012091D6013091D7018E
:1032E00041E02F37340730F08FEF8093B3002F5F2A
:1032F00030400FC02F3F3105C9F0C0F0A9014F5F2A
:1033000050404F37510550F480E88093B300205867
:1033100030403093D7012093D60112C08FEF8093B5
:10332000B3005093D7014093D6010AC08091D601D3
:103330008093B3001092D7011092D6011092E3014E
:10334000FF91EF919F918F915F914F913F912F91BD
:103350000F900FBE0F901F90189510927C008FEC6D
:1033600080937A000895CF93DF931092ED0183E06C
:1033700090E00E94512AC82FDD27C531D10508F001
:103380002A97C7BD84E690E00E94B815809113018A
:10339000909114018052934010F4C0E0D0E0CA3FF5
:1033A000D105F8F4C7BD82E390E00E94B8158CEC1B
:1033B00093E09F938F9387E891E19F938F93E091A0
:1033C000E403F091E50309958091130190911401B4
:1033D0000F900F900F900F908052934010F0219615
:1033E000DECFC093D6056C2F83E090E00E94592A6F
:1033F0008091370680FF0AC08091D6058A508B3EA7
:1034000028F08091FD0380648093FD03C7BD8CE2AA
:1034100091E00E94B815DF91CF910895EF92FF924D
:103420001F93CF9310E080ED97E00E9496157C01EA
:10343000CCE8133019F4CB3008F0C9E010E08091EB
:10344000FC019091FD018C5F934024F48091120166
:1034500081500AC08091FC019091FD0187509440F9
:1034600034F0809112018F5F8093120101C011E04E
:103470008091FA019091FB018C5F934024F480913C
:10348000110181500AC08091FA019091FB0187508F
:10349000944034F0809111018F5F8093110101C03D
:1034A0001F5F8091F8019091F9018C5F934024F4A3
:1034B0008091100181500AC08091F8019091F9012A
:1034C00087509440C4F0809110018F5F8093100169
:1034D00013C08EEC93E09F938F9387E891E19F93C5
:1034E0008F93E091E403F091E50309950F900F901D
:1034F0000F900F905FC01F5F82E180932702809141
:1035000021028E7F8093210285EA8093BC00809106
:1035100012018A3040F48091FD0381608093FD03A5
:103520008AE08093120180911201863F40F08091E1
:10353000FD0381608093FD0385EF809312018091EC
:1035400011018A3040F48091FD0382608093FD0375
:103550008AE08093110180911101863F40F08091B3
:10356000FD0382608093FD0385EF809311018091BC
:1035700010018A3040F48091FD0384608093FD0344
:103580008AE08093100180911001863F40F0809185
:10359000FD0384608093FD0385EF8093100180918B
:1035A0002702882339F0C7010E949F15882309F05C
:1035B00090CFF5CF10920F018FEC80937A0080911D
:1035C0000F018823E1F3CA3020F48AE090E00E94E2
:1035D000B815C15009F02DCF86E490E00E94B815CF
:1035E000CF911F91FF90EF9008951F920F920FB609
:1035F0000F921124EF92FF920F931F932F933F93FB
:103600004F935F936F937F938F939F93AF93BF93EA
:10361000EF93FF9380910502282F332744275527E6
:103620008F5F80930502F9012231310508F0C5C38F
:10363000E25CFF4F0C948278809178009091790041
:1036400046C0809178009091790029C180917800DE
:1036500090917900909308028093070254C1809161
:103660003C0390913D032091780030917900821BBA
:10367000930B9093CB058093CA058091CA059091D6
:10368000CB0590931202809311025BC18091780068
:103690009091790020913E0330913F03821B930B60
:1036A0009093D5058093D4058091D4059091D5054C
:1036B000909314028093130282C380910B02909125
:1036C0000C022091780030917900820F931F909323
:1036D0000C0280930B0281E073C3809109029091E8
:1036E0000A022091780030917900820F931F909305
:1036F0000A028093090284E063C380911D019091C6
:103700001E019C01220F331F280F391F8091780062
:103710009091790063E070E00E94E777260F371FF1
:10372000369527953695279530931E0120931D01D8
:1037300085E046C3809178009091790040913803EC
:1037400050913903841B950B9093F3018093F20100
:103750008091F2019091F301029704F122E04E3E34
:10376000520784F4209106022B5F20930602255015
:103770008091A2029091A302845F914018F4215F8E
:103780002093060280910602853684F14F5F5F4FD9
:103790005093390340933803845626C08091F20138
:1037A0009091F3018F5F9F4F0CF532E04732530742
:1037B000ECF0209106022550209306022B5F8091A9
:1037C000A2029091A302845F914018F42F5020939D
:1037D0000602809106028C394CF4415050405093BF
:1037E0003903409338038C59809306028091780006
:1037F000909179009093CD058093CC058091F20152
:103800009091F3019C01442737FD4095542F8091FE
:10381000F3029091F402A091F502B091F602820FAA
:10382000931FA41FB51F8093F3029093F402A093FB
:10383000F502B093F6022091F3023091F402409128
:10384000F5025091F60257FF04C021503C4F4F4FF4
:103850005F4F6AE055954795379527956A95D1F75B
:103860008091F3029091F402A091F502B091F602DA
:10387000821B930BA40BB50B8093F3029093F4027D
:10388000A093F502B093F6022EC1809109029091A7
:103890000A022091780030917900820F931F909353
:1038A0000A0280930902109204028CC280910101E5
:1038B0008A3071F48091780090917900209107020C
:1038C00030910802820F931F01969695879517C035
:1038D0004091070250910802843158F020917800FD
:1038E00030917900240F351F8FEF97E0821B930BE7
:1038F00006C08091780090917900840F951F909375
:10390000F9018093F80186E05BC280913C039091BD
:103910003D032091780030917900821B930B9093A6
:10392000CB058093CA058091CA059091CB05209163
:10393000110230911202820F931F9093F70180932E
:10394000F60187E03DC28091780090917900209146
:103950003E0330913F03821B930B9093D5058093D8
:10396000D4058091D4059091D50520911302309112
:103970001402820F931F9093F5018093F4011FC2EC
:1039800020910B0230910C02809178009091790087
:10399000280F391F30930C0220930B0280910101F4
:1039A0008A3019F4220F331F04C0220F331F220F55
:1039B000331F30930C0220930B0220910B023091A5
:1039C0000C02C90137FD079603E0959587950A9586
:1039D000E1F79093FD018093FC0180910D0290919D
:1039E0000E02820F931F97FD0196959587959093F0
:1039F0000E0280930D022091480330914903821BEF
:103A0000930B90931C0180931B0120910202309133
:103A1000030280911B0190911C01280F391F37FF71
:103A200002C02F5F3F4F35952795309303022093B7
:103A3000020251CE2091090230910A028091780051
:103A400090917900280F391F30930A0220930902C0
:103A5000809101018A3019F4220F331F04C0220F14
:103A6000331F220F331F30930A0220930902209143
:103A7000090230910A02C90137FD0796F3E09595D6
:103A80008795FA95E1F79093FB018093FA01809175
:103A90000F0290911002820F931F97FD019695954A
:103AA00087959093100280930F02209146033091E6
:103AB0004703821B930B90931A0180931901209165
:103AC0000002309101028091190190911A01280F92
:103AD000391F37FF02C02F5F3F4F35952795309331
:103AE00001022093000283E06BC11092050281E085
:103AF00080930F018091E9019091EA0101969093E2
:103B0000EA018093E9018091780090917900909387
:103B10001401809313018091130190911401AA273D
:103B2000BB27209115023091160240911702509147
:103B30001802280F391F4A1F5B1F2093150230936C
:103B400016024093170250931802809119028F5F5A
:103B500080931902803108F432C18091150190914F
:103B60001601A0911701B09118017C018D0163E04D
:103B7000EE0CFF1C001F111F6A95D1F7E81AF90A15
:103B80000A0B1B0BE20EF31E041F151F8091ED01A3
:103B9000992787FD9095A92FB92FBC01CD0120EB66
:103BA00030E240E050E00E94BC77DC01CB01E81A33
:103BB000F90A0A0B1B0BD801C7010496A11DB11D00
:103BC000B7FF05C0D801C7010B96A11DB11D23E0A9
:103BD000B595A795979587952A95D1F78093150167
:103BE00090931601A0931701B09318018091CE0510
:103BF0009091CF057C010027F7FC0095102F809154
:103C0000150190911601A0911701B0911801E81AC1
:103C1000F90A0A0B1B0BE092D302F092D402009334
:103C2000D5021093D6022091EE013091EF01409120
:103C3000F0015091F10157FF04C0215F3F4F4F4FFA
:103C40005F4F84E055954795379527958A95D1F72D
:103C50008091EE019091EF01A091F001B091F101FE
:103C6000821B930BA40BB50B8093EE019093EF0195
:103C7000A093F001B093F1018091EE019091EF01DA
:103C8000A091F001B091F1018E0D9F1DA01FB11FF9
:103C90008093EE019093EF01A093F001B093F101B6
:103CA0008091EE019091EF01A091F001B091F101AE
:103CB000B7FF03C00F96A11DB11D14E0B595A795E0
:103CC000979587951A95D1F72091D3023091D40218
:103CD000281B390B84E0213038071CF020E034E049
:103CE00006C08CEF2030380714F420E03CEF8091C0
:103CF000EB019091EC018091EB019091EC0197FF29
:103D000003C0909581959F4FA901F3E0440F551F83
:103D1000FA95E1F78D5B9240C4F08091EB019091B0
:103D2000EC019C01E4E0220F331FEA95E1F7281B28
:103D3000390B240F351F37FF02C0215F3F4F74E05E
:103D4000359527957A95E1F717C08091EB01909111
:103D5000EC019C0165E0220F331F6A95E1F7281BF7
:103D6000390B240F351F37FF02C0215E3F4F45E05E
:103D7000359527954A95E1F73093EC012093EB01B7
:103D80008091150290911602A0911702B09118022D
:103D9000B7FF03C00196A11DB11DB595A7959795D5
:103DA00087958093150290931602A0931702B09303
:103DB000180288E08093190202C01092050282E086
:103DC000809304028091040280937C00809105021C
:103DD000882319F08FEC80937A00FF91EF91BF91C7
:103DE000AF919F918F917F916F915F914F913F9193
:103DF0002F911F910F91FF90EF900F900FBE0F909A
:103E00001F90189590E2E9EDF5E08FE491938150D1
:103E100087FFFCCF089590911C02903540F4E92F64
:103E2000FF27E752FA4F80839F5F90931C0208950B
:103E3000AF92BF92CF92DF92FF920F931F93CF93D7
:103E4000DF9320911A0220FF0AC080911B02882371
:103E500011F0815002C080911F0180931B0221FF4D
:103E60000CC090911B0280911F01981719F41092B9
:103E70001B0203C09F5F90931B02822F992780FF34
:103E800004C081FF02C010921B020E94021F809199
:103E90001B02282F33279BE0C92E9FE1D92EC0910A
:103EA000E403D091E5038A3098F481E180931C0209
:103EB0003F932F9385E094E09F938F93DF92CF926F
:103EC000FE0109952DB73EB72A5F3F4F2DBF11C0A8
:103ED00080E180931C023F932F938AE094E09F93AC
:103EE0008F93DF92CF92FE0109958DB79EB706960C
:103EF0008DBF20911B02822F9927AA27BB27FC0187
:103F0000419710F00C944D28E05BFF4F0BE0C02E62
:103F10000FE1D02EC091E403D091E5030C94827898
:103F200010921C028FE094E09F938F930BE01FE1AF
:103F3000DF92CF92FE01099584E180931C020F90DD
:103F40000F900F900F9085E690E09F938F9388E5F8
:103F500090E09F938F931F921F92809101016AE0DE
:103F60000E94DB77892F99279F938F93809101017E
:103F70000E94DB7799279F938F938FE194E09F9323
:103F80008F93DF92CF92E091E403F091E5030995DE
:103F900088E280931C02EDB7FEB73E96EDBF87EA3C
:103FA00096E09F938F930E94C92B99279F938F939D
:103FB00084E394E09F938F93DF92CF92E091E403A8
:103FC000F091E50309958091FE032DB73EB7285F78
:103FD0003F4F2DBF84FF06C08CE380931C0282E418
:103FE00094E0D2C09091FD03992351F08CE380932B
:103FF0001C02892F99279F938F938FE494E03BC1F4
:10400000909122029923B1F08CE380931C02892FB6
:1040100099279F938F9386E694E09F938F931F93A6
:104020000F93E091E403F091E5030995EDB7FEB736
:10403000369679C49091B303992371F08CE3809301
:104040001C02892F99279F938F938BE794E09F936E
:104050008F931F930F93D9C480913C0190913D01A0
:10406000069710F00C9456288CE380931C028CE881
:1040700094E0A5C7809116081BE0C12E1FE1D12E48
:10408000C091E403D091E50380FF6BC010921C0245
:104090008091D3029091D402A091D502B091D60222
:1040A000BC01CD0125E030E040E050E00E943078D6
:1040B0003F932F9389E994E09F938F93DF92CF9260
:1040C000FE01099584E180931C028DB79EB7069688
:1040D0008DBF8091CF029091D002A091D102B0917A
:1040E000D202BC01CD0125E030E040E050E00E946A
:1040F00030783F932F9386EA94E09F938F93DF92DB
:10410000CF92E091E403F091E503099588E2809372
:104110001C02EDB7FEB73696EDBF8091130190916A
:1041200014019F938F9383EB94E09F938F93DF927F
:10413000CF92E091E403F091E50309958CE380933D
:104140001C022DB73EB72A5F3F4F2DBF87B5992779
:104150009F938F9380EC94E09F938F93DF92CF9205
:104160008EC010921C028DEC94E09F938F93DF928F
:10417000CF92FE01099584E180931C020F900F906D
:104180000F900F908CED94E09F938F93DF92CF92DE
:104190001AC710921C0285EE94E09F938F930BE058
:1041A0001FE1DF92CF92FE01099584E180931C020A
:1041B0000F900F900F900F908091330390913403E4
:1041C000A0913503B0913603B7FF04C081509C4FD6
:1041D000AF4FBF4FCAE0B595A79597958795CA95FC
:1041E000D1F7BF93AF939F938F9382EF94E09F9308
:1041F0008F931F930F93E091E403F091E5030995EA
:1042000088E280931C02EDB7FEB73896EDBF80912F
:104210002B0390912C03A0912D03B0912E03B7FF97
:1042200004C081509C4FAF4FBF4FFAE0B595A795A2
:1042300097958795FA95D1F7BF93AF939F938F93F7
:1042400081E095E09F938F931F930F93E091E40398
:10425000F091E50309958CE380931C022DB73EB7DE
:10426000285F3F4F2DBF8091D3079091D4079F9334
:104270008F9380E195E09F938F931F930F93E0912D
:10428000E403F091E50309958DB79EB706968DBFBF
:104290000DC7E1E0FE2EC1E0D0E00FE517E09F2D55
:1042A000969584E1989FC001112480931C02F80127
:1042B000828193819F938F932196DF93CF93219750
:1042C000808191819F938F93DF93CF938FE195E0CE
:1042D0009F938F938BE09FE19F938F93E091E403F3
:1042E000F091E50309952DB73EB7245F3F4F2DBFF1
:1042F00032E0F30E22960C5F1F4F88E08F1578F6A0
:10430000D5C610921C0280912C06E82FFF27EE0FD5
:10431000FF1FE35AF84F808191819F938F93809183
:104320002B06E82FFF27EE0FFF1FE35AF84F80817F
:1043300091819F938F9381E395E09F938F93DF9279
:10434000CF92FE01099584E180931C02EDB7FEB780
:104350003896EDBF80912E06E82FFF27EE0FFF1F46
:10436000E35AF84F808191819F938F9380912D061E
:10437000E82FFF27EE0FFF1FE35AF84F808191814E
:1043800081589F4F9F938F9381E495E09F938F93E4
:10439000DF92CF92E091E403F091E503099588E282
:1043A00080931C022DB73EB7285F3F4F2DBF8091F1
:1043B0003006E82FFF27EE0FFF1FE35AF84F8081EA
:1043C000918181589F4F9F938F9380912F06E82F63
:1043D000FF27EE0FFF1FE35AF84F8081918181582C
:1043E0009F4F9F938F9381E595E09F938F93DF92EB
:1043F000CF92E091E403F091E50309958CE380937B
:104400001C028DB79EB708968DBF80913206E82FAB
:10441000FF27EE0FFF1FE35AF84F808191818158EB
:104420009F4F9F938F9380913106E82FFF27EE0FC8
:10443000FF1FE35AF84F8081918181589F4F9F93CE
:104440008F9381E695E063C210921C0281E795E0AC
:104450009F938F930BE01FE1DF92CF92FE010995AE
:10446000809101010F900F900F900F908A3009F00A
:104470009DC084E180931C02809148039091490380
:104480009C0197FF02C0295F3F4F287F821B930B3F
:104490009F938F93809148039091490397FD0796CE
:1044A00073E0959587957A95E1F79F938F93209187
:1044B00048033091490337FF02C0295F3F4F63E053
:1044C000359527956A95E1F78091FC019091FD0162
:1044D000821B930B9F938F938FE795E09F938F930E
:1044E0001F930F93E091E403F091E503099588E2AF
:1044F00080931C022DB73EB7265F3F4F2DBF8091A2
:104500004603909147039C0197FF02C0295F3F4FEC
:10451000287F821B930B9F938F93809146039091EA
:10452000470397FD079653E0959587955A95E1F7D0
:104530009F938F93209146033091470337FF02C02A
:10454000295F3F4F43E0359527954A95E1F78091E4
:10455000FA019091FB01821B930B9F938F9380E94B
:1045600095E09F938F931F930F93E091E403F09155
:10457000E50309958CE380931C028DB79EB70A96DC
:104580008DBF80914403909145039F938F938091B9
:104590004403909145032091F8013091F901821B69
:1045A000930B9F938F9381EA95E0ADC08B3019F008
:1045B000843108F4ADC084E180931C0280914803EB
:1045C000909149039C0197FF02C0215F3F4F207FDC
:1045D000821B930B97FD0196959587959F938F93DB
:1045E000809148039091490397FD0F9624E095959B
:1045F00087952A95E1F79F938F93209148033091F7
:10460000490337FF02C0295F3F4FC3E03595279527
:10461000CA95E1F78091FC019091FD01821B930BFB
:104620009F938F938FEA95E09F938F931F930F93A0
:10463000E091E403F091E503099588E280931C0280
:104640002DB73EB7265F3F4F2DBF80914603909117
:1046500047039C0197FF02C0215F3F4F207F821BD1
:10466000930B97FD0196959587959F938F938091D6
:1046700046039091470397FD0F96A4E09595879583
:10468000AA95E1F79F938F932091460330914703BA
:1046900037FF02C0295F3F4FF3E035952795FA9524
:1046A000E1F78091FA019091FB01821B930B9F939C
:1046B0008F9381EC95E09F938F931F930F93E091DD
:1046C000E403F091E50309958CE380931C028DB718
:1046D0009EB70A968DBF809144039091450397FD44
:1046E0000196959587959F938F9380914403909120
:1046F00045032091F8013091F901821B930B9F93A0
:104700008F9383ED95E09F938F931F930F9303C136
:104710008D3009F0CBC484E180931C02809112019A
:1047200099279F938F93809148039091490397FD18
:104730000F9674E0959587957A95E1F79F938F93FF
:10474000209148033091490337FF02C0295F3F4F52
:1047500063E0359527956A95E1F78091FC0190918A
:10476000FD01821B930B9F938F9382EE95E09F93A5
:104770008F931F930F93E091E403F091E503099564
:1047800088E280931C022DB73EB7265F3F4F2DBFB6
:104790008091110199279F938F9380914603909167
:1047A000470397FD0F9654E0959587955A95E1F745
:1047B0009F938F93209146033091470337FF02C0A8
:1047C000295F3F4F43E0359527954A95E1F7809162
:1047D000FA019091FB01821B930B9F938F9386EFBD
:1047E00095E09F938F931F930F93E091E403F091D3
:1047F000E50309958CE380931C028DB79EB70A965A
:104800008DBF8091100199279F938F9380914403CE
:104810009091450397FD0196959587959F938F936A
:1048200080914403909145032091F8013091F90162
:10483000821B930B9F938F938AE096E09F938F93B5
:104840001F930F93E091E403F091E5030995EDB711
:10485000FEB73A9668C010921C028EE196E09F93D4
:104860008F93DF92CF92FE01099584E180931C0221
:104870000F900F900F900F9080913E0390913F0307
:104880009F938F938091F4019091F5019F938F9363
:104890008BE296E09F938F93DF92CF92E091E403B7
:1048A000F091E503099588E280931C022DB73EB78D
:1048B000285F3F4F2DBF80913C0390913D039F9314
:1048C0008F938091F6019091F7019F938F938AE3E4
:1048D00096E09F938F93DF92CF92E091E403F09163
:1048E000E50309958CE380931C028DB79EB708966B
:1048F0008DBF80913803909139039F938F9380915E
:10490000F2019091F3019F938F9389E496E09F9336
:104910008F93DF92CF92E091E403F091E503099544
:10492000EDB7FEB73896EDBFC1C310921C0280915F
:104930001D0190911E016AE070E00E94FB779F9339
:104940008F9380911D0190911E016AE070E00E949A
:10495000FB777F936F9388E596E09F938F93DF9229
:10496000CF92FE01099584E180931C022DB73EB7DA
:10497000285F3F4F2DBF8091B6089091B7086AE03D
:1049800070E00E94E7779F938F938091B608909193
:10499000B7086AE070E00E94E7777F936F938CE638
:1049A00096E09F938F93DF92CF92E091E403F09192
:1049B000E503099588E280931C028DB79EB708969F
:1049C0008DBF8091B8089091B9089F938F9380E82C
:1049D00096E09F938F93DF92CF92E091E403F09162
:1049E000E50309958CE380931C02EDB7FEB736967C
:1049F000EDBF8091BA089091BB089F938F9380E997
:104A000096E09F938F93DF92CF92E091E403F09131
:104A1000E50309952DB73EB72A5F3F4F4FC110926E
:104A20001C0282EA96E09F938F93DF92CF92FE0161
:104A3000099584E180931C020F900F900F900F90C6
:104A400080915D0790915E079F938F938BEA96E02C
:104A50009F938F93DF92CF92E091E403F091E5036F
:104A6000099588E280931C028DB79EB706968DBF8C
:104A70008091D90299279F938F938BEB96E09F9318
:104A80008F93DF92CF92E091E403F091E5030995D3
:104A90008CE380931C02EDB7FEB73696EDBF809194
:104AA0005C07992701979F938F938BEC96E0A9CF92
:104AB00010921C028BED96E09F938F93DF92CF9222
:104AC000FE01099584E180931C020F900F900F90D6
:104AD0000F9080918E0190918F019F938F9383EE21
:104AE00096E09F938F93DF92CF92E091E403F09151
:104AF000E503099588E280931C028DB79EB7069660
:104B00008DBF8091D3079091D4079F938F9381EFAE
:104B100096E09F938F93DF92CF92E091E403F09120
:104B2000E50309958CE380931C02EDB7FEB736963A
:104B3000EDBF8091F1029091F2029F938F938FEFDE
:104B400096E05FCFCAEDCC2EC2E0DC2E20E030E054
:104B5000E901B3E0FB2EC0931C02F60181916F01C5
:104B600099279F938F9389010F5F1F4F1F930F9377
:104B70008DE097E09F938F938BE09FE19F938F93BE
:104B8000E091E403F091E50309952DB73EB7285F66
:104B90003F4F2DBFFA9464969801F7FEDCCF86C292
:104BA000AEEDCA2EA2E0DA2EC0E0D0E08E01F3E036
:104BB000FF2E00931C02F60181916F0199279F93AC
:104BC0008F932596DF93CF938AE197E09F938F93FE
:104BD0008BE09FE19F938F93E091E403F091E503D5
:104BE00009952DB73EB7285F3F4F2DBFFA940C5E55
:104BF0001F4F2497F7FEDDCF59C210921C0287E2A7
:104C000097E09F938F930BE01FE1DF92CF92FE011D
:104C1000099584E180931C020F900F900F900F90E4
:104C200080916D0199279F938F938FE297E09F93D7
:104C30008F93DF92CF92E091E403F091E503099521
:104C400088E280931C028DB79EB706968DBF809137
:104C5000D4019091D50197FD0396959587959595EB
:104C600087959F938F938DE397E09F938F931F93E7
:104C70000F93E091E403F091E50309958CE38093B1
:104C80001C02EDB7FEB73696EDBF80915A06992704
:104C90009F938F938091590699279F938F938BE4CD
:104CA00097E09F938F931F930F93E091E403F0910C
:104CB000E50309952DB73EB7285F3F4F2DBFF6C1DD
:104CC00010921C0289E597E09F938F937BE0A72EBB
:104CD0007FE1B72EDF92CF92FE0109950F900F90E2
:104CE0000F900F90CCEFD6E000E010E062E0F62EDF
:104CF000802F8C5E80931C028B8D99278F7790700C
:104D00009F938F938B8999278F7790709F938F9321
:104D10008B8599278F7790709F938F938B8199279D
:104D20008F7790709F938F9389E697E09F938F93EF
:104D3000BF92AF92E091E403F091E50309958DB73E
:104D40009EB70C968DBFFA940C5E1F4FA096F7FE8F
:104D5000CFCFACC110921C028AE797E09F938F934C
:104D60005BE0A52E5FE1B52EDF92CF92FE010995A3
:104D70000F900F900F900F90CCEFD6E000E010E076
:104D800042E0F42E802F8C5E80931C028F8D992739
:104D900087FD90959F938F938F89992787FD909595
:104DA0009F938F938F85992787FD90959F938F93DE
:104DB0008F81992787FD90959F938F9389E897E03E
:104DC0009F938F93BF92AF92E091E403F091E5033C
:104DD0000995EDB7FEB73C96EDBFFA940C5E1F4FF8
:104DE000A096F7FECFCF62C110921C028AE997E02D
:104DF0009F938F930BE01FE1DF92CF92FE01099505
:104E000084E180931C020F900F900F900F9080917F
:104E10001707881F8827881F97E0899FC0011124E2
:104E20008D969F938F9380910F07881F8827881FE7
:104E300096E0899FC00111248D969F938F93809156
:104E40000707881F8827881F95E0899FC0011124C4
:104E50008D969F938F938091FF06881F8827881FC8
:104E60009927880F991F880F991F8D969F938F936D
:104E700089EA97E09F938F93DF92CF92E091E403CA
:104E8000F091E503099588E280931C022DB73EB7A7
:104E9000245F3F4F2DBF80913707881F8827881FC9
:104EA0009BE0899FC00111248D969F938F938091E1
:104EB0002F07881F8827881F9AE0899FC001112427
:104EC0008D969F938F9380912707881F8827881F2F
:104ED00099E0899FC00111248D969F938F938091B3
:104EE0001F07881F8827881F992723E0880F991F8D
:104EF0002A95E1F78D969F938F938DEB97E09F9383
:104F00008F93DF92CF92E091E403F091E50309954E
:104F10008CE380931C028DB79EB70C968DBF809159
:104F20003F07881F8827881F9CE0899FC0011124A4
:104F30008D969F938F9381ED97E09F938F93DF9250
:104F4000CF92E091E403F091E50309958091470742
:104F5000EDB7FEB73696EDBF87FF12C080E48093B1
:104F60001C0282EE97E09F938F93DF92CF92E091A5
:104F7000E403F091E50309950F900F900F900F90C7
:104F800080914F0787FF12C084E480931C0285EE56
:104F900097E09F938F931F930F93E091E403F09119
:104FA000E50309950F900F900F900F908091570790
:104FB00087FF7CC088E480931C0288EE97E09F9373
:104FC0008F931F930F93E091E403F091E50309950C
:104FD0000F900F900F900F9069C010921C028BEEF3
:104FE00097E09F938F93DF92CF92FE01099584E122
:104FF00080931C020F900F900F900F908091AA0148
:105000009091AB019F938F9389EF97E09F938F933C
:10501000DF92CF92E091E403F091E503099588E2F5
:1050200080931C022DB73EB72A5F3F4F2DBF809162
:10503000AC019091AD019F938F9386E098E09F9390
:105040008F93DF92CF92E091E403F091E50309950D
:1050500089E480931C028DB79EB706968DBF83E1CD
:1050600098E09F938F93DF92CF92E091E403F091C9
:10507000E503099580911A020F900F900F900F9001
:1050800083FF14C01092AD011092AC0160E070E09B
:105090008EE090E00E946A2A09C080911F012817C3
:1050A00019F4215020931F0110921B0210921A0232
:1050B000DF91CF911F910F91FF90DF90CF90BF9024
:1050C000AF900895F999FECF92BD81BDF89A80B551
:1050D00099270895F999FECF1FBA92BD81BD60BD91
:1050E0000FB6F894FA9AF99A0FBE08954AEA20E0AA
:1050F00030E02617370740F4FC018191480F2F5FFD
:105100003F4F26173707C8F3842F99270895EAEAF7
:1051100040E050E04617570778F49C01F999FECF1C
:1051200032BD21BDF89A80B5E80F4F5F5F4F2F5F0A
:105130003F4F4617570790F38E2F9927089581E028
:1051400080932D0682E080932C0683E080932B06CB
:1051500084E080932E0685E080932F0686E080937E
:10516000300687E08093310688E08093320689E03C
:10517000809333068AE0809334068BE08093350673
:105180008CE08093360608958AE580932A06809104
:105190000101843150F08AE080934A0610926E0635
:1051A0008BE1809346068EE40AC083E080934A0632
:1051B00080E280936E068EE18093460685E58093BB
:1051C0006B0680936C0680E280936D0610929506C4
:1051D0008AE68093370682E28093970610929806BB
:1051E00064E06093510610928D0610928A0648E0A2
:1051F0004093440656EE5093450680E4809347065C
:105200009EE1909338068FEF80933A062FE020932B
:105210003B069093390610923D0640933E0684E18A
:1052200080933F061092400620933C06109253064E
:10523000109254061092550610925606109270065F
:1052400010927106109272061092730690E8909375
:10525000570632E33093580682E0809396062093F7
:10526000590650935A0660935F068DE78093620655
:10527000809363068093640690935B0625E52093F4
:105280005C0686E480935D068CED80935E068CE37D
:1052900080936006109261068FE58093740683EF19
:1052A000809376068AEA809378068093790688E26E
:1052B0008093750680937706309365069AE5909300
:1052C0006606309367068EEF80937A0684E68093B5
:1052D0007B0690937C0690937D0690937E068BE4EC
:1052E00080937F0620938006809381061092820629
:1052F00086E08093830640938406909385068AE235
:105300008093860685EF809387068CE880938806D5
:1053100085E08093890610928B0610928C0681E2BC
:1053200080934E0681E480934F069093500610922E
:105330008E0610928F061092900686E98093910651
:105340009093680687E38093690610929206109204
:105350009306109294060895CF93DF930E94C42879
:105360008AE08093410680E18093420626E0209304
:1053700043069AE59093480688E780934906909300
:105380004B0680934C0620934D0680E28093520694
:105390008CE380936A068BE480936F06A9E9B6E0FC
:1053A0008CE0E0E2F1E0ED01019009928A95E1F7ED
:1053B0006BE770E0CD018F5690400E947628809375
:1053C000A506DF91CF910895CF93DF930E94C42863
:1053D00088E08093410630E13093420626E0209336
:1053E000430694E69093480688E780934906909395
:1053F0004B0680934C0620934D063093520686E46C
:1054000080936A0680936F06A9E9B6E08CE0E6E235
:10541000F1E0ED01019009928A95E1F76BE770E008
:10542000CD018F5690400E9476288093A506DF918B
:10543000CF910895CF93DF930E94C42826E0209354
:1054400041068AE08093420684E08093430694E616
:105450009093480688E78093490690934B06809383
:105460004C0620934D0680E18093520686E480939B
:105470006A0680936F06A9E9B6E08CE0EEE2F1E0FF
:10548000ED01019009928A95E1F76BE770E0CD019B
:105490008F5690400E9476288093A506DF91CF9189
:1054A0000895F999FECF92BD81BDF89A80B59927EC
:1054B0000895F999FECF1FBA92BD81BD60BD0FB6A8
:1054C000F894FA9AF99A0FBE089562E678E20E947B
:1054D0004A7608954AE658E20E9484760895EF924B
:1054E000FF920F931F93CF93C82F8150853008F000
:1054F000C3E08CE7C89F8001112488EEE82E8FEF6F
:10550000F82EE00EF11E6BE770E0C7010E948728BD
:10551000682F98012D593F4F8FB39927AC014270E6
:10552000507081FDF9CF32BD21BDF89A80B5861744
:1055300011F0CA0121C08FB399279C0122703070ED
:1055400081FDF9CFF2BCE1BCF89A80B58A3511F043
:10555000C90112C08CE7C89FC0011124489722E6F8
:1055600038E24CE750E0BC018AE296E00E942576E2
:105570000E94196881E090E0CF911F910F91FF90F8
:10558000EF900895282F863010F025E003C088237F
:1055900009F421E0F999FECF1FBA82E090E092BDB4
:1055A00081BD20BD0FB6F894FA9AF99A0FBE0895FE
:1055B000CF93C82F80912A068A3509F04FC0C63094
:1055C00010F0C5E003C0CC2309F448C00E94267542
:1055D0008091980682FF07C080914F06843618F0AC
:1055E00080E580934F066BE770E08AE296E00E94C8
:1055F00076288093A5068CE7C89FC00111242AE66F
:1056000038E24CE750E06AE276E048970E94627622
:105610002AE638E24CE050E06BE276E080E590E08C
:105620000E9462766CE070E08BE296E00E94762841
:10563000282FF999FECF1FBA8CE590E092BD81BD6D
:1056400020BD0FB6F894FA9AF99A0FBE8C2F0E94DB
:10565000C22A0E94196881E090E002C080E090E0D8
:10566000CF9108956DE470E088EE93E00E94872862
:10567000482F8FB399279C012270307081FDF9CF9C
:1056800085E394E092BD81BDF89A80B5841779F4E2
:105690008FB399279C012270307081FDF9CF88EE7D
:1056A00093E092BD81BDF89A80B5813011F0C901B7
:1056B000089522E638E24EE450E068EE73E086EAB0
:1056C00096E00E94257681E090E008958091A606FC
:1056D0008130A9F46DE470E086EA96E00E947628B5
:1056E0008093F3062AE638E24EE450E066EA76E07C
:1056F00088EE93E00E94627681E090E0089580E079
:1057000090E00895CF93DF9381E08093A606E6EAC8
:10571000F6E08FE0158616861786108A815034963B
:1057200087FFF8CF80E48093B3068093B40610928D
:10573000B5068093B6068093B70690EC9093B806B2
:105740001092B9068093BA068093BB061092BC06ED
:105750009093BD069093BE068093BF061092C0063C
:105760008093C1069093C206A7EAB6E087E0E4E31F
:10577000F1E0ED01019009928A95E1F76DE470E0A6
:10578000CD0101970E9476288093F306DF91CF9197
:105790000895F999FECF82E090E092BD81BDF89A1C
:1057A00080B5282F863078F023E0322FF999FECF8C
:1057B0001FBA82E090E092BD81BD30BD0FB6F89473
:1057C000FA9AF99A0FBE822F992708951F93CF93C3
:1057D000C82F162F863010F0C5E003C0882309F4C7
:1057E000C1E08C2F99278230910541F083309105DB
:1057F00044F4019731F40E94AC2905C00E94E429C9
:1058000002C00E941A2A1123E1F06CE070E080E5EA
:1058100090E00E948728282FF999FECF8CE590E030
:1058200092BD81BDF89A80B5821759F422E638E21C
:105830004CE050E060E570E08BE296E00E94257657
:1058400002C00E949F288C2F0E94D82ACF911F91BE
:105850000895DF92EF92FF920F931F93CF93FF244F
:10586000DF2CEF2C81E090E00E94512A8A3511F064
:1058700031E0E32E6CE070E080E590E00E94872844
:10588000C82FF999FECF8CE590E092BD81BDF89AC2
:1058900080B58C1711F421E0D22EC1E001E010E0B8
:1058A000EE2029F48C2F0E946F2A8823C9F591E0FD
:1058B000F92E1F930F938BE198E09F938F9387E8C6
:1058C00091E19F938F93E091E403F091E5030995B3
:1058D0002DB73EB72A5F3F4F2DBF0230110549F06B
:1058E000033011054CF40130110531F40E94AC294C
:1058F00005C00E94E42902C00E941A2ADD2059F046
:1059000022E638E24CE050E060E570E08BE296E0A1
:105910000E94257602C00E949F288C2F0E94D82AC0
:10592000CF5F0F5F1F4FC63008F4BACFFF2019F0CA
:1059300083E00E94C22A0E94C92BC82F0E946F2AAE
:105940008C2F99279F938F9381E498E09F938F9357
:1059500007E811E11F930F93E091E403F091E50351
:10596000099581E090E00E94512A2DB73EB72A5F49
:105970003F4F2DBF8F3F21F00E94322B882399F497
:105980008AE598E09F938F931F930F93E091E40330
:10599000F091E50309950E94822B0E94662B0F90DF
:1059A0000F900F900F90EE2029F06AE581E090E0D3
:1059B0000E94592A1092290690E0E3EBF6E0CFE02E
:1059C0008081349618160CF49F5FC150C7FFF8CF42
:1059D00090932906892F99279F938F9387EA96E0C2
:1059E0009F938F938BE798E09F938F931F930F93D1
:1059F000E091E403F091E50309950E9486058DB7D7
:105A00009EB708968DBFCF911F910F91FF90EF9099
:105A1000DF900895982F2FB7F8943998389A88B165
:105A2000836088B98091B9008C7F8093B9008AE245
:105A30008093B8001092270210922502109224023F
:105A4000992379F0ECEFF6E08BE01082118212825C
:105A5000138214821582168217828150389687FF2E
:105A6000F4CF78942FBF08951092270284E9809391
:105A7000BC0080E88093BC001092BD001092BA0078
:105A80001092BB001092B9001092B800109223023D
:105A900080E00E940A2D1092BB0085E88093BC0034
:105AA0008091210282608093210208951F920F92BB
:105AB0000FB60F9211242F933F934F935F938F93C1
:105AC0009F93EF93FF9380912702282F332744273A
:105AD00055278F5F80932702F9012731310508F0A0
:105AE000C2C2EF59FF4F0C94827881E08093230269
:105AF00009C0809125028C3090F4809125028F5F3F
:105B00008093250280912502E82FFF27EE0FFF1FCB
:105B1000EE0FFF1FEA55F94F8585181654F780914F
:105B200025028C3070F01092200210921F02109209
:105B3000250285E08093270280912402880F8D5AE8
:105B400004C080912502880F8E5A8093BB0085E89F
:105B50007FC280912502E82FFF2783E0EE0FFF1F11
:105B60008A95E1F7E450F94F81818093BB0085E885
:105B70008093BC0080912502E82FFF27EE0FFF1FC6
:105B8000EE0FFF1FEE0FFF1FE450F94F808180FFE3
:105B900091C080912502E82FFF27EE0FFF1FEE0F27
:105BA000FF1FEE0FFF1FE450F94F8281882329F079
:105BB00080912906873008F46CC280911F02909171
:105BC0002002892B09F065C280911D0290911E026E
:105BD000892B09F05EC26EC08091250221E030E081
:105BE00002C0220F331F8A95E2F780911D02909127
:105BF0001E0228233923232B79F080912502E82FD8
:105C0000FF27EE0FFF1FEE0FFF1FEE0FFF1FE450E9
:105C1000F94F80E184830DC080912502E82FFF2792
:105C2000EE0FFF1FEE0FFF1FEE0FFF1FE450F94FA7
:105C3000148280912502E82FFF2753E0EE0FFF1F0B
:105C40005A95E1F7E450F94F8481282F332743E038
:105C5000220F331F4A95E1F780912502E82FFF2795
:105C600093E0EE0FFF1F9A95E1F7E450F94F828120
:105C70008770822B8093BB0085E88093BC002091C5
:105C8000250281E090E002C0880F991F2A95E2F773
:105C900020911F023091200282239323892B51F0FF
:105CA00084EF96E090932B0280932A0288E0809301
:105CB0002C02EFC184E089C1E0912A02F0912B020D
:105CC00081918093BB0085E88093BC00F0932B0208
:105CD000E0932A0280912C02815080932C02882329
:105CE00009F4D7C183E071C18091B900803351F5C7
:105CF00080912802882329F4809125028F5F809368
:105D0000280280912502E82FFF2783E0EE0FFF1F76
:105D10008A95E1F7E450F94F838199278F77907046
:105D20008F3791057CF480912502E82FFF27EE0F35
:105D3000FF1FEE0FFF1FEE0FFF1FE450F94F83818F
:105D40008F5F83831092270284E98093BC008AE0EE
:105D500090E090933D0180933C01809125028F5FFC
:105D600080932502109227026DC18091B900803482
:105D7000C9F180912402E82FFF27EE0FFF1FEE0FDD
:105D8000FF1FEE0FFF1FE450F94F83818F7783834E
:105D9000809124028F5F80932402809124028C30B2
:105DA000A0F01092240210921E0210921D02809107
:105DB00029028F5F809329028C3038F010922902DB
:105DC000809121028D7F8093210280912102816048
:105DD000809321021092270284E98093BC001092E4
:105DE000230273C080912402E82FFF27EE0FFF1FCC
:105DF000EE0FFF1FEE0FFF1FE450F94F8381806805
:105E0000838380912402E82FFF27EE0FFF1FEE0F00
:105E1000FF1FEE0FFF1FE450F94F808180FF2FC05E
:105E200080912402E82FFF2753E0EE0FFF1F5A95C1
:105E3000E1F7E450F94F84819927009751F040979A
:105E4000D9F584EF96E090932B0280932A0288E0A4
:105E500031C080912402992743E0880F991F4A9509
:105E6000E1F78F5F984F90932B0280932A029091D5
:105E70002402809129029817E1F483E01BC08091ED
:105E80002402992733E0880F991F3A95E1F78F5F35
:105E9000984F90932B0280932A028091210281FDDA
:105EA00006C09091240280912902981711F482E093
:105EB00001C081E080932C0280912C02813011F48A
:105EC00085E801C085EC8093BC0080912802809316
:105ED000220210922802DDC0E0912A02F0912B02EA
:105EE0008091BB00808380912A0290912B020196C1
:105EF00090932B0280932A0280912C0281508093F0
:105F00002C02823010F085EC5DC0813011F485E800
:105F100059C08091210281FF2DC08091A10280FD96
:105F20001DC080912402E82FFF2723E0EE0FFF1F02
:105F30002A95E1F7E450F94F86818A3F79F4809100
:105F40002402E82FFF2793E0EE0FFF1F9A95E1F759
:105F5000E450F94F8081816080830CC080912402DD
:105F6000E82FFF2783E0EE0FFF1F8A95E1F7E4504B
:105F7000F94F1082809124028F5F809324028091D8
:105F800024028C30A0F01092240210921E02109273
:105F90001D02809129028F5F809329028C3038F096
:105FA00010922902809121028D7F8093210210920C
:105FB000270284E98093BC00809121028160809354
:105FC000210265C08093BC0086E08093270261C0F7
:105FD00088E9BBCD80912602880F805FB6CD809185
:105FE000260299278130910561F0823091051CF4D9
:105FF000892B21F04EC0029739F04BC080911201DD
:10600000A4CD80911101A1CD809110019ECD80E899
:106010009CCD1092270284E98093BC001092230249
:106020008AE090E090933D0180933C0180912602AC
:10603000823088F4809126028F5F8093260282E16D
:1060400080932702809121028E7F8093210285EA2E
:106050008093BC001EC010922602809121028160B4
:106060008093210216C01092270284E98093BC001D
:10607000809121028160809321028AE090E09093D8
:106080003D0180933C01109225021092240210924F
:106090002302FF91EF919F918F915F914F913F91DB
:1060A0002F910F900FBE0F901F9018951F93CF93B5
:1060B000DF93182F8091D802882321F48091B901B1
:1060C000882319F081E090E097C01D3008F092C05D
:1060D0001123B1F0E12FFF2723E0EE0FFF1F2A95D8
:1060E000E1F7E450F94F35978081359688230CF01D
:1060F00081C03897808180FD03C083E090E07CC040
:106100008091F406823019F084E090E075C067E079
:1061100070E084EF96E00E9476289091FB06891744
:1061200019F085E090E068C080ED97E00E94961538
:10613000EC018091210280FD05C0CE010E949F15D7
:106140008823B9F3112319F48FEF90E00BC0212FAE
:1061500033272150304081E090E002C0880F991F22
:106160002A95E2F79093200280931F02A1E0B0E00D
:10617000ECEFF6E040E050E06BE0CD01042E02C011
:10618000880F991F0A94E2F720911F023091200294
:1061900082239323892B11F01182128261504F5F69
:1061A0005F4F389667FFE9CF1092250210922702C1
:1061B000809121028E7F8093210285EA8093BC002A
:1061C0008091210280FD05C0CE010E949F15882389
:1061D000B9F380911F0290912002892B29F0CE0102
:1061E0000E949F15882311F380911F029091200235
:1061F000009711F082E090E0DF91CF911F91089518
:106200000F931F93CF93DF93982F8091D802882309
:1062100021F48091B901882319F081E090E092C0C7
:106220009D30A0F4992319F486E090E08BC0C92F2B
:10623000DD27FE0133E0EE0FFF1F3A95E1F7E45052
:10624000F94F35978081359687FD03C082E090E055
:1062500079C03897808180FD03C083E090E072C0F0
:1062600080ED97E00E9496158C018091210280FDBF
:1062700005C0C8010E949F158823B9F3219721E02A
:1062800030E0C90102C0880F991FCA95E2F79093C8
:106290001E0280931D02D901ECEFF6E040E050E0D1
:1062A0006BE0CD01042E02C0880F991F0A94E2F71B
:1062B00020911D0230911E0282239323892B11F01D
:1062C0001182128261504F5F5F4F389667FFE9CFAE
:1062D000109224021092F4061092FB0610922702EC
:1062E000809121028E7F8093210285EA8093BC00F9
:1062F0008091210280FD05C0C8010E949F1588235E
:10630000B9F380911D0290911E02892B29F0C801DA
:106310000E949F15882311F38091F406823019F0B2
:1063200084E090E00FC067E070E084EF96E00E94A8
:1063300076289091FB06891719F085E090E002C05D
:1063400080E090E0DF91CF911F910F910895CF935E
:10635000DF9380E022E83FEFC1E9D7E0EDE5F7E029
:10636000DF01853020F411961C921E9202C0318309
:1063700020831982188222968F5F129632968A3174
:1063800080F3109245031092440310924703109239
:1063900046031092490310924803DF91CF9108956C
:1063A0001F920F920FB60F9211240F931F932F93EA
:1063B0003F934F935F936F937F938F939F93AF938D
:1063C000BF93CF93DF93EF93FF938091970682FD66
:1063D000E1C0409186005091870080912E029091FB
:1063E0002F02481B590B8091860090918700909353
:1063F0002F0280932E02CA018D549440A091300246
:10640000B0913102835F9A4178F480913002809399
:106410005C07149714F01092400181E090E0909393
:106420003102809330022BC2AD30B1050CF027C28F
:10643000CA018B5F9040845B914008F086C08091D8
:106440003E0190913F01481B590BE0919206EE23CB
:1064500051F0FF27EE0FFF1FE35AF84F8081918123
:1064600084369105ECF4FD01EA0FFB1FE35AF84F67
:1064700080819181FA01E81BF90BCF01F7FF03C07E
:10648000909581959F4F06975CF48091D902883C46
:1064900020F48091D902865F01C088EC8093D902F4
:1064A000FD01EA0FFB1FE35AF84F808191819C01A7
:1064B000220F331F280F391F240F351F37FF02C04B
:1064C0002D5F3F4FE901D595C795D595C795CA0171
:1064D00001968C179D0714F4219706C04150504037
:1064E000C417D5070CF421968091D902833CE0F0C3
:1064F0008D010A0F1B1FF801E35AF84F808191812B
:106500009E01281B390BC90163E070E00E94FB77F4
:10651000CB01880F991F860F971F0F56184FD80170
:1065200011969C938E9307C0AA0FBB1FAF56B84F0E
:1065300011961C921E92E0913002F0913102EE0F02
:10654000FF1FE35AF84FD183C0832091300230916E
:1065500031022F5F3F4F3093310220933002809100
:106560000101843108F08BC12530310511F45D9AA9
:1065700001C05D9880913002909131028630910582
:1065800011F45C9A01C05C98079711F45B9A77C18B
:106590005B9875C1409186005091870080913202CE
:1065A00090913302481B590B80918600909187008F
:1065B0009093330280933202CA018D5494406091CB
:1065C0009C02835F9A4108F07AC060932D0280910B
:1065D0002D02843008F453C090915C0780912D0205
:1065E000981709F04CC050919D025B3008F43FC0F1
:1065F0001092400110929C0240E05F31C0F0E42F05
:10660000FF27EE0FFF1F9F0128593D4FDF01A35ABF
:10661000B84F8D919C91D9018D939C93DF01AF561A
:10662000B84F8D919C91EE57FD4F91838083E42F5D
:10663000FF27EE0FFF1F9F01235A384FDF01AC5C8D
:10664000BD4F8D919C91D90111969C938E93DF0142
:10665000A25BBD4F8D919C91EF56F84F9183808343
:10666000842F8F5F482F8D3040F280939C02809161
:106670009D028F3FB9F08F5F80939D0213C0809180
:106680009D02853620F08AE080939D0202C0109220
:106690009D02809101018A3011F0843110F0289A16
:1066A00001C0289881E080939C028091D8028823C1
:1066B00009F0E5C080912D0280935C07E0C06D3049
:1066C00008F0B5C0CA018B5F9040845B914008F030
:1066D00090C080913E0190913F01481B590BE62FDD
:1066E000FF27EE0FFF1FEC5CFD4F80819181FA01C7
:1066F000E81BF90BCF0105960B9720F5E091920668
:10670000EE2351F0FF27EE0FFF1FE35AF84F808171
:10671000918184369105B4F480919D028A3120F0F4
:106720008091D902865F05C08B3028F08091D90214
:106730008E5F8093D9028091D902893C18F088EC51
:106740008093D902E62FFF27EE0FFF1FEC5CFD4F71
:10675000808191819C01220F331F280F391F240F44
:10676000351F37FF02C02D5F3F4FE901D595C79513
:10677000D595C795CA0101968C179D0714F42197EA
:1067800006C041505040C417D5070CF421968091A3
:10679000D9028E3BD8F0E62FFF27EE0FFF1FDF0157
:1067A000AC5CBD4F8D919C919E01281B390BC9019A
:1067B00063E070E00E94FB77CB01880F991F860F82
:1067C000971FE25BFD4F9183808308C0E62FFF2770
:1067D000EE0FFF1FE25BFD4F1182108280919C0241
:1067E000E82FFF27EE0FFF1FEC5CFD4FD183C08326
:1067F00009C0809101018A3011F0843110F0289A8B
:1068000001C0289880910101843188F480919C0214
:10681000853011F45D9A05C05D98863011F45C9A5C
:1068200005C05C98873011F45B9A01C05B98809139
:106830009C02843120F48F5F80939C0220C08431BD
:10684000F1F4809101018A3011F0843110F0289A1E
:1068500001C028988EE180939C022CE0C1E9D7E02A
:10686000A8E6B2E0EDE5F7E08D919D9191838083FC
:106870003296198218822296215027FFF5CFFF9178
:10688000EF91DF91CF91BF91AF919F918F917F91C8
:106890006F915F914F913F912F911F910F910F90A9
:1068A0000FBE0F901F901895EF92FF920F931F93BA
:1068B000809146069927880F991F880F991F7C01A0
:1068C0000027F7FC0095102F80913303909134033B
:1068D000A0913503B0913603BC01CD01A801970109
:1068E0000E94307830938A052093890580912B038C
:1068F00090912C03A0912D03B0912E03BC01CD01EA
:10690000A80197010E94307830938C0520938B0565
:1069100080911A0890911B0897FD0396959587958D
:106920009595879590938E0580938D0580912A0883
:1069300090912B0897FD039695958795959587954A
:106940009093900580938F05809144039091450327
:106950002091F8013091F901821B930B90939205DD
:10696000809391058091D3029091D402A091D50299
:10697000B091D602BC01CD0125E030E040E050E00E
:106980000E94307830939405209393058091F20112
:106990009091F301909396058093950580918E01D7
:1069A00090918F0190939A058093990580911D0194
:1069B00090911E0190939C0580939B058091D90234
:1069C000992790939E0580939D058091D307909180
:1069D000D4079093A00580939F058091FD06992789
:1069E0009093A2058093A105809105079927909324
:1069F000A4058093A30580910D0799279093A60580
:106A00008093A5058091150799279093A8058093F9
:106A1000A7058091D4019091D5019093B205809300
:106A2000B1058091B6089091B7089093B605809310
:106A3000B5058091BA089091BB089093B8058093F2
:106A4000B7058091CF029091D002A091D102B09170
:106A5000D202BC01CD0125E030E040E050E00E94D0
:106A600030783093BA052093B9058091F102909166
:106A7000F2029093C0058093BF058091BC089927CE
:106A80009093C4058093C3058091A4039091A503BE
:106A90009093C6058093C5058091A2039091A303AE
:106AA0009093C8058093C7058091FD03882321F446
:106AB0008091FE03882321F080918805816003C0C6
:106AC000809188058E7F809388051F910F91FF909C
:106AD000EF9008951F93CF93DF93182FEB018091D0
:106AE000D802882309F5809101018C3010F429988F
:106AF00001C0299A11501F3F81F0D093DB01C09350
:106B0000DA018091DA019091DB01892BD1F7CE0176
:106B10008C0F9D1F0E94AB15EDCF809101018C3031
:106B200010F4299A01C02998DF91CF911F910895FF
:106B3000CF93DF93809101018D3011F40E940E1AE2
:106B400010927A008091FC019091FD019093DF07F3
:106B50008093DE078091FA019091FB019093CF071B
:106B60008093CE078091F8019091F90190932008CD
:106B700080931F082091F4013091F501C901880F1D
:106B8000991F880F991F820F931F820F931F909355
:106B90001B0880931A082091F6013091F701C90172
:106BA000880F991F880F991F820F931F820F931FC1
:106BB00090932B0880932A088FEC80937A00AAED9B
:106BC000B2E0CFE2D6E097E08991E82FFF27EE0F01
:106BD000FF1FE35AF84F0190F081E02DE158FF4F7D
:106BE0001E161F061CF0E0E0F0E005C0EF3FF105C7
:106BF00014F0EFEFF0E08C91282F3327E217F30722
:106C000014F4815004C02E173F0714F48F5F8C9347
:106C10009150119697FFD8CF80916B069927AA279C
:106C2000BB27BC01CD0124EC39E040E050E00E94DC
:106C3000BC77DC01CB018093860190938701A09300
:106C40008801B093890180916C069927AA27BB27F8
:106C5000BC01CD010E94BC77DC01CB018093820195
:106C600090938301A0938401B0938501DF91CF912C
:106C70000895A0E0B0E0EFE3F6E30C945178882E9D
:106C8000C0E0D0E07E016E011092FD03469AD093E1
:106C90003F03C0933E03D0933D03C0933C03D09386
:106CA0003903C0933803D0934903C0934803D0936A
:106CB0004703C0934603D0934503C0934403109207
:106CC0006A01109269011092ED010E94983584E6E4
:106CD00090E00E94B8150E9498358091370680FF99
:106CE00010C08091130190911401875B934038F498
:106CF00080911301909114018E5E924010F40E94D5
:106D0000B3190FE18AE090E00E94B8158091F80174
:106D10009091F901C80FD91F8091FC019091FD015C
:106D2000E80EF91E8091FA019091FB01C80ED91E60
:106D3000015007FFE7CF9701205F3F4F369527951A
:106D4000369527953093490320934803C601409612
:106D500096958795969587959093470380934603DC
:106D60006096F5E0D695C795FA95E1F7D09345037F
:106D7000C0934403909343038093420330934103B1
:106D800020934003882009F441C080911A08909113
:106D90001B0897FF03C0909581959F4F6CE070E0B2
:106DA0000E94FB779B0170933F0360933E038091A9
:106DB0002A0890912B0897FF03C0909581959F4FCB
:106DC0006CE070E00E94FB7770933D0360933C039E
:106DD0008091CC059091CD05909339038093380331
:106DE000B90184E090E00E946A2A60913C037091AE
:106DF0003D0386E090E00E946A2A6091380370911A
:106E0000390388E090E00E946A2A65C084E090E03F
:106E10000E94652A90933F0380933E0386E090E0B2
:106E20000E94652A90933D0380933C0388E090E0A4
:106E30000E94652A9C0190933903809338038091C6
:106E40003E0390913F038150984050F480913C0361
:106E500090913D038150984018F421503440D8F16E
:106E60008CE998E09F938F9387E891E19F938F93AC
:106E7000E091E403F091E503099580911A0890915F
:106E80001B0897FF03C0909581959F4F6CE070E0C1
:106E90000E94FB7770933F0360933E0380912A0822
:106EA00090912B0897FF03C0909581959F4F6CE0C0
:106EB00070E00E94FB7770933D0360933C038091E8
:106EC000CC059091CD0590933903809338030F90B2
:106ED0000F900F900F901092DF071092DE07109224
:106EE000CF071092CE071092200810921F0884E658
:106EF00090E00E94B8158091F4019091F5019C01F9
:106F0000220F331F220F331F280F391F280F391F5D
:106F100030931B0820931A088091F6019091F70195
:106F20008C01000F111F000F111F080F191F080FF0
:106F3000191F10932B0800932A0880914606C82E2B
:106F4000DD24EE24FF24442737FD4095542FC7014C
:106F5000B6010E94BC774B015C01609333037093D0
:106F6000340380933503909336039801442737FD0B
:106F70004095542FC701B6010E94BC77DC01CB01BC
:106F800080932B0390932C03A0932D03B0932E0397
:106F90008092130390921403A0921503B0921603EB
:106FA00080930B0390930C03A0930D03B0930E03F7
:106FB000109203031092040310920503109206032B
:106FC0008091150190911601A0911701B0911801BF
:106FD0009093CF058093CE051092EC011092EB01B7
:106FE0001092F3021092F4021092F5021092F6023F
:106FF00000918E0110918F011093F2020093F10223
:1070000084E690E090938B0180938A0182E390E084
:107010009093DB018093DA0180916B069927AA2770
:10702000BB27BC01CD0124EC39E040E050E00E94D8
:10703000BC77DC01CB018856954CAF4FBF4F809396
:10704000860190938701A0938801B0938901809174
:107050006C069927AA27BB27BC01CD010E94BC77EB
:10706000DC01CB018856954CAF4FBF4F8093820116
:1070700090938301A0938401B093850110924701FE
:1070800010924601C801AA2797FDA095BA2F20911A
:107090004201309143014091440150914501BC01AE
:1070A000CD010E94BC77DC01CB0180932608909330
:1070B0002708A0932808B09329081092EE02109296
:1070C000ED020E9419688091A10284608093A10260
:1070D0008FEF8093A6081092A70880E28093A808FB
:1070E000CAEDD2E0AFE2B6E007E08D91E82FFF27CE
:1070F000EE0FFF1FE35AF84F8081918181588993E9
:10710000015007FFF2CF84E68093D9028091D80125
:10711000882311F0469A579A809148039091490329
:1071200080569940815C9B4228F08091FD038160EC
:107130008093FD03809146039091470380569940C8
:10714000815C9B4228F08091FD0382608093FD0367
:1071500080914403909145038C529140895795400A
:1071600028F08091FD0384608093FD0380913E03AD
:1071700090913F038C529140835C914028F0809124
:10718000FD0388608093FD0380913C0390913D0353
:107190008C529140835C914028F08091FD03806186
:1071A0008093FD0380913803909139038050924081
:1071B0008355914028F08091FD0380628093FD0308
:1071C00086E480937D01ECE0CDB7DEB70C946D785A
:1071D000A3E1B0E0EEEEF8E30C944B788091440329
:1071E000909145032091F8013091F901821B930B96
:1071F0009093200880931F088091020290910302CF
:1072000097FD07969C0113E0359527951A95E1F7B0
:107210003093DF072093DE078091000290910102F6
:1072200097FD0796B3E095958795BA95E1F790930A
:10723000CF078093CE073093EA072093E907909316
:10724000E2078093E10780911A0890911B08AC0136
:10725000440F551F480F591F2091F4013091F5013B
:10726000C901880F991F880F991F820F931F820FE2
:10727000931F480F591F57FF02C04D5F5F4F559531
:1072800047955595479550931B0840931A08809150
:107290002A0890912B08AC01440F551F480F591F25
:1072A0002091F6013091F701C901880F991F880FCD
:1072B000991F820F931F820F931F480F591F57FF6B
:1072C00002C04D5F5F4F5595479555954795509333
:1072D0002B0840932A082091F4013091F501C9014F
:1072E000880F991F880F991F820F931F820F931F7A
:1072F0009C01442737FD4095542F809123039091A2
:107300002403A0912503B0912603820F931FA41F8D
:10731000B51F8093230390932403A0932503B09378
:1073200026032091F6013091F701C901880F991FBA
:10733000880F991F820F931F820F931F9C01442770
:1073400037FD4095542F80911F0390912003A09109
:107350002103B0912203820F931FA41FB51F8093B6
:107360001F0390932003A0932103B09322038091E5
:10737000F3079091F4072091F4013091F501820F09
:10738000931F9093F4078093F307809122089091C4
:1073900023082091F6013091F701820F931F9093FB
:1073A00023088093220880913A0390913B03019631
:1073B00090933B0380933A038091CC059091CD0547
:1073C0002091380330913903821B930B9C01442791
:1073D00037FD4095542F80911B0390911C03A09181
:1073E0001D03B0911E03820F931FA41FB51F80932E
:1073F0001B0390931C03A0931D03B0931E038FECFB
:1074000080937A0010920F0120910B0330910C03AE
:1074100040910D0350910E0329873A874B875C8773
:1074200029543B46414050402CF028E43BE641E0E3
:1074300050E00DC089859A85AB85BC85885B9449F1
:10744000AE4FBF4F4CF428EB34E94EEF5FEF2D8386
:107450003E834F83588708C089859A85AB85BC8554
:107460008D839E83AF83B8872091130330911403DB
:1074700040911503509116032D873E874F87588BF7
:1074800029543B46414050402CF028E43BE641E083
:1074900050E00DC08D859E85AF85B889885B944985
:1074A000AE4FBF4F4CF428EB34E94EEF5FEF29832A
:1074B0003A834B835C8308C08D859E85AF85B889F0
:1074C00089839A83AB83BC83A0911F08B091200865
:1074D000BB8BAA8BFD01CF01AA2797FDA095BA2FE0
:1074E000A0900303B0900403C0900503D09006035E
:1074F000A80EB91ECA1EDB1EA0920303B09204039D
:10750000C0920503D0920603E0902608F090270869
:107510000091280810912908E80EF91E0A1F1B1F68
:10752000E0922608F0922708009328081093290873
:10753000F091BC02F98BFF2309F098C18091BB0246
:10754000882309F093C18091160886FF8FC180912E
:10755000CE079091CF07AA2797FDA095BA2FBC011F
:10756000CD0129813A814B815C810E94BC779B01CE
:10757000AC0197FF04C02150384F4F4F5F4FBBE025
:107580005595479537952795BA95D1F7809169011B
:10759000682E772488249924CA01B901A401930193
:1075A0000E94BC77DC01CB01809354039093550378
:1075B000A0935603B0935703B7FF04C08150904F78
:1075C000AF4FBF4F1C012D01ACE055944794379449
:1075D0002794AA95D1F720925403309255034092F4
:1075E0005603509257038091DE079091DF07AA2738
:1075F00097FDA095BA2FBC01CD012D813E814F8111
:1076000058850E94BC7797FF04C06150784F8F4F18
:107610009F4FFBE09595879577956795FA95D1F7FC
:10762000A40193010E94BC77DC01CB018093580335
:1076300090935903A0935A03B0935B03B7FF04C020
:107640008150904FAF4FBF4F9C01AD01ECE055957D
:10765000479537952795EA95D1F7209358033093AE
:10766000590340935A0350935B03809154039091C4
:1076700055039093C6078093C50780915803909156
:1076800059039093CA078093C90722193309440903
:107690005509209358033093590340935A0350934C
:1076A0005B03E20EF31E041F151FE0922608F09202
:1076B00027080093280810932908809168018823DF
:1076C000B1F457FF04C02F5F3F4F4F4F5F4F5595A9
:1076D000479537952795A21AB30AC40AD50AA092EE
:1076E0000303B0920403C0920503D09206032A89D3
:1076F0003B8979010027F7FC0095102F80915803F2
:1077000090915903A0915A03B0915B03E80EF91EC2
:107710000A1F1B1FC801B70129813A814B815C8177
:107720000E94BC779B01AC0197FF04C02150384FE9
:107730004F4F5F4F6BE055954795379527956A9565
:10774000D1F780916A01A82EBB24CC24DD24CA0184
:10775000B901A60195010E94BC77DC01CB018093A1
:107760004C0390934D03A0934E03B0934F03B7FF88
:1077700004C08150904FAF4FBF4F3C014D013CE0E2
:1077800095948794779467943A95D1F760924C03D7
:1077900070924D0380924E0390924F03C801B7013F
:1077A0002D813E814F8158850E94BC7797FF04C090
:1077B0006150784F8F4F9F4F2BE095958795779528
:1077C00067952A95D1F7A60195010E94BC77DC0147
:1077D000CB018093500390935103A0935203B09335
:1077E0005303B7FF04C08150904FAF4FBF4FAC0160
:1077F000BD018CE075956795579547958A95D1F7AA
:10780000409350035093510360935203709353037A
:107810002A893B8937FF03C0309521953F4F21349A
:107820003105E4F1D401C30197FE07C0B095A095DE
:10783000909581959F4FAF4FBF4F81389105A1051E
:10784000B10584F4DB01CA0177FF07C0B095A095AC
:10785000909581959F4FAF4FBF4F81389105A105FE
:10786000B105E4F081E08093EF0218C01092CA07DE
:107870001092C9071092C6071092C50710925003C4
:1078800010925103109252031092530310924C0322
:1078900010924D0310924E0310924F0380915003AB
:1078A00090915103A0915203B0915303BC01CD01BB
:1078B00024E630E040E050E00E943078E0904C0355
:1078C000F0904D03E21AF30AF092DD07E092DC0734
:1078D00080914C0390914D03A0914E03B0914F03C2
:1078E000BC01CD0124E630E040E050E00E94307859
:1078F000DA01C90120915003309151038C01021B20
:10790000130B1093D1070093D007809142019091FF
:107910004301A0914401B0914501BC01CD0128E68D
:1079200031E040E050E00E94BC7720912608309181
:10793000270840912808509129082617370748073B
:10794000590764F0261B370B480B590B2093260868
:10795000309327084093280850932908209126083F
:1079600030912708409128085091290857FF0CC0F2
:10797000260F371F481F591F2093260830932708CA
:1079800040932808509329086091CE077091CF0743
:107990006E0D7F1D9B01442737FD4095542F80912C
:1079A000070390910803A0910903B0910A03820F85
:1079B000931FA41FB51F8093070390930803A09300
:1079C0000903B0930A038091C1029091C202681B1F
:1079D000790BCB01AA2797FDA095BA2F29853A8567
:1079E0004B855C85820F931FA41FB51F80930B03EB
:1079F00090930C03A0930D03B0930E03C0908201EB
:107A0000D0908301E0908401F0908501C816D906DA
:107A1000EA06FB06C4F488EA91E6A0E0B0E08C191F
:107A20009D09AE09BF0980930B0390930C03A093AB
:107A30000D03B0930E038093070390930803A09364
:107A40000903B0930A0322273327A9012C193D0902
:107A50004E095F0980910B0390910C03A0910D03D7
:107A6000B0910E0382179307A407B507B4F4D701AA
:107A7000C601885A9146A040B04080930B03909372
:107A80000C03A0930D03B0930E0380930703909310
:107A90000803A0930903B0930A036091DE07709175
:107AA000DF07600F711F9B01442737FD4095542F5E
:107AB00080910F0390911003A0911103B0911203D4
:107AC000820F931FA41FB51F80930F039093100381
:107AD000A0931103B09312038091BF029091C00252
:107AE000681B790BCB01AA2797FDA095BA2F2D858E
:107AF0003E854F855889820F931FA41FB51F809321
:107B0000130390931403A0931503B0931603E0900E
:107B10008601F09087010091880110918901E81693
:107B2000F9060A071B07C4F488EA91E6A0E0B0E072
:107B30008E199F09A00BB10B80931303909314032C
:107B4000A0931503B093160380930F039093100333
:107B5000A0931103B093120322273327A9012E19F2
:107B60003F09400B510B8091130390911403A09196
:107B70001503B091160382179307A407B507B4F451
:107B8000D801C701885A9146A040B04080931303A2
:107B900090931403A0931503B093160380930F03DF
:107BA00090931003A0931103B093120380910303E9
:107BB00090910403A0910503B091060380931703ED
:107BC00090931803A0931903B0931A0380911303A1
:107BD00090911403A0911503B09116038093330381
:107BE00090933403A0933503B093360380910B0335
:107BF00090910C03A0910D03B0910E0380932B0381
:107C000090932C03A0932D03B0932E0380910F0328
:107C100090911003A0911103B091120380932F0350
:107C200090933003A0933103B09332038091070304
:107C300090910803A0910903B0910A038093270350
:107C400090932803A0932903B0932A0380911B01EA
:107C500090911C0197FD079603E0959587950A95ED
:107C6000E1F79093DF078093DE07809119019091EF
:107C70001A0197FD079613E0959587951A95E1F7F8
:107C80009093CF078093CE078091FC019091FD01E6
:107C90000F9734F488E19CEF9093DF078093DE0721
:107CA0008091FC019091FD01079734F480E398EFF7
:107CB0009093DF078093DE07209101012A30A9F419
:107CC0008091FC019091FD01835F934034F088EE38
:107CD00093E09093DF078093DE078091FC01909101
:107CE000FD018A5F9340DCF014C08091FC0190910B
:107CF000FD01815D974034F088EE93E09093DF07BB
:107D00008093DE078091FC019091FD01805E974099
:107D100034F080ED97E09093DF078093DE07809149
:107D2000FA019091FB010F9734F488E19CEF909356
:107D3000CF078093CE078091FA019091FB010797BE
:107D400034F480E398EF9093CF078093CE072A30E6
:107D5000A9F48091FA019091FB01835F934034F084
:107D600088EE93E09093CF078093CE078091FA013D
:107D70009091FB018A5F9340DCF014C08091FA017E
:107D80009091FB01815D974034F088EE93E09093F1
:107D9000CF078093CE078091FA019091FB01805E1E
:107DA000974034F080ED97E09093CF078093CE0713
:107DB00060917401662309F4AFC040911B0150919A
:107DC0001C0180915C0390915D03481B590B5093FB
:107DD00063034093620320911B0130911C01280F23
:107DE000391F37FF02C02F5F3F4F359527953093DE
:107DF0005D0320935C03413851051CF080E890E05E
:107E000005C040585F4F34F480E89FEF90936303C0
:107E1000809362034091190150911A0180915E0391
:107E200090915F03481B590B50936103409360038B
:107E30002091190130911A01280F391F37FF02C014
:107E40002F5F3F4F3595279530935F0320935E0357
:107E5000413851051CF080E890E005C040585F4F64
:107E600034F480E89FEF9093610380936003462F82
:107E700055278091620390916303849FB001859F91
:107E8000700D949F700D11249B0177FF02C0215F3C
:107E90003F4FF4E035952795FA95E1F78091DE079D
:107EA0009091DF07820F931F9093DF078093DE0787
:107EB0008091600390916103849FD001859FB00DF4
:107EC000949FB00D1124AD019D01B7FF02C0215F49
:107ED0003F4FE4E035952795EA95E1F78091CE078D
:107EE0009091CF07820F931F9093CF078093CE0777
:107EF00080911B0190911C01860F971F90931C018C
:107F000080931B018091190190911A01840F951F94
:107F100090931A01809319010091E1071091E207F3
:107F20008091C5079091C607101611065CF59C015B
:107F300097FF04C022273327281B390BC901AA2722
:107F400097FDA095BA2F2091680133274427552724
:107F5000BC01CD010E94BC779B01AC0197FF04C01E
:107F6000215C3F4F4F4F5F4F76E0559547953795D2
:107F700027957A95D1F78091DC079091DD07820FE4
:107F8000931F27C097FF03C0909581959F4FAA2705
:107F900097FDA095BA2F20916801332744275527D4
:107FA000BC01CD010E94BC779B01AC0197FF04C0CE
:107FB000215C3F4F4F4F5F4F66E055954795379592
:107FC00027956A95D1F78091DC079091DD07821B98
:107FD000930B9093DD078093DC07E090E907F09026
:107FE000EA078091C9079091CA071E141F045CF527
:107FF0009C0197FF04C022273327281B390BC90196
:10800000AA2797FDA095BA2F20916801332744270E
:108010005527BC01CD010E94BC779B01AC0197FFA5
:1080200004C0215C3F4F4F4F5F4F96E055954795F9
:10803000379527959A95D1F78091D0079091D107E0
:10804000820F931F27C097FF03C0909581959F4F84
:10805000AA2797FDA095BA2F2091680133274427BE
:108060005527BC01CD010E94BC779B01AC0197FF55
:1080700004C0215C3F4F4F4F5F4F86E055954795B9
:10808000379527958A95D1F78091D0079091D107A0
:10809000821B930B9093D1078093D0078091160891
:1080A00087FF44C0B989BB2309F040C08091BB025F
:1080B0008823E1F5E1E0EE16E1E0FE064CF0809168
:1080C000DE079091DF078E0D9F1D805091400DC0FF
:1080D000F0E0EF16FFEFFF0664F48091DE07909169
:1080E000DF078E0D9F1D80509F4F9093DF07809379
:1080F000DE0721E0013012074CF08091CE0790910D
:10810000CF07800F911F805091400CC03FEF00308F
:10811000130764F48091CE079091CF07800F911FD1
:1081200080509F4F9093CF078093CE07E2E1CD5EC2
:108130000C9467788091D802882301F58091A10280
:108140008C7F8093A102A2E0B4E0ECEFF6E09BE02C
:108150008091B901882309F48C938D9181831282D7
:108160009150389697FFF4CF8091B901882359F048
:108170008091B90181508093B90105C08091A1021D
:1081800081608093A10280912302882319F01092CC
:108190002302089580932502809327028091210273
:1081A0008E7F8093210285EA8093BC000895CF934F
:1081B000DF93AAEDB2E0CFE2D6E057E09991E92F44
:1081C000FF27EE0FFF1FE35AF84F0190F081E02DDB
:1081D000E158FF4FEF3FF10521F01CF0EFEFF0E029
:1081E00004C0F7FF02C0E0E0F0E0993111F4EC9335
:1081F0001BC04C91242F3327E217F307A9F0CF01BE
:10820000821B930B97FD039695958795959587957A
:10821000242F280F2C93822F9927E817F90714F49D
:10822000215001C02F5F2C935150119657FFC6CF9C
:1082300080913906883F38F0EFEFF0E0E81BF10954
:10824000E652FD4F808180937A0180917A018823E4
:1082500029F0843618F084E680937A0180913B06F9
:10826000883F38F0EFEFF0E0E81BF109E652FD4FF0
:1082700080818093780180917801882329F0843669
:1082800018F084E68093780180914806883F38F0A2
:10829000EFEFF0E0E81BF109E652FD4F808180939B
:1082A0007301809173018B3010F48AE002C08F3F1C
:1082B00011F48093730180917506883F38F0EFEFD9
:1082C000F0E0E81BF109E652FD4F80818093F5074D
:1082D0008091F507863010F485E002C08F3F11F4DD
:1082E0008093F50780917706883F38F0EFEFF0E054
:1082F000E81BF109E652FD4F808180931D088091B3
:108300001D08863010F485E002C08F3F11F4809381
:108310001D0880916206873F19F4429905C006C086
:10832000863F31F4439B02C08CE80BC086E409C051
:10833000883F38F0EFEFF0E0E81BF109E652FD4F1F
:1083400080818093F20780916306873F19F44299F8
:1083500005C006C0863F31F4439B02C08CE80BC0C9
:1083600086E409C0883F38F0EFEFF0E0E81BF10940
:10837000E652FD4F80818093CB0780916406883F51
:1083800038F0EFEFF0E0E81BF109E652FD4F808195
:108390008093FB0780913A06883F38F0EFEFF0E0DA
:1083A000E81BF109E652FD4F8081809379018091AD
:1083B0003D06883F38F0EFEFF0E0E81BF109E652A8
:1083C000FD4F80818093770180913F06883F38F090
:1083D000EFEFF0E0E81BF109E652FD4F808180935A
:1083E000750180914706883F38F0EFEFF0E0E81B19
:1083F000F109E652FD4F8081809376018091490614
:10840000883F38F0EFEFF0E0E81BF109E652FD4F4E
:1084100080818093720180914A06883F38F0EFEFA7
:10842000F0E0E81BF109E652FD4F80818093740172
:1084300080914B06883F38F0EFEFF0E0E81BF10940
:10844000E652FD4F80818093710180914C06883FF8
:1084500038F0EFEFF0E0E81BF109E652FD4F8081C4
:108460008093700180915206883F38F0EFEFF0E082
:10847000E81BF109E652FD4F808180936E018091E7
:108480005306883F38F0EFEFF0E0E81BF109E652C1
:10849000FD4F80818093B60280915406883F38F06A
:1084A000EFEFF0E0E81BF109E652FD4F8081809389
:1084B000B50280915506883F38F0EFEFF0E0E81BF9
:1084C000F109E652FD4F80818093B40280915606F7
:1084D000883F38F0EFEFF0E0E81BF109E652FD4F7E
:1084E00080818093B30280917006883F38F0EFEF6F
:1084F000F0E0E81BF109E652FD4F80818093B20263
:1085000080917106883F38F0EFEFF0E0E81BF10949
:10851000E652FD4F80818093B10280917206883FC0
:1085200038F0EFEFF0E0E81BF109E652FD4F8081F3
:108530008093B00280917306883F38F0EFEFF0E04F
:10854000E81BF109E652FD4F80818093AF028091D4
:108550005706883F38F0EFEFF0E0E81BF109E652EC
:10856000FD4F808180936D0180915B06883F38F0DC
:10857000EFEFF0E0E81BF109E652FD4F80818093B8
:108580006C0180916506883F38F0EFEFF0E0E81B62
:10859000F109E652FD4F808180936B01809168065E
:1085A000883F38F0EFEFF0E0E81BF109E652FD4FAD
:1085B000808180936A0180916906883F38F0EFEFEF
:1085C000F0E0E81BF109E652FD4F808180936901DC
:1085D00080916A06883F38F0EFEFF0E0E81BF10980
:1085E000E652FD4F80818093680180919106883F1B
:1085F00038F0EFEFF0E0E81BF109E652FD4F808123
:108600008093DA079091AE03992321F08091DA07E5
:10861000981720F08091DA07882311F49093DA07F5
:108620008091370680931608809197068093FA0709
:1086300080916F06883F38F0EFEFF0E0E81BF1091A
:10864000E652FD4F80818093670180918A06883FC2
:1086500038F0EFEFF0E0E81BF109E652FD4F8081C2
:1086600080932D0880916E01282F33272F5F3F4F75
:108670008CE398E2B9010E94FB7770937C016093D0
:108680007B018091450680931E088091440680936B
:10869000E30790918C069333E0F181E08093AE0282
:1086A000983F58F0EFEFF0E0E91BF109E652FD4F7B
:1086B0008081823310F41092AE0280917D0120916E
:1086C000AE028217B1F0833088F4222319F08CEDCA
:1086D00095E002C088EC90E09093DB018093DA0192
:1086E00085E08093C30220937D0103C08150809375
:1086F0007D0180916D0890916E0897FF0FC0809169
:10870000AE02882359F08091FD0380688093FD03B9
:1087100005C01092AE028AE080937D0180916D08C1
:1087200090916E0897FF1DC08091D8028823C9F0F0
:108730008091AE028823A9F08091070190910801F1
:108740008F5F9F4F71F488E99AE39093DB018093E8
:10875000DA0180E094EA9093080180930701109277
:10876000AE028091AE02882369F08091A002816000
:108770008093A00280916A01823D48F4825E8093DA
:108780006A0105C08091A0028E7F8093A002DF91D4
:10879000CF910895A7E1B0E0E0EDF3E40C944B78BD
:1087A0000E94E8388091980682FF27C08091BD0220
:1087B0009091BE020097F1F002E088359007D4F462
:1087C0009C0197FF02C02D5F3F4F3595279535954A
:1087D000279580914F069927289FA001299F500D2A
:1087E000389F500D1124CA0164E670E00E94FB77A7
:1087F000CB0106C08DE290E003C080914F0699271F
:1088000090939F0280939E026091E3027091E40234
:108810007A8369838091E30799270A966817790715
:1088200014F49A8389838091D902843608F06AC04F
:108830008091A00282FD66C08091780390917903B7
:10884000009731F0019790937903809378030BC0E0
:108850001092D8029093A3028093A2028091A10269
:108860008D7E8093A102809101018A3011F08431C4
:1088700010F0289A01C028988091A2029091A3023A
:10888000895E9340E0F18091BC088536C0F180910B
:108890009E0290919F029A8389838091A1028061B8
:1088A0008093A10280912B06A82FBB27AA0FBB1F84
:1088B000FD01EF56F84F1182108280912C06282F6F
:1088C0003327220F331FC9018F56984FFC011182A5
:1088D0001082A35AB84F11961C921E92235A384FF9
:1088E000D90111961C921E9280912E06E82FFF2727
:1088F000EE0FFF1FE35AF84F11821082ABC21092A5
:10890000D802A8C28091D9028D3808F4A3C2809100
:10891000A1028F7E8093A1029091500682E3989FDE
:10892000C00111249093790380937803E981FA813F
:10893000B9978CF08091D802882369F08091A202C7
:108940009091A302FFEF8F3F9F0729F0019690932C
:10895000A3028093A2028091A2029091A3028F3F72
:10896000910509F008F51092FB021092FC0210929A
:10897000FD021092FE021092F7021092F80210927D
:10898000F9021092FA021092640310926503109299
:10899000660310926703109203031092040310926F
:1089A00005031092060305C08091A10282608093A6
:1089B000A10280912D06E82FFF27EE0FFF1FE35A3B
:1089C000F84F80819181813591050CF437C1209158
:1089D000D802222309F032C180912E06E82FFF270A
:1089E000EE0FFF1FE35AF84F808191818C3491057F
:1089F0000CF401C180917A038F5F80937A03893CE4
:108A000008F41CC120937A031092A3021092A202D0
:108A100030912B06E32FFF27EE0FFF1FE35AF84F8D
:108A20008081918187349105B4F480912C06E82FE0
:108A3000FF27EE0FFF1FE35AF84F808191810190CD
:108A4000F081E02DF7FF03C0F095E195FF4FE7348B
:108A5000F1050CF478C041E020912C06A22FBB2731
:108A6000AA0FBB1FA35AB84F8D919C9111978734C1
:108A7000910544F0E32FFF27EE0FFF1FE35AF84F55
:108A8000808191818D919C918734910574F08091C2
:108A90002B06E82FFF27EE0FFF1FE35AF84F8081C8
:108AA0009181873491050CF042E0E22FFF27EE0F11
:108AB000FF1FE35AF84F808191818634910574F449
:108AC00080912B06E82FFF27EE0FFF1FE35AF84F88
:108AD00080819181873491050CF043E0E22FFF27DC
:108AE000EE0FFF1FE35AF84F808191818A5B9F4F01
:108AF00074F480912B06E82FFF27EE0FFF1FE35A37
:108B0000F84F80819181873491050CF044E0E22F89
:108B1000FF27EE0FFF1FE35AF84F808191818A5B98
:108B20009F4F74F480912B06E82FFF27EE0FFF1F55
:108B3000E35AF84F80819181863491050CF445E029
:108B4000842F0E94C22A80912C06E82FFF27EE0F67
:108B5000FF1FE35AF84F808191810190F081E02D51
:108B6000F7FF03C0F095E195FF4F7E97CCF480911D
:108B70002B06E82FFF27EE0FFF1FE35AF84F8081E7
:108B800091818A5B9F4F64F481E080931804109276
:108B9000C40288EE93E09093DB018093DA014EC02B
:108BA0000E94C92B0E946F2A80E00E94CD0580910F
:108BB00051060E94D2738091160880FF10C08091E8
:108BC000130190911401875B934038F48091130155
:108BD000909114018E5E924010F40E94B31910928D
:108BE000D80180E00E94393681E08093C4028093EE
:108BF000D801579A1AC080819181855B9F4FE4F418
:108C000080917A038F5F80937A03893CB8F0209338
:108C1000D80220937A031092A3021092A20281E05C
:108C20000E94393681E08093C4020E94C92B68E714
:108C300070E00E946A3502C020937A0380912D066D
:108C4000E82FFF27EE0FFF1FE35AF84F8081918135
:108C50008B5A9F4F0CF0FEC03091D802E0912E0647
:108C6000332309F0CCC0FF27EE0FFF1FE35AF84F64
:108C700080819181855B9F4F0CF0BEC020918D0655
:108C8000E22FFF27EE0FFF1FE35AF84F80819181FB
:108C9000855B9F4F1CF0222309F0AEC080917B03BF
:108CA0008F5F80937B03893C08F4D4C030937B03AF
:108CB0008091FD03882309F098C08091C402882325
:108CC00009F493C08091B303882309F08EC081E03A
:108CD00090E09093A3028093A20281E08093D80257
:108CE000109264031092650310926603109267035A
:108CF00010920303109204031092050310920603CE
:108D00001092FF02109200031092010310920203CE
:108D100080914606E82EFF240027112780911A082B
:108D200090911B089C01442737FD4095542FC801A2
:108D3000B7010E94BC77DC01CB01809313039093B1
:108D40001403A0931503B093160380912A08909101
:108D50002B089C01442737FD4095542FC801B701CB
:108D60000E94BC77DC01CB0180930B0390930C0332
:108D7000A0930D03B0930E038091330390913403BD
:108D8000A0913503B091360380930F0390931003A5
:108D9000A0931103B093120380912B0390912C03A5
:108DA000A0912D03B0912E038093070390930803A5
:108DB000A0930903B0930A031092FB021092FC02E5
:108DC0001092FD021092FE021092F7021092F80229
:108DD0001092F9021092FA028091A10288608093A9
:108DE000A10284E68093C30235C08CED95E0909398
:108DF000DB018093DA012EC010927B032BC0FF278A
:108E0000EE0FFF1FE35AF84F808191818C3491055A
:108E1000FCF020918D06E22FFF27EE0FFF1FE35A93
:108E2000F84F80819181855B9F4F14F0222381F45C
:108E300080917C038F5F80937C03893C58F0109273
:108E4000D80210927C031092A3021092A20202C0D8
:108E500010927C0380914001815080934001809169
:108E600040018F3F21F08091A10284FFA9C30E949D
:108E7000D740B090410680918503909186039C0174
:108E8000220F331F280F391FC0902B06AC2DBB2794
:108E9000AA0FBB1FFD01E35AF84F4B2D55278081C8
:108EA0009181849FF001859FF00D949FF00D112416
:108EB0002E0F3F1F37FF02C02D5F3F4FB901759541
:108EC000679575956795AF56B84F80914206082F04
:108ED00011278D919C91809F7001819FF00C909F34
:108EE000F00C11246E0D7F1D709386036093850333
:108EF00080918703909188039C01220F331F280FD4
:108F0000391FD0902C06AD2DBB27AA0FBB1FFD012A
:108F1000E35AF84F80819181849FF001859FF00D85
:108F2000949FF00D11242E0F3F1F37FF02C02D5FBD
:108F30003F4FA9015595479555954795AF56B84F61
:108F40008D919C91809F7001819FF00C909FF00CFF
:108F500011244E0D5F1D5093880340938703809129
:108F6000AE02882309F448C0CB0177FD0396DC01EB
:108F7000B595A795B595A795CA0157FD0396FC0130
:108F8000F595E795F595E79580919C01682F7727F2
:108F900067FD70956A9F90016B9F300D7A9F300D31
:108FA00011248091B503482F552747FD50954E9FBA
:108FB000C0014F9F900D5E9F900D1124280F391F07
:108FC00037FF02C0295F3F4F93E0359527959A956B
:108FD000E1F73093EA022093E9026E9F90016F9FC0
:108FE000300D7E9F300D11244A9FC0014B9F900D84
:108FF0005A9F900D11243FC080918B06E82FFF27C8
:10900000E85BFE4F868180939C0190819093B5032D
:10901000A82FBB27A7FDB095A69F9001A79F300D55
:10902000B69F300D1124E92FFF27E7FDF095E49F4F
:10903000C001E59F900DF49F900D1124280F391F5A
:1090400037FF02C0295F3F4F83E0359527958A950A
:10905000E1F73093EA022093E902A49F9001A59FD3
:10906000300DB49F300D1124E69FC001E79F900D95
:10907000F69F900D1124281B390B37FF02C0295F82
:109080003F4F03E0359527950A95E1F73093E802C5
:109090002093E70280912E06E82FFF27EE0FFF1F97
:1090A000E35AF84F80819181909581959F4F9093DD
:1090B000E6028093E5028530910514F0049705C01F
:1090C0000FEF8C3F900734F404969093E602809360
:1090D000E50204C01092E6021092E5028091A1031D
:1090E000882309F43EC0282F33278091E90290910C
:1090F000EA0297FD079613E0959587951A95E1F793
:10910000289FA001299F500D389F500D1124CA019E
:1091100057FD0F96B4E095958795BA95E1F7909332
:10912000EA028093E9028091E7029091E80297FDBC
:109130000796A3E095958795AA95E1F7289FB0013A
:10914000299F700D389F700D1124CB0177FD0F966C
:10915000F4E095958795FA95E1F79093E80280936E
:10916000E7028090E9029090EA028091A403909136
:10917000A503881A990A9092EA028092E902009166
:10918000E7021091E8028091A2039091A303081BCB
:10919000190B1093E8020093E70280912D06E82F47
:1091A000FF27EE0FFF1FE35AF84FE080F1808FE7B3
:1091B00090E0E80EF91EF092E402E092E302809162
:1091C00073019927AA2797FDA095BA2FBC01CD015D
:1091D0000E943077DC01CB0120E030E040E251E436
:1091E000BC01CD010E949E76DC01CB01BC01CD010A
:1091F0000E940277DC01CB018093240880917201E8
:109200008093FC07809171019927AA2797FDA0956B
:10921000BA2FBC01CD010E943077DC01CB0120E0E8
:1092200030E040E251E4BC01CD010E949E76DC01B9
:10923000CB01BC01CD010E940277DC01CB01809300
:10924000D507809170018093EB078091240480FF03
:1092500059C080912D08813808F454C080911D04B4
:10926000992787FD90952B2D3327829FD001839FCF
:10927000B00D929FB00D11248A0E9B1E9092EA02AF
:109280008092E90280911E04992787FD9095829F24
:10929000F001839FF00D929FF00D11240E0F1F1F00
:1092A0001093E8020093E70280911F04282F3327D0
:1092B00027FD30958091E5029091E602820F931F81
:1092C0009093E6028093E50280912104282F3327B2
:1092D00027FD309580913C069927289F8001299F82
:1092E000100D389F100D1124109347010093460173
:1092F0008091200499278E159F0524F49093E40211
:109300008093E3028091E3029091E40297FF04C00E
:109310001092E4021092E3028091160882FF02C0CC
:109320001092FC074091E9025091EA02CA0157FDF0
:1093300003969C01359527953595279537FF03C0F2
:10934000309521953F4F8091A6029091A7028217F8
:109350009307B4F4CA0157FF03C0909581959F4FBE
:1093600097FD039695958795959587959093A70278
:109370008093A6028536910544F084E690E001C012
:1093800001979093A7028093A6024091E702509123
:10939000E802CA0157FD03969C013595279535953E
:1093A000279537FF03C0309521953F4F8091A40248
:1093B0009091A50282179307B4F4CA0157FF03C026
:1093C000909581959F4F97FD0396959587959595D7
:1093D00087959093A5028093A4028536910544F069
:1093E00084E690E001C001979093A5028093A402C7
:1093F0008091A10284FF08C01092A7021092A602D9
:109400001092A5021092A402ED2DFF27EE0FFF1F70
:10941000E35AF84F40916606242F332780819181CB
:109420002817390744F48091950682FF04C081E033
:109430008093BA0213C0ED2DFF27EE0FFF1FE35AF2
:10944000F84F842F992720916706821B910920816C
:1094500031812817390714F41092BA0240912C0672
:10946000E42FFF27EE0FFF1FE35AF84F50916606D7
:10947000852F992722273327281B390B808191813B
:109480008217930744F48091950683FF04C081E01E
:109490008093B90216C08091B902882391F0E42F1D
:1094A000FF27EE0FFF1FE35AF84F809167069927B9
:1094B000851B9109208131818217930714F4109242
:1094C000B902EC2DFF27EE0FFF1FE35AF84F409132
:1094D0006606242F3327808191812817390744F4A9
:1094E0008091950680FF04C081E08093B70217C089
:1094F0008091B702882399F0EC2DFF27EE0FFF1F14
:10950000E35AF84F842F992720916706821B91090F
:10951000208131812817390714F41092B702409145
:109520002B06E42FFF27EE0FFF1FE35AF84F509151
:109530006606852F992722273327281B390B808120
:1095400091818217930744F48091950681FF04C0AE
:1095500081E08093B80216C08091B802882391F010
:10956000E42FFF27EE0FFF1FE35AF84F80916706A5
:109570009927851B9109208131818217930714F463
:109580001092B8028091BA02882319F48091B9022E
:10959000811181E08093BB028091B702882321F47E
:1095A0008091B802882351F081E08093BC02109230
:1095B000BB021092BA021092B90202C08093BC02A0
:1095C0008091BB02882321F48091BC02882369F03A
:1095D00080916506992729813A818217930714F4AF
:1095E0009A83898381E08093EF028091A00299277A
:1095F0009C012470307082FF2DC08091A403909153
:10960000A503909581959F4F9093EA028093E9027C
:109610008091A2039091A303909581959F4F909381
:10962000E8028093E70280918001909181019093FC
:10963000E4028093E302809116088B778B66809317
:1096400016088091FA078C7B8093FA0788EC809348
:1096500079011EC08091A10284FF1AC03093E602F6
:109660002093E5023093EA022093E9023093E80266
:109670002093E7029AE59093240888E78093FC07FB
:109680009093D5078093EB071092BB021092BC0217
:109690008091EE079091EF07A091F007B091F1074C
:1096A00020913303309134034091350350913603B8
:1096B000820F931FA41FB51F8093EE079093EF07AF
:1096C000A093F007B093F1078091F6079091F70708
:1096D000A091F807B091F907E0902B03F0902C03CC
:1096E00000912D0310912E03EB82FC820D831E83CB
:1096F0008E0D9F1DA01FB11F8093F6079093F70753
:10970000A093F807B093F9078091E5079091E607D9
:10971000A091E707B091E807E0902F03F0903003A5
:109720000091310310913203EF82F88609871A877E
:109730008E0D9F1DA01FB11F8093E5079093E60734
:10974000A093E707B093E8078091D6079091D707D9
:10975000A091D807B091D907E0902703F090280393
:109760000091290310912A03EB86FC860D871E8742
:109770008E0D9F1DA01FB11F8093D6079093D70712
:10978000A093D807B093D907F090BC02FF86FF20C2
:1097900029F48091BB02882309F460C0109223034E
:1097A00010922403109225031092260310921F0397
:1097B0001092200310922103109222031092EE07C0
:1097C0001092EF071092F0071092F1071092F6072F
:1097D0001092F7071092F8071092F9071092E50718
:1097E0001092E6071092E7071092E8071092D6074A
:1097F0001092D7071092D8071092D90780911303BF
:1098000090911403A0911503B091160380930F0358
:1098100090931003A0931103B093120380910B0354
:1098200090910C03A0910D03B0910E038093070358
:1098300090930803A0930903B0930A031092EA01DE
:109840001092E9011092C0021092BF021092C2025F
:109850001092C1020F85002309F0F8C18091BB026C
:10986000882309F0F3C18091CC059091CD058150FA
:1098700092402CF48091D802882309F4E7C190909B
:10988000A608A090460620901A0830901B08409029
:109890002A0850902B0819140CF0E3C0BB24CC24E8
:1098A000DD24CA01B901A60195010E943078790131
:1098B0008A0180916F0890917008281A390AC101B5
:1098C000AA2797FDA095BA2FE81AF90A0A0B1B0BD5
:1098D0006B817C818D819E81A60195010E943078EB
:1098E00059016A018091710890917208481A590AC9
:1098F000C201AA2797FDA095BA2FA81AB90ACA0AC9
:10990000DB0A292C332427FC3094432C532CC80128
:10991000B701A20191010E94BC7797FF04C061507A
:109920007E4F8F4F9F4F3B014C0109E095948794E8
:10993000779467940A95D1F7C601B501A201910108
:109940000E94BC7797FF04C061507E4F8F4F9F4F9E
:109950005B016C0119E0D594C794B794A7941A954C
:10996000D1F78091A6029091A702813491053CF431
:109970008091A4029091A50281349105D4F0D40184
:10998000C30197FE03C00196A11DB11D3C014D010D
:109990009594879477946794D601C501D7FE03C048
:1099A0000196A11DB11D5C016D01D594C794B794BA
:1099B000A79480912E06E82FFF27EE0FFF1FE35A92
:1099C000F84F808191810190F081E02DF7FF03C075
:1099D000F095E195FF4F7A97A4F0C401B30123E01D
:1099E00030E040E050E00E94307839014A01C60181
:1099F000B50123E030E040E050E00E9430785901AA
:109A00006A018091A808282F332727FD3095432F1E
:109A1000532F261537054805590514F439014A0115
:109A2000992787FD9095909581959F4FAA2797FD3F
:109A3000A095BA2F681679068A069B0614F43C0195
:109A40004D012A153B054C055D0514F459016A01C9
:109A5000A816B906CA06DB060CF0D0C05C016D0181
:109A6000CDC0EA2CFF2400271127CA01B901A801A3
:109A700097010E94307839014A01C101AA2797FD58
:109A8000A095BA2F681A790A8A0A9B0A6B817C8191
:109A90008D819E81A80197010E94307859016A0149
:109AA000C201AA2797FDA095BA2FA81AB90ACA0A17
:109AB000DB0AD401C30197FE03C00F96A11DB11D9F
:109AC0003C014D01F4E09594879477946794FA955E
:109AD000D1F7D601C501D7FE03C00F96A11DB11D58
:109AE0005C016D01E4E0D594C794B794A794EA951E
:109AF000D1F78091A6029091A702813491053CF4A0
:109B00008091A4029091A50281349105A4F0C40132
:109B1000B30123E030E040E050E00E9430783901AA
:109B20004A01C601B50123E030E040E050E00E9468
:109B3000307859016A0180912E06E82FFF27EE0F39
:109B4000FF1FE35AF84F808191810190F081E02D51
:109B5000F7FF03C0F095E195FF4F7A97A4F0C40199
:109B6000B30123E030E040E050E00E94307839015A
:109B70004A01C601B50123E030E040E050E00E9418
:109B8000307859016A0189E180938C0121E26216E3
:109B90007104810491042CF070E2672E712C812CE9
:109BA000912C30EE63163FEF73063FEF83063FEFD5
:109BB000930644F460EE662E6FEF762E6FEF862EDE
:109BC0006FEF962E41E2A416B104C104D1042CF02B
:109BD00050E2A52EB12CC12CD12C50EEA5165FEF72
:109BE000B5065FEFC5065FEFD50644F440EEA42E40
:109BF0004FEFB42E4FEFC42E4FEFD42E80911303AE
:109C000090911403A0911503B0911603861997093A
:109C1000A809B9098093130390931403A093150323
:109C2000B093160380910B0390910C03A0910D0348
:109C3000B0910E038A199B09AC09BD0980930B03EF
:109C400090930C03A0930D03B0930E038091E90150
:109C50009091EA018F3F910509F008F4C4C56F8522
:109C6000662309F04EC58091BB02882309F049C5DF
:109C70008091EF02882309F044C570916E06788BBD
:109C8000772309F43EC58091EE079091EF07A091EC
:109C9000F007B091F107B7FF04C081509F4FAF4F5D
:109CA000BF4FE92EFA2E0B2F112707FD1A95E092D0
:109CB000EE07F092EF070093F0071093F107809101
:109CC000F6079091F707A091F807B091F907B7FF51
:109CD00004C081509F4FAF4FBF4F892F9A2FAB2F9A
:109CE000BB27A7FDBA95898B9A8BAB8BBC8B8093D6
:109CF000F6079093F707A093F807B093F9078091C0
:109D00004606A82EBB24CC24DD24209123033091C9
:109D100024034091250350912603C601B5010E94FA
:109D2000BC7797FF04C061507F4F8F4F9F4F672EC6
:109D3000782E892E992487FC9A946092230370923E
:109D40002403809225039092260320911F033091D3
:109D500020034091210350912203C601B5010E94C6
:109D6000BC7797FF04C061507F4F8F4F9F4F272EC6
:109D7000382E492E552447FC5A9420921F033092C6
:109D80002003409221035092220380911B03909163
:109D90001C03A0911D03B0911E03B7FF04C08150A6
:109DA0009F4FAF4FBF4F892F9A2FAB2FBB27A7FDD8
:109DB000BA9580931B0390931C03A0931D03B0934B
:109DC0001E03D801C70186199709A809B90980930C
:109DD000700390937103A0937203B0937303209167
:109DE0006D06E22EFF2400271127BC01CD01A8013A
:109DF00097010E94307859016A0120937D033093C6
:109E00007E0340937F035093800389899A89AB89AD
:109E1000BC8982199309A409B509809374039093AE
:109E20007503A0937603B0937703BC01CD01A8011D
:109E300097010E94307820938103309382034093EE
:109E4000830350938403D601C501D7FE04C081501B
:109E50009F4FAF4FBF4F892F9A2FAB2FBB27A7FD27
:109E6000BA959093C0028093BF0257FF04C021505F
:109E70003F4F4F4F5F4FBB2757FDBA95A52F942FEC
:109E8000832F9093C2028093C1028091A602909189
:109E9000A70281349105DCF48091A4029091A5027F
:109EA00081349105A4F480912E06E82FFF27EE0F50
:109EB000FF1FE35AF84F808191810190F081E02DDE
:109EC000F7FF03C0F095E195FF4F7A97E4F080919A
:109ED000A6088F3FC1F48091BF029091C00297FD08
:109EE0000196959587959093C0028093BF028091CB
:109EF000C1029091C20297FD019695958795909326
:109F0000C2028093C1028091E5079091E607A0917B
:109F1000E707B091E807B7FF04C081509F4FAF4FEC
:109F2000BF4F892F9A2FAB2FBB27A7FDBA958093E0
:109F3000E5079093E607A093E707B093E8078091C1
:109F4000D6079091D707A091D807B091D907B7FF4E
:109F500004C081509F4FAF4FBF4F892F9A2FAB2F17
:109F6000BB27A7FDBA958093D6079093D707A093F8
:109F7000D807B093D9078091330390913403A0910F
:109F80003503B09136032F81388549855A85281BC2
:109F9000390B4A0B5B0B20936803309369034093A2
:109FA0006A0350936B0380912B0390912C03A09133
:109FB0002D03B0912E03EB84FC840D851E85E81AD9
:109FC000F90A0A0B1B0BE0926C03F0926D030093ED
:109FD0006E0310936F0320937003309371034093CB
:109FE000720350937303E0927403F092750300932D
:109FF00076031093770380910F0390911003A09143
:10A000001103B0911203821B930BA40BB50B809329
:10A010000F0390931003A0931103B0931203809148
:10A02000070390910803A0910903B0910A038E19C8
:10A030009F09A00BB10B8093070390930803A09393
:10A040000903B0930A0388898823E1F02091ED0287
:10A050003091EE02213831054CF08091440390910B
:10A0600045030196909345038093440320583F4F46
:10A070004CF48091440390914503019790934503DC
:10A08000809344031092EE021092ED0281E090E082
:10A0900090938A0380938903E0907003F09071039A
:10A0A0000091720310917303D801C70117FF07C015
:10A0B00088279927DC018E199F09A00BB10B8150CD
:10A0C0009240A040B04034F084E090E090938A0346
:10A0D0008093890380918F0390919003A0919103C5
:10A0E000B09192032091EE073091EF074091F00775
:10A0F0005091F107821B930BA40BB50B815E914B22
:10A10000AF4FBF4F8F539C49A040B04028F0809183
:10A11000A70889310CF4FFC021E0E21620E1F20625
:10A1200020E0020720E012070CF473C080918B033B
:10A13000882309F46AC0D801C70117FF07C0882720
:10A140009927DC018E199F09A00BB10B9C01AD0171
:10A15000B7FF04C021503E4F4F4F5F4FF9E0559578
:10A16000479537952795FA95D1F780918903909176
:10A170008A03820F931F90938A0380938903D801E7
:10A18000C70117FF03C00796A11DB11DE3E0B595F8
:10A19000A79597958795EA95D1F780937D0390933E
:10A1A0007E03A0937F03B093800389589341A0401E
:10A1B000B04064F088E893E1A0E0B0E080937D03D4
:10A1C00090937E03A0937F03B093800320917D033F
:10A1D00030917E0340917F035091800357FF04C06C
:10A1E00021503F4F4F4F5F4F232F342F452F55277F
:10A1F00047FD5A958091BF029091C002820F931F34
:10A200009093C0028093BF0206C081E080938B03CD
:10A2100002C010928B0340E0E41640EFF4064FEFCB
:10A2200004074FEF14070CF073C080918C03882350
:10A2300009F46AC0D801C70117FF07C0882799270A
:10A24000DC018E199F09A00BB10B9C01AD01B7FF7A
:10A2500004C021503E4F4F4F5F4F69E055954795E1
:10A26000379527956A95D1F78091890390918A0354
:10A27000820F931F90938A0380938903D801C701AB
:10A2800017FF03C00796A11DB11D23E0B595A79543
:10A29000979587952A95D1F780937D0390937E03B8
:10A2A000A0937F03B093800388579C4EAF4FBF4F5E
:10A2B00064F488E79CEEAFEFBFEF80937D0390934B
:10A2C0007E03A0937F03B093800320917D033091A0
:10A2D0007E0340917F035091800357FF04C02150BB
:10A2E0003F4F4F4F5F4F232F342F452F552747FDAB
:10A2F0005A958091BF029091C002820F931F909354
:10A30000C0028093BF0211C081E080938C030DC016
:10A3100010928C030AC010928A031092890384E67B
:10A3200090E090938B0180938A016889262F3327D0
:10A330008091890390918A032817390724F4309378
:10A340008A03209389031091A708112379F0212F04
:10A35000332727FD30958091890390918A03281730
:10A36000390724F430938A032093890340917003C2
:10A3700050917103609172037091730341385105DC
:10A380006105710574F08091480390914903209113
:10A39000890330918A03820F931F9093490380931E
:10A3A000480340585F4F6F4F7F4F74F480914803CC
:10A3B000909149032091890330918A03821B930B6A
:10A3C000909349038093480381E090E090938A033F
:10A3D00080938903C0907403D0907503E090760356
:10A3E000F0907703D701C601F7FE07C088279927A9
:10A3F000DC018C199D09AE09BF0981509240A04033
:10A40000B04034F084E090E090938A038093890315
:10A410008091930390919403A0919503B09196033A
:10A420002091F6073091F7074091F8075091F9070E
:10A43000821B930BA40BB50B815E914BAF4FBF4FAB
:10A440008F539C49A040B04018F019310CF4FFC064
:10A4500001E0C01600E1D00600E0E00600E0F006F2
:10A460000CF473C080918D03882309F46AC0D7016E
:10A47000C601F7FE07C088279927DC018C199D09C2
:10A48000AE09BF099C01AD01B7FF04C021503E4F8A
:10A490004F4F5F4F09E055954795379527950A959A
:10A4A000D1F78091890390918A03820F931F909333
:10A4B0008A0380938903D701C601F7FE03C007967C
:10A4C000A11DB11D13E0B595A795979587951A9590
:10A4D000D1F78093810390938203A0938303B09379
:10A4E000840389589341A040B04064F088E893E128
:10A4F000A0E0B0E08093810390938203A093830354
:10A50000B0938403209181033091820340918303AF
:10A510005091840357FF04C021503F4F4F4F5F4F6E
:10A52000232F342F452F552747FD5A958091C1027F
:10A530009091C202820F931F9093C2028093C10236
:10A5400006C081E080938D0302C010928D0320E04D
:10A55000C21620EFD2062FEFE2062FEFF2060CF024
:10A5600073C080918E03882309F46AC0D701C601A5
:10A57000F7FE07C088279927DC018C199D09AE09D1
:10A58000BF099C01AD01B7FF04C021503E4F4F4FA2
:10A590005F4FE9E05595479537952795EA95D1F7AF
:10A5A0008091890390918A03820F931F90938A036D
:10A5B00080938903D701C601F7FE03C00796A11D4A
:10A5C000B11D73E0B595A795979587957A95D1F7C5
:10A5D0008093810390938203A0938303B0938403B9
:10A5E00088579C4EAF4FBF4F64F488E79CEEAFEFA7
:10A5F000BFEF8093810390938203A0938303B09372
:10A600008403209181033091820340918303509110
:10A61000840357FF04C021503F4F4F4F5F4F232FFC
:10A62000342F452F552747FD5A958091C1029091AF
:10A63000C202820F931F9093C2028093C10211C085
:10A6400081E080938E030DC010928E030AC0109299
:10A650008A031092890384E690E090938B018093A3
:10A660008A014889242F33278091890390918A0396
:10A670002817390724F430938A03209389038091A3
:10A68000A708882379F0282F332727FD309580915C
:10A69000890390918A032817390724F430938A0399
:10A6A0002093890340917403509175036091760360
:10A6B00070917703413851056105710574F08091FF
:10A6C0004603909147032091890330918A03820FBA
:10A6D000931F909347038093460340585F4F6F4FFB
:10A6E0007F4FCCF4809146039091470320918903DA
:10A6F00030918A03821B930B909347038093460308
:10A700000AC01092C2021092C1021092C0021092AE
:10A71000BF021092EF028091FC07882341F410924F
:10A72000C2021092C1021092C0021092BF02809128
:10A73000EE079091EF07A091F007B091F107809399
:10A740008F0390939003A0939103B0939203809111
:10A75000F6079091F707A091F807B091F907809359
:10A76000930390939403A0939503B0939603109250
:10A7700023031092240310922503109226031092B3
:10A780001F031092200310922103109222031092B3
:10A790001B0310921C0310921D0310921E031092B3
:10A7A000EE071092EF071092F0071092F107109247
:10A7B000F6071092F7071092F8071092F907109217
:10A7C000E5071092E6071092E7071092E80710924B
:10A7D000D6071092D7071092D8071092D907109277
:10A7E000EA011092E901E090E502F090E602C7016B
:10A7F000F7FE04C0882799278E199F0904973CF01B
:10A800008091160884FD03C082E38093C3021091F7
:10A810004306A12EBB24CC24DD24B701882777FD75
:10A820008095982F9701F7FE04C0222733272E1911
:10A830003F09442737FD4095542F0E94BC779B0168
:10A84000AC01C601B5010E94BC7797FF04C06150FE
:10A850007E4F8F4F9F4F59E09595879577956795D8
:10A860005A95D1F79B01812F99278E9DD0018F9DFD
:10A87000B00D9E9DB00D1124CD01B7FD03969595A9
:10A88000879595958795280F391F8091C5029091DE
:10A89000C602280F391F442737FD4095542F2093B7
:10A8A000640330936503409366035093670380917C
:10A8B000030390910403A0910503B0910603821B4A
:10A8C000930BA40BB50B8093030390930403A09305
:10A8D0000503B09306038155934CA040B04064F04B
:10A8E00080E593ECA0E0B0E0809303039093040331
:10A8F000A0930503B0930603809103039091040392
:10A90000A0910503B0910603805B9C43AF4FBF4FFE
:10A9100064F480EB9CE3AFEFBFEF8093030390936D
:10A920000403A0930503B093060300918E011091D8
:10A930008F0117FDFCC08091160883FFF8C080913D
:10A940008D01815080938D01882309F0F4C08DE042
:10A9500080938D018091330390913403A09135034E
:10A96000B0913603B7FF04C081509E4FAF4FBF4F29
:10A9700039E0B595A795979587953A95D1F77C01DC
:10A9800097FF04C0F094E194F108F39480912B03B5
:10A9900090912C03A0912D03B0912E03B7FF04C01A
:10A9A00081509E4FAF4FBF4F29E0B595A795979522
:10A9B00087952A95D1F79C0197FF03C03095219583
:10A9C0003F4FE216F3060CF47901B701F7FE02C01F
:10A9D000695F7F4F2B01A3E055944794AA95E1F757
:10A9E00022E030E0420E531E609026087090270847
:10A9F00080902808909029082091420130914301CD
:10AA00004091440150914501C401B3010E94307846
:10AA100059016A013093D4072093D307021B130B0B
:10AA2000C801845E9D4F68E671E00E94FB779C013F
:10AA3000245B304080918A0190918B01009731F026
:10AA4000019790938B0180938A011BC049E1E41622
:10AA5000F104BCF48091ED029091EE02820F931FFD
:10AA60009093EE028093ED028091C302882349F017
:10AA700081508093C302882321F4B092F202A09205
:10AA8000F10280918A0190918B01892BF9F48091D8
:10AA90008C019927289FB001299F700D389F700D58
:10AAA0001124CB01B2010E94FB77CB01AA2797FDAD
:10AAB000A095BA2F680E791E8A1E9B1E60922608EA
:10AAC0007092270880922808909229088091C302EA
:10AAD000882369F58091F1029091F2022091D307C9
:10AAE0003091D407821B930B845E9D4F68E671E022
:10AAF0000E94FB779C01245B304080917601869513
:10AB00009927289FD001299FB00D389FB00D11249F
:10AB10009D01B7FF02C0215F3F4FF4E035952795B7
:10AB2000FA95E1F73093C6022093C50204C0109253
:10AB3000C6021092C5028091EF02882381F0109224
:10AB4000F7021092F8021092F9021092FA02109293
:10AB5000FB021092FC021092FD021092FE02F09095
:10AB6000BC02FF20F1F48091FC07282F33274427F3
:10AB700055278091330390913403A0913503B09110
:10AB80003603BC01CD010E94BC77DC01CB01BC01C6
:10AB9000CD0128EF3AE240E050E00E9430783901E0
:10ABA00002C066247724E090BB02EE20F1F480918D
:10ABB000FC07282F33274427552780912B0390919A
:10ABC0002C03A0912D03B0912E03BC01CD010E9456
:10ABD000BC77DC01CB01BC01CD0128EF3AE240E0BB
:10ABE00050E00E943078290102C04424552480910D
:10ABF000D0079091D107893C91051CF088EC90E03A
:10AC000005C088539F4F34F488E39FEF9093D1079A
:10AC10008093D0078091DC079091DD07893C9105F6
:10AC20001CF088EC90E005C088539F4F34F488E313
:10AC30009FEF9093DD078093DC078091DE07909172
:10AC4000DF07AA2797FDA095BA2F20912408A22EEE
:10AC5000BB24CC24DD24BC01CD01A60195010E94BA
:10AC6000BC779B01AC018091D0079091D107AA27B6
:10AC700097FDA095BA2FE7E0880F991FAA1FBB1F69
:10AC8000EA95D1F7280F391F4A1F5B1F57FF04C0F1
:10AC9000215C3F4F4F4F5F4F76E055954795379575
:10ACA00027957A95D1F78301020F131F1093DF07C1
:10ACB0000093DE078091CE079091CF07AA2797FDDA
:10ACC000A095BA2FBC01CD01A60195010E94BC77C9
:10ACD0009B01AC018091DC079091DD07AA2797FDCD
:10ACE000A095BA2F67E0880F991FAA1FBB1F6A950E
:10ACF000D1F7280F391F4A1F5B1F57FF04C0215C83
:10AD00003F4F4F4F5F4FF6E0559547953795279545
:10AD1000FA95D1F74201820E931E9092CF0780924E
:10AD2000CE0780911F0890912008880F991FAA27AD
:10AD300097FDA095BA2F2091D50733274427552793
:10AD4000BC01CD010E94BC775B016C0197FF08C07C
:10AD50002FE330E040E050E0A20EB31EC41ED51E2B
:10AD6000E6E0D594C794B794A794EA95D1F780917B
:10AD7000EB07282F332744275527809117039091FD
:10AD80001803A0911903B0911A03BC01CD010E94D0
:10AD9000BC77DC01CB01BC01CD0120EF35E540E003
:10ADA00050E00E943078B501620F731F7093200845
:10ADB00060931F080150104134F080E090E19093BF
:10ADC000DF078093DE078091DE079091DF078050D8
:10ADD000904F34F480E090EF9093DF078093DE078C
:10ADE00051E0851650E1950634F080E090E19093B3
:10ADF000CF078093CE078091CE079091CF078050E8
:10AE0000904F34F480E090EF9093CF078093CE077B
:10AE10006150704134F080E090E19093200880937D
:10AE20001F0880911F08909120088050904F34F4A3
:10AE300080E090EF9093200880931F08809100019C
:10AE4000482F552780911D0190911E0148175907E1
:10AE500094F420911D0130911E0109811A81049FF3
:10AE6000C001059F900D149F900D1124B9010E94FF
:10AE7000E7777A83698329813A81220F331F220F72
:10AE8000331F3A8329834091160840FD02C00C9479
:10AE9000375FEE2009F0EBC7FF2009F0E8C700E0BC
:10AEA00010E048018091BD029091BE029093B405DC
:10AEB0008093B30520914A0330914B03211531054E
:10AEC00009F03FC08091130190911401895993407A
:10AED00058F087B5853F20F48091ED01815011C075
:10AEE00081E08093A0034EC08091130190911401E2
:10AEF0008436910508F587B58B30D0F08091ED014F
:10AF00008F5F8093ED019AE0890290011124809176
:10AF1000D605821B87BD8CE291E09093DB01809384
:10AF2000DA018EE591E090934B0380934A032AC0A7
:10AF300081E080939F0326C0F0929F03F092A003CC
:10AF400021C08091D3029091D402A091D502B091FA
:10AF5000D60264E0880F991FAA1FBB1F6A95D1F71C
:10AF60008093EE019093EF01A093F001B093F10173
:10AF70001093EC010093EB012150304030934B03D0
:10AF800020934A032091790141FF24C02233D8F451
:10AF9000809190018150809390018F3FD9F510925C
:10AFA000F0028091D3029091D402A091D502B09189
:10AFB000D6028093CF029093D002A093D102B09397
:10AFC000D20281E004C081E08093F00288EC80939B
:10AFD000900120C08091460190914701820F911D00
:10AFE00020913C063327829FA001839F500D929FA2
:10AFF000500D1124CA01AA2797FDA095BA2F80935E
:10B00000CF029093D002A093D102B093D20281E0FC
:10B010008093F0028091330390913403A091350323
:10B02000B0913603E0904201F09043010091440159
:10B0300010914501BC01CD01A80197010E94307813
:10B0400059016A0180912B0390912C03A0912D034B
:10B05000B0912E03BC01CD01A80197010E94307868
:10B06000B901C5010E947E6D5C01CC971CF05CE3C8
:10B07000A52EB12CC5010E94426C5C0180E2809338
:10B0800041011092CE021092CD028091F0028823ED
:10B0900009F45FC58091A10299279C01207130704D
:10B0A00084FD57C58091A00282608093A0027091B8
:10B0B000FA07872F992741E0C42ED12CC822D92224
:10B0C00080FD04C08091160881FD10C0C980DA801F
:10B0D00030939803209397033093CE022093CD02B0
:10B0E0008091A102806C8093A102ABC28091A102E9
:10B0F00081FF7AC20091800110918101C8010F96F1
:10B100002090E3023090E402821593050CF058C0C1
:10B1100080919F03882309F053C08091A10287FF8B
:10B1200015C08091A1028F778093A1028091D302F4
:10B130009091D402A091D502B091D6028093CF0213
:10B140009093D002A093D102B093D2028091A10239
:10B1500080648093A102E090DA07EE20F1F0809104
:10B16000CF029091D002A091D102B091D202BC0145
:10B17000CD0124E630E040E050E00E9430788E2D92
:10B180009927AA27BB2782179307A407B5072CF492
:10B19000D092CE02C092CD0210C0C101801B910B93
:10B1A0000F9797FF03C0909581959F4F9093CE0284
:10B1B0008093CD028BE2809341011092C70216C1A9
:10B1C000C8010F9728163906C4F52091A003222341
:10B1D000A1F58091A10286FF15C08091A1028F7B0D
:10B1E0008093A1028091D3029091D402A091D502C4
:10B1F000B091D6028093CF029093D002A093D10257
:10B20000B093D2028091A10280688093A102C10113
:10B21000801B910B0F9697FF03C0909581959F4FD0
:10B22000909581959F4F9093CE028093CD028DE2B1
:10B23000809341012093C702D9C08DE380934101DF
:10B240006091C802662371F12091C9023091CA024F
:10B250004091CB025091CC028091CF029091D002CC
:10B26000A091D102B091D20282179307A407B5072B
:10B27000CCF48091A10280648093A102862F99274B
:10B280009093CE028093CD028AE08093C7028EE530
:10B29000809341018091A10287FFA8C08091A10203
:10B2A0008F7733C0662309F443C02091C9023091DF
:10B2B000CA024091CB025091CC028091CF02909172
:10B2C000D002A091D102B091D202281739074A07C3
:10B2D0005B0774F58091A10280688093A102862F9C
:10B2E0009927909581959F4F9093CE028093CD02A0
:10B2F00086EF8093C70286E7809341018091A10287
:10B3000086FF74C08091A1028F7B8093A1028091FF
:10B31000D3029091D402A091D502B091D60280932D
:10B32000CF029093D002A093D102B093D2025EC01C
:10B330008091A102807C09F459C08091C7028823C2
:10B3400079F5E090D302F090D4020091D5021091EB
:10B35000D602D801C70180589040A040B04020914B
:10B36000CF023091D0024091D1025091D202821787
:10B370009307A407B5075CF4D801C70180589F4F15
:10B38000AF4FBF4F281739074A075B075CF0809320
:10B39000CF029093D002A093D102B093D20202C008
:10B3A0001092C7028091A1028F738093A102109224
:10B3B00098031092970371FF06C084EF91E0909379
:10B3C000DB018093DA018091D702882379F48091A0
:10B3D000D3029091D402A091D502B091D602C39726
:10B3E000A105B1051CF081E08093D702609197031D
:10B3F000709198038091CD029091CE02680F791FD1
:10B400007093980360939703CB0177FF04C088275C
:10B410009927861B970B855F91400CF4CEC0409115
:10B42000C702442389F18091C9029091CA022091F8
:10B43000CF023091D002821B930B0996439748F4B8
:10B440008091C9029091CA02A091CB02B091CC0226
:10B4500012C0242F332727FD3095432F532F80917F
:10B46000CF029091D002A091D102B091D202820F6E
:10B47000931FA41FB51F8093CF029093D002A09377
:10B48000D102B093D20224C080913C062091CF0219
:10B490003091D0024091D1025091D2021616170677
:10B4A00044F463E00E94DB77280F311D411D511DDC
:10B4B00007C063E00E94DB77281B3109410951096D
:10B4C0002093CF023093D0024093D1025093D20206
:10B4D0001092980310929703E090D302F090D40258
:10B4E0000091D5021091D602D801C7018050944036
:10B4F000A040B0402091CF023091D0024091D102C3
:10B500005091D20282179307A407B5075CF4D801C3
:10B51000C70180509C4FAF4FBF4F281739074A07CC
:10B520005B0744F08093CF029093D002A093D102A6
:10B53000B093D2028091FA0781FF06C084E690E0C2
:10B540009093DB018093DA01809140068823A9F56E
:10B550008091C802882389F54091BD025091BE02B6
:10B5600057FF02C04D5F5F4F5595479555954795DD
:10B5700080911D0190911E01209100013327489F69
:10B58000F001499FF00D589FF00D1124CF01B90132
:10B590000E94FB777093810160938001663471058E
:10B5A0001CF486E490E005C06739710534F086E943
:10B5B00090E0909381018093800180914A03909163
:10B5C0004B03892BD1F18091D3029091D402A091A9
:10B5D000D502B091D6028093CF029093D002A0936F
:10B5E000D102B093D20229C08091D3029091D402AB
:10B5F000A091D502B091D60280599140A040B040B0
:10B600008093CF029093D002A093D102B093D20244
:10B6100080914006882311F0992702C088E790E0C6
:10B620009093810180938001E980FA80F092BE02BC
:10B63000E092BD028EE280934101C090BD02D090A5
:10B64000BE02E090D302F090D4020091D502109196
:10B65000D6022091CF023091D0024091D102509178
:10B66000D2022E153F054007510724F08091FA07BA
:10B6700080FDBBC280914A0390914B03892B39F026
:10B68000C090BD02D090BE0200E010E0D7C0D8014B
:10B69000C701821B930BA40BB50B80936803909397
:10B6A0006903A0936A03B0936B03823000E89007AC
:10B6B0000FEFA0070FEFB0072CF481E090E8AFEF99
:10B6C000BFEF09C08F5F9F47A040B04064F08FEF8D
:10B6D0009FE7A0E0B0E08093680390936903A09394
:10B6E0006A03B0936B030091680310916903809122
:10B6F0007801282F3327442755278091680390919C
:10B700006903A0916A03B0916B03BC01CD010E9453
:10B71000BC7797FF04C0615E7F4F8F4F9F4F25E03E
:10B7200095958795779567952A95D1F760936803E6
:10B730007093690380936A0390936B0365302EEFD7
:10B7400072072FEF82072FEF92072CF484E09EEF11
:10B75000AFEFBFEF09C0605074408040904064F08C
:10B7600080E094E0A0E0B0E08093680390936903E8
:10B77000A0936A03B0936B03809068039090690371
:10B780002091EB013091EC0137FF02C0295F3F4F60
:10B7900083E0359527958A95E1F74FEF22383407F6
:10B7A0001CF421E83FEF05C02038310514F020E8F3
:10B7B00030E0C901AA2797FDA095BA2F20917A0100
:10B7C000332744275527BC01CD010E94BC7797FF42
:10B7D00004C06D5F7F4F8F4F9F4FB2E09595879567
:10B7E00077956795BA95D1F79B015FEF6130750743
:10B7F0001CF420E03FEF06C06F3F710519F014F014
:10B8000020E031E08091A102807C49F0C90137FD40
:10B8100003969C0135952795359527950DC0809108
:10B82000FA0780FF09C0C90137FD07969C01F3E0C4
:10B8300035952795FA95E1F7820E931E20917701B1
:10B84000222309F454C06091F3027091F4028091B4
:10B85000F5029091F60297FF04C061587F4F8F4F19
:10B860009F4FE7E09595879577956795EA95D1F78E
:10B870003327442755270E94BC7797FF04C0615E99
:10B880007F4F8F4F9F4F55E095958795779567959B
:10B890005A95D1F7609368037093690380936A03A4
:10B8A00090936B036138AFEF7A07AFEF8A07AFEF82
:10B8B0009A072CF480E89FEFAFEFBFEF0AC06F3F0D
:10B8C00071058105910569F064F080E091E0A0E0E8
:10B8D000B0E08093680390936903A0936A03B093E8
:10B8E0006B038091680390916903880E991E809183
:10B8F0007501282F33278091AA08992787FD9095F5
:10B90000289FF001299FF00D389FF00D11249F0111
:10B91000F7FF02C021583F4F220F232F221F330B66
:10B92000FFEF21383F071CF420E83FEF06C02F3F10
:10B93000310519F014F020E031E0820E931EC401AD
:10B94000AA2797FDA095BA2FE090BD02F090BE0205
:10B950009701442737FD4095542FBC01CD010E942B
:10B96000BC7797FF04C061507E4F8F4F9F4F29E0F7
:10B9700095958795779567952A95D1F7C61AD70A31
:10B980008091CD029091CE02892B09F060C01E14E7
:10B990001F040CF05CC0980117FF03C0309521957F
:10B9A0003F4F2D33310540F48091EB029091EC0232
:10B9B0008C159D0574F526C02C53304085E03695D6
:10B9C00027958A95E1F72031310510F02FE030E01E
:10B9D0004091EB025091EC0210161106E4F480E164
:10B9E00090E0821B930B489F9001499F300D589F18
:10B9F000300D1124B4E036952795BA95E1F72C1552
:10BA00003D0520F580917E0190917F01C816D906F1
:10BA1000F4F06C011CC0205F3F4F80917E0190913B
:10BA20007F01829F8001839F100D929F100D112432
:10BA30009801A4E036952795AA95E1F74C155D0588
:10BA400014F06A0104C0C216D30608F06901C601E9
:10BA5000AA2797FDA095BA2FFDE0880F991FAA1F6E
:10BA6000BB1FFA95D1F79501442737FD4095542F18
:10BA7000BC01CD010E94307820936C0330936D039C
:10BA800040936E0350936F03C0906C03D0906D038E
:10BA90008091990390919A039C01220F331F280FE4
:10BAA000391F2C0D3D1D37FF02C02D5F3F4FA901EF
:10BAB000559547955595479550939A03409399030B
:10BAC00080913806282F3327220F331F220F331F70
:10BAD000241735076CF480911E08282F3327220F76
:10BAE000331F220F331F205530404217530724F0D5
:10BAF00030939A03209399038091FA0780FF14C032
:10BB00008091990390919A0329813A818217930732
:10BB100024F030939A032093990340919903509114
:10BB20009A035A83498361C029813A812E193F09BA
:10BB300037FF02C02D5F3F4F3595279535952795E7
:10BB40006091990370919A03620F731F7A836983DE
:10BB50004CC080914006882301F56091BD02709130
:10BB6000BE0277FF02C06D5F7F4F75956795759533
:10BB7000679540911D0150911E0180910001282F71
:10BB80003327649FC001659F900D749F900D112411
:10BB9000B9010E94FB77CB0101C0992790938101E5
:10BBA000809380018091800190918101873491057B
:10BBB0001CF486E490E005C08639910534F086E9EE
:10BBC00090E0909381018093800189819A81909384
:10BBD0009A03809399038091A102806C8093A102C3
:10BBE0008091A0028D7F8093A0028091A10299276D
:10BBF0009C012270307081FF2BC180919B0390913A
:10BC00009C03A0919D03B0919E030097A105B105EF
:10BC100021F08091D7028130B1F4E981FA81CF011E
:10BC2000AA2797FDA095BA2F1EE0880F991FAA1F7B
:10BC3000BB1F1A95D1F780939B0390939C03A0930D
:10BC40009D03B0939E038091D702813019F482E066
:10BC50008093D702E980FA80C701AA2797FDA095B3
:10BC6000BA2F9501442737FD4095542FBC01CD01D3
:10BC70000E94BC77DC01CB0180936C0390936D0331
:10BC8000A0936E03B0936F03B7FF04C08150904E32
:10BC9000AF4FBF4F7C018D01ADE015950795F7942F
:10BCA000E794AA95D1F7E0926C03F0926D030093AC
:10BCB0006E0310936F036091A2027091A3022FE0B4
:10BCC000603A720750F580919B0390919C03A0917C
:10BCD0009D03B0919E039C01AD01FAE056954795F6
:10BCE00037952795FA95D1F7821B930BA40BB50BCB
:10BCF000A8019701E4E0220F331F441F551FEA9566
:10BD0000D1F7820F931FA41FB51F80939B039093BD
:10BD10009C03A0939D03B0939E0360547F4118F54C
:10BD200080919B0390919C03A0919D03B0919E03F1
:10BD30009C01AD016CE056954795379527956A951E
:10BD4000D1F7821B930BA40BB50BA8019701F2E06E
:10BD5000220F331F441F551FFA95D1F7820F931FEF
:10BD6000A41FB51F38C08091EB019091EC01809128
:10BD7000EB019091EC0197FF03C0909581959F4F47
:10BD80008436910584F58091D3029091D40220915C
:10BD9000CF023091D002821B930B81509F4F8F5F57
:10BDA000914008F580919B0390919C03A0919D0385
:10BDB000B0919E039C01AD01EEE0569547953795F5
:10BDC0002795EA95D1F7821B930BA40BB50B8E0D2B
:10BDD0009F1DA01FB11F80939B0390939C03A09372
:10BDE0009D03B0939E0380919B0390919C03A0912F
:10BDF0009D03B0919E037EE0B695A7959795879594
:10BE00007A95D1F79093BE028093BD0240913E0691
:10BE1000442399F055279C01BA010E94FB77C90180
:10BE2000861B970B9093EC028093EB02260F371F33
:10BE300030937F0120937E011FC01092EC0210927C
:10BE4000EB028FEF93E090937F0180937E0114C00B
:10BE50001092D70210929B0310929C0310929D03A4
:10BE600010929E033093BE022093BD0205C08091C4
:10BE7000A102806C8093A1028091AF0381FF37C043
:10BE800089819A8197FD03969595879595958795D4
:10BE900020919E0230919F022817390760F480910B
:10BEA000BD029091BE02892B31F0220F331F220F69
:10BEB000331F3A8329838091D3029091D402A091B9
:10BEC000D502B091D6028093CF029093D002A09376
:10BED000D102B093D20288E99AE39093DB01809378
:10BEE000DA0180E09EE090930801809307012091A1
:10BEF000E307822F9927880F991F880F991F88962B
:10BF000069817A818617970714F09A8389837091E3
:10BF10001E087D8B872F9927880F991F880F991FDF
:10BF200080559040A981BA818A179B0714F49A839F
:10BF3000898380912202882341F48091BC088F3F3D
:10BF400021F48091B3038823E9F08091A2029091BB
:10BF5000A3020297C097B0F4E981FA811E161F066A
:10BF60008CF481E090E09093A3028093A202E22EF1
:10BF7000FF24EE0CFF1CEE0CFF1C8701085D1F4F19
:10BF80001A83098329813A81309398052093970574
:10BF90008091640390916503A0916603B09167035B
:10BFA00012E0880F991FAA1FBB1F1A95D1F70091A5
:10BFB0001F0810912008081B190B213A31058CF03D
:10BFC000C90137FD019695958795801791070CF467
:10BFD0008C01909581959F4F081719076CF48C017F
:10BFE0000BC00135110514F000E510E03FEF003BF8
:10BFF000130714F400EB1FEF4D89242F3327220F72
:10C00000331F220F331FC90169817A81861B970B69
:10C01000801791070CF48C0189819A81821B930B04
:10C02000081719070CF48C018091DE079091DF0747
:10C030006091E9027091EA02861B970B9093ED07DD
:10C040008093EC07D090FC072091FB023091FC021A
:10C050004091FD025091FE02DD2041F0661A770A00
:10C06000C301AA2797FDA095BA2F04C0AA2797FD60
:10C07000A095BA2F280F391F4A1F5B1F2093FB0280
:10C080003093FC024093FD025093FE028091FB022C
:10C090009091FC02A091FD02B091FE0281509A4F56
:10C0A000A040B04064F080E09AEFA0E0B0E0809360
:10C0B000FB029093FC02A093FD02B093FE028091DC
:10C0C000FB029091FC02A091FD02B091FE02805013
:10C0D0009640AF4FBF4F64F480E096E0AFEFBFEF04
:10C0E0008093FB029093FC02A093FD02B093FE02AA
:10C0F000C0904D062091EC073091ED0778E0E72ED7
:10C10000EC1498F08C2D9927829FA001839F500DED
:10C11000929F500D1124CA0157FD07967C0163E0E0
:10C12000F594E7946A95E1F712C08C2D86959927CE
:10C13000829FB001839F700D929F700D1124CB01DF
:10C1400077FD03967C01F594E794F594E794A0902D
:10C150007B01B0907C019501442737FD4095542F19
:10C160008091FB029091FC02A091FD02B091FE0231
:10C17000BC01CD010E943078E20EF31E9090670161
:10C18000692D772788279927980117FF04C0222750
:10C190003327201B310B37FF02C02F5F3F4F3595F0
:10C1A0002795A981BA812A0F3B1F442737FD409567
:10C1B000542F0E94BC7797FF04C0615C7F4F8F4F64
:10C1C0009F4F26E095958795779567952A95D1F7A6
:10C1D0009B016E157F050CF47B01309521953F4F37
:10C1E000E216F3060CF479018091CE079091CF0707
:10C1F0006091E7027091E802861B970B9093CD0740
:10C200008093CC072091F7023091F8024091F90217
:10C210005091FA02DD2041F0461A570AC201AA27BE
:10C2200097FDA095BA2F04C0AA2797FDA095BA2F15
:10C23000280F391F4A1F5B1F2093F7023093F80223
:10C240004093F9025093FA028091F7029091F8021C
:10C25000A091F902B091FA0281509A4FA040B040EB
:10C2600064F080E09AEFA0E0B0E08093F702909352
:10C27000F802A093F902B093FA028091F70290912C
:10C28000F802A091F902B091FA0280509640AF4FA7
:10C29000BF4F64F480E096E0AFEFBFEF8093F7020A
:10C2A0009093F802A093F902B093FA022091CC0780
:10C2B0003091CD0748E04C1598F08C2D9927829F3E
:10C2C000B001839F700D929F700D1124CB0177FDFB
:10C2D00007966C01B3E0D594C794BA95E1F712C004
:10C2E000C6948C2D9927829FD001839FB00D929F79
:10C2F000B00D1124CD01B7FD03966C01D594C79400
:10C30000D594C7949501442737FD4095542F8091CB
:10C31000F7029091F802A091F902B091FA02BC01E3
:10C32000CD010E943078C20ED31E692D7727882751
:10C330009927980117FF04C022273327201B310BB0
:10C3400037FF02C02F5F3F4F35952795E981FA816E
:10C350002E0F3F1F442737FD4095542F0E94BC7776
:10C3600097FF04C0615C7F4F8F4F9F4FE6E095952C
:10C37000879577956795EA95D1F79B016C157D05B3
:10C380000CF46B01309521953F4FC216D3060CF487
:10C3900069018091E307282E332450908E066CEFBC
:10C3A000862E66E0962E53EBA52E56E0B52E4BE07A
:10C3B000442E3DEF632E37E0732ED5012C911216DB
:10C3C0000CF029C1203429F4E981FA81FF8BEE8B2E
:10C3D0001FC049815A81CA01AA2797FDA095BA2F8B
:10C3E000332727FD3095432F532FBC01CD010E94E9
:10C3F000BC7797FF04C0615C7F4F8F4F9F4F26E053
:10C4000095958795779567952A95D1F77F8B6E8B54
:10C41000F5012181203439F42E893F892E0D3F1DED
:10C420003F8B2E8B2AC0203C39F44E895F894E19F0
:10C430005F095F8B4E8B21C0C701AA2797FDA0958E
:10C44000BA2F332727FD3095432F532FBC01CD0141
:10C450000E94BC7797FF04C0615C7F4F8F4F9F4F56
:10C46000B6E09595879577956795BA95D1F7AE899A
:10C47000BF89A60FB71FBF8BAE8BF5012281203479
:10C4800039F42E893F892C0D3D1D3F8B2E8B2AC000
:10C49000203C39F44E895F894C195D095F8B4E8BC6
:10C4A00021C0C601AA2797FDA095BA2F332727FDE3
:10C4B0003095432F532FBC01CD010E94BC7797FFCD
:10C4C00004C0615C7F4F8F4F9F4FA6E09595879585
:10C4D00077956795AA95D1F7AE89BF89A60FB71F43
:10C4E000BF8BAE8BF5012381203439F42E893F892F
:10C4F000200F311F3F8B2E8B2AC0203C39F44E89F0
:10C500005F89401B510B5F8B4E8B21C0C801AA274E
:10C5100097FDA095BA2F332727FD3095432F532F32
:10C52000BC01CD010E94BC7797FF04C0615C7F4FC6
:10C530008F4F9F4FF6E09595879577956795FA957C
:10C54000D1F7AE89BF89A60FB71FBF8BAE8BF301A2
:10C55000808191812E893F898217930764F4B90104
:10C56000680F791F77FF02C06F5F7F4F75956795E2
:10C570007F8B6E8B1DC0552049F44E895F89440F17
:10C58000551F481B590B5F8B4E8B12C051E0551540
:10C5900078F4252D33276E897F89861B970BB90187
:10C5A0000E94FB77AE89BF89A60FB71FBF8BAE8BEA
:10C5B000C101880F991F880F991FEE89FF898E1777
:10C5C0009F0764F4FD898F2F9927880F991F880F83
:10C5D000991F2E893F892817390714F09F8B8E8B5E
:10C5E0008E899F8997FD0396959587959595879553
:10C5F000F4018183880F991F880F991F2E893F8925
:10C60000281B390BC901880F8283EE89FF89D3016A
:10C61000ED93FC9303C0F401118212824A9422E04C
:10C6200030E0620E731E44E050E0A40EB51E68E0D8
:10C6300070E0860E971E47FEC0CEE2E1C95E0C9404
:10C64000677884B1806A84B93D9A82E58CBD1DBC4F
:10C65000459A81E0809330088AEA8093410883E814
:10C66000809342088AE08093430810924508109214
:10C67000440810924708109246081092A908109298
:10C680006508089530913008332309F085C00DB452
:10C6900007FE82C084E08093D901459A2EB580912F
:10C6A000B60399278130910589F0823091051CF4F9
:10C6B000892B21F03EC00297B9F03BC0309364084B
:10C6C0002093B7032138A9F581E008C0253549F446
:10C6D0008091B703820F8093B70382E08093B60303
:10C6E00028C03093B60325C080916408E82FFF2747
:10C6F000EA57F74F20838F5F809364089091B703C8
:10C700008032A0F0291769F480E2A6E8B8E0E6E6F6
:10C71000F8E00D9001928A95E1F781E08093650839
:10C7200002C0309365081092B60303C0920F909335
:10C73000B70320914008223208F028C04598000035
:10C7400000000000000000000000000000000000E9
:10C7500000000000000000000000000000000000D9
:10C760000000000000000000000000000000E09158
:10C770003908F0913A08E20FF11D80818EBD809159
:10C7800062089081890F8093620803C081E08093E2
:10C7900030082F5F209340080895EF92FF920F9387
:10C7A0001F93809146069927880F991F880F991F1C
:10C7B0007C010027F7FC0095102F809133039091A6
:10C7C0003403A0913503B0913603BC01CD01A8011B
:10C7D00097010E9430783093450820934408809157
:10C7E0002B0390912C03A0912D03B0912E03BC013B
:10C7F000CD01A80197010E9430783093470820931B
:10C800004608209126083091270840912808509129
:10C810002908DA01C90163E0880F991FAA1FBB1F0D
:10C820006A95D1F7820F931FA41FB51F820F931F24
:10C83000A41FB51F20914201309143014091440152
:10C8400050914501BC01CD010E94307830934D08D4
:10C8500020934C0880914403909145032091F80166
:10C860003091F901821B930B9093530880935208E7
:10C87000E0913A03F0913B038091F3079091F40724
:10C88000BF010E94FB779B01220F331F220F331F32
:10C89000260F371F260F371F37FF02C02D5F3F4F70
:10C8A0003595279535952795309349082093480865
:10C8B0008091220890912308BF010E94FB779B0181
:10C8C000220F331F220F331F260F371F260F371F4C
:10C8D00037FF02C02D5F3F4F35952795359527953A
:10C8E00030934B0820934A0810923B0310923A036E
:10C8F0001092F4071092F307109223081092220866
:10C900008091430899278D30910509F48CC08E30B1
:10C9100091055CF48B30910509F4B4C08C3091051D
:10C920000CF035C10A9761F0E7C18F30910509F429
:10C93000B3C18F3091050CF480C14097A9F1DCC1DF
:10C940008091B602809356088091B5028093570873
:10C950008091B402809358088091B3028093590863
:10C960008091B20280935A088091B10280935B0853
:10C970008091B00280935C088091AF0280935D0843
:10C980008091A10280935E088091A102837F8093B1
:10C99000A1020E94C92B80935F0880918F0680932B
:10C9A00060088091A002A6C18091B6089091B70856
:10C9B00090935708809356088091BA089091BB08CD
:10C9C000909359088093580880911D0190911E0101
:10C9D00080935A088091000180935B088091410107
:10C9E00080935C089091B80390935D08E92FFF272E
:10C9F000A3E0EE0FFF1FAA95E1F7E450F94F8681FF
:10CA000080935E08838180935F08878180936008AC
:10CA1000858180936108892F8F5F6CE00E94DB77AE
:10CA20009093B80369C180917A06809356088091EB
:10CA30007B068093570880917C06809358088091EC
:10CA40007D068093590880917E0680935A088091D4
:10CA5000820680935B088091830680935C088091B6
:10CA6000840680935D088091870680935E0880919C
:10CA7000850680935F088091860680936008809188
:10CA8000880638C1F89480912D06E82FFF27EE0F15
:10CA9000FF1FE35AF84F0190F081E02DE038F105D7
:10CAA0001CF0EFE7F0E006C02FEFE138F20714F4D6
:10CAB000E1E8FFEFE093560880912E06E82FFF276C
:10CAC000EE0FFF1FE35AF84F0190F081E02DE038A0
:10CAD000F1051CF0EFE7F0E006C06FEFE138F60774
:10CAE00014F4E1E8FFEFE093570880912C06E82F5B
:10CAF000FF27EE0FFF1FE35AF84F0190F081E02D62
:10CB0000E038F1051CF0EFE7F0E006C08FEFE13808
:10CB1000F80714F4E1E8FFEFE093580880912B0642
:10CB2000E82FFF27EE0FFF1FE35AF84F0190F08127
:10CB3000E02DE038F1051CF0EFE7F0E006C02FEF44
:10CB4000E138F20714F4E1E8FFEF7894E093590834
:10CB50008091DA0280935A088091DB0280935B080F
:10CB60008091DC0280935C088091DD0280935D08F7
:10CB70008091DE0280935E088091DF0280935F08DF
:10CB80008091E002809360088091E102B3C08091BF
:10CB90001804863018F01092180485E08093560827
:10CBA00080918906809357088091D3029091D40296
:10CBB000A091D502B091D602BC01CD0125E030E0B4
:10CBC00040E050E00E943078309359082093580894
:10CBD0008091CF029091D002A091D102B091D20267
:10CBE000BC01CD0125E030E040E050E00E9430780B
:10CBF00030935B0820935A0880917F0680935C08ED
:10CC00008091800680935D088091810680935E0804
:10CC10008091D90280935F0880915D0790915E07B3
:10CC200080936008809197059091980597FD0396F1
:10CC300095958795959587955DC01092560888E5DE
:10CC40008093570884E0809358088FE180935908B7
:10CC50008091010180935A088091FD0380935B08C5
:10CC60008091FE0380935C081092FD038071809395
:10CC7000FE038091FF0380935D08809116088093E6
:10CC80005E088091FA0780935F0880918B068093FD
:10CC90006008809198062EC080915F0680935608A8
:10CCA000809196068093570880916D018093580873
:10CCB00080915806809359088091590680935A08AC
:10CCC00080915A0680935B0880916C0180935C0888
:10CCD00080915C0680935D0880915D0680935E087C
:10CCE00080915E0680935F088091BC088093600805
:10CCF0008091C1058093610880916508882309F4BB
:10CD00004AC18AEF80939B0181E080938D0140911D
:10CD1000670850916808CA0181509E4F8F5F934009
:10CD2000B0F42091690830916A08C90181509E4F82
:10CD30008F5F934060F48091370685FF08C0509361
:10CD4000A5034093A4033093A3032093A2038091EF
:10CD50006D0890916E0821E08936920724F4909333
:10CD60008F0180938E01209177083091780880910F
:10CD7000DA019091DB018217930740F48091AE01B4
:10CD8000882321F43093DB012093DA018091660837
:10CD900099278836910509F468C08936910524F4ED
:10CDA0008736910551F0FFC08936910509F496C088
:10CDB0008B36910509F4E2C0F6C080917908809322
:10CDC000A60880917A088093A80880917B088093B8
:10CDD000A70880917C0880938C0180917D088093C6
:10CDE000AA0880917E0880939C0180917F0880939F
:10CDF000B503809180088093A1038091AE028823BF
:10CE0000F9F0209181083091820837FD19C03093E4
:10CE1000F2022093F10290916106992389F08FE04C
:10CE2000989FC0011124281B390BC90188599E4FB6
:10CE300068E671E00E94FB779093F2028093F10222
:10CE40002091AC033091AD038091830890918408C8
:10CE5000280F391F37FF02C02F5F3F4F35952795A9
:10CE60003093AD032093AC039EC0809179088093EA
:10CE70003B0880917A0880933C0880917B088093DE
:10CE80003D0880917C0880933E0880917D088093C6
:10CE90003F088091870590917E08892B80938705B4
:10CEA00090918805937080917F088C70982B909357
:10CEB0008805809180088093B303809181088093D6
:10CEC0009101809182088093A908809183088093C2
:10CED000AF03809184088093AE0365C08091790888
:10CEE0008093310880917A088093320880917B0882
:10CEF0008093330880917C088093340880917D086A
:10CF000090917E08909336088093350880917F0831
:10CF10009091800890933808809337088091810819
:10CF2000992787FD90959093900780938F07809124
:10CF300082088093C80280918308909184089C01A4
:10CF4000442737FD4095542FDA01C90163E0880F6B
:10CF5000991FAA1FBB1F6A95D1F7820F931FA41FA9
:10CF6000B51F820F931FA41FB51F8093C902909312
:10CF7000CA02A093CB02B093CC0215C0809179086D
:10CF80008093B20380917A088093B10380917B08EB
:10CF90008093B00308C01092A5031092A4031092CE
:10CFA000A3031092A2031F910F91FF90EF90089599
:10CFB00080913008882309F43BC0459881E498E0CB
:10CFC00090933A08809339089091B403E92FFF2792
:10CFD000EE56FE4F9F5F9093B40380818093430889
:10CFE000993010F01092B403109230080E94CD6373
:10CFF00081E0809340080000000000000000000075
:10D000000000000000000000000000000000000020
:10D010000000000000000000000000000000000010
:10D0200000000000000080914108809362088EBDDE
:10D03000089587B18C6087B9429843981092BA03DB
:10D0400080E880939E011092B90380939D0108951A
:10D050008091BF0381508093BF038F3F09F019C1B6
:10D0600089E08093BF038091A1029927807390701B
:10D07000892B21F48091FE0380FF1DC080917806EA
:10D08000882351F08091C203882319F484E08093AF
:10D09000BA0381E08093C203809179068823B9F0B6
:10D0A0008091C303882319F484E08093B90381E05D
:10D0B0008093C3030CC01092C2031092C3038091EB
:10D0C00074068093C003809176068093C10380919B
:10D0D000C203882309F045C080919506282F332785
:10D0E00024FF07C08091D802882319F425FD52C07F
:10D0F00053C090917506983F48F08091F5078D3D9B
:10D1000028F08091C00388236CF00AC0983F78F023
:10D110008091F507853059F48091C00387FF02C0E4
:10D12000429801C0429A81E080939E0136C080916E
:10D13000BA0381508093BA038F3F79F58091F50748
:10D1400086958093BA0380919E01813011F480E826
:10D1500001C0869580939E0180919E019091C003AD
:10D1600017C08091BA0381508093BA038F3FA9F40E
:10D1700089E08093BA0380919E01813011F480E8A8
:10D1800001C0869580939E0180919E0190917806C2
:10D19000892311F0429A01C042988091C3038823E9
:10D1A00009F043C09091950697FF07C08091D8027F
:10D1B000882319F496FD52C053C090917706983F8A
:10D1C00048F080911D088D3D28F08091C10388238F
:10D1D0006CF00AC0983F78F080911D08853059F4B2
:10D1E0008091C10387FF02C0439801C0439A81E048
:10D1F00080939D0136C08091B90381508093B9031B
:10D200008F3F79F580911D0886958093B9038091B1
:10D210009D01813011F480E801C0869580939D01C5
:10D2200080919D019091C10317C08091B9038150F5
:10D230008093B9038F3FA9F489E08093B90380916B
:10D240009D01813011F480E801C0869580939D0195
:10D2500080919D0190917906892311F0439A01C034
:10D260004398429B04C08091A002886003C08091D3
:10D27000A002877F8093A002439B06C08091A002FA
:10D2800080618093A00208958091A0028F7E809398
:10D29000A00208954FB724E130E0F8948091C900CE
:10D2A0008F778093C9008091C9008F7B8093C900DC
:10D2B0008091C9008F7D8093C9005A9A52985B9AD9
:10D2C000539A832F99278093CD002093CC0080918F
:10D2D000C80082608093C80080E18093C90080917B
:10D2E000CA008F778093CA008091CA008F7B809399
:10D2F000CA008091CA008F7D8093CA008091CA00C5
:10D300008F7E8093CA008091CA00877F8093CA0075
:10D310008091C9008B7F8093C9008091CA0084608E
:10D320008093CA008091CA0082608093CA00809175
:10D33000C80087FF03C08091CE00F9CF8091C9005B
:10D3400080688093C9004FBF0895A0E0B0E0EBEA89
:10D35000F9E60C945578482F00E010E080919F0189
:10D36000813061F410929F0184E48093C60310928F
:10D37000C8031092C7031092C90333C28091C60339
:10D38000882319F421E030E001C098019091C7038F
:10D39000992371F4232B11F081E010C084E4809371
:10D3A000C6039093C8039093C7039093C90302C226
:10D3B000913069F4232B09F0F3C182E08093C70315
:10D3C0008091C8038F5F8093C80383E0F1C19230DE
:10D3D000D1F4232B09F0E4C183E08093C60340938A
:10D3E000C9039091C803923039F41092CA0347FFE1
:10D3F00003C081E08093CA0383E08093C7039F5FEB
:10D400009093C803D7C1933009F0CAC1232B09F008
:10D41000C7C19093C60382E08093C7038091C8037D
:10D420008F5F8093C8032091C903822F9927782F9B
:10D430006627842F9927682B792B8091510681309C
:10D4400051F47370CB018050924063E070E00E9411
:10D45000FB77EB0119C0823069F47770CB01805003
:10D46000944066E070E00E94FB77EB0126952695DC
:10D4700026950CC0EB01D370C856D140CE01D7FD24
:10D480000196EC01D595C79526952695022F112773
:10D490000F7010700F5F1F4F0D30110508F079C12C
:10D4A0000230110519F404E010E005C00430110544
:10D4B00011F402E010E06801C00ED11EF601E35A3B
:10D4C000F84F808191819E01281B390BC90137FFDC
:10D4D00003C0909581959F4F069704F5E0919206C1
:10D4E000EE2351F0FF27EE0FFF1FE35AF84F808124
:10D4F00091818436910594F48091D902883C30F46E
:10D500008091D902865F8093D90208C088EC80930D
:10D51000D90280916F008F7D80936F00F601E35AEE
:10D52000F84F808191819C01220F331F280F391FF2
:10D530002C0F3D1F37FF02C02D5F3F4F7901F5943F
:10D54000E794F594E794CE0101968E159F0524F497
:10D550000894E108F10808C0CE010197E816F90621
:10D560001CF40894E11CF11C0630110509F0D1C02F
:10D57000C536D1050CF4A8C09091C503E92FFF274B
:10D58000E555F74FE081ED3729F48091C40380958C
:10D590008093C403963061F48091C403882311F012
:10D5A000E338B9F0882309F08BC0ED3791F088C0DB
:10D5B000993009F085C08091C403882329F48091B3
:10D5C000B408833831F07CC08091B4088D3709F0FD
:10D5D00077C08091AC088D3739F48091AD088338DD
:10D5E000B1F483E89FEF0FC0833889F48091AD08D0
:10D5F000833829F4109268071092670708C08D37A6
:10D6000031F48DE790E090936807809367078091ED
:10D61000AE08992787FD909590936A0780936907D4
:10D620008091AF08992787FD909590937407809318
:10D6300073078091B008992787FD9095909376079E
:10D64000809375078091C5038930D1F58091B20828
:10D650008D3749F480916D0790916E0705969093F0
:10D660006E0780936D078091B3088D3749F48091E0
:10D670006D0790916E07059790936E0780936D07E5
:10D6800080916D0790916E0783589F4F1CF483E83B
:10D690009FEF09C080916D0790916E078E379105BD
:10D6A00034F08DE790E090936E0780936D07809142
:10D6B000B108992787FD9095909372078093710721
:10D6C0001092C5031092C403CA30D1055CF4809156
:10D6D000C5038F5F8093C503E82FFF27E555F74FFC
:10D6E00083E880838091C5038A3011F41092C503CA
:10D6F0008FEFCC39D8076CF48091C503E82FFF2752
:10D70000E555F74F8DE780838091C4038095809322
:10D71000C4038091D902843BD0F0F601E35AF84F5C
:10D7200080819181F701E81BF90BCF0163E070E084
:10D730000E94FB77CB01880F991F860F971F21E965
:10D7400037E0C20ED31EF6019183808307C021E922
:10D7500037E0C20ED31EF60111821082053011058A
:10D7600040F4000F111F035A184FF801F182E082B4
:10D7700021C00530110529F4D0936C07C0936B07C5
:10D7800019C007301105B1F4D0937007C0936F072B
:10D7900011C00231110570F081E080939F010AC031
:10D7A00081E080939F011092C8031092CA0384E421
:10D7B0008093C6038091C803803198F08091CA039A
:10D7C000882331F480919F01882311F480934001D4
:10D7D0001092C8031092CA031092C70384E4809386
:10D7E000C603E8E0CDB7DEB70C947178CF93FC01A7
:10D7F00097FF05C0CFEFF095E195FF4F01C0C1E065
:10D8000028E631E0CF01B9010E94FB77FC018B359E
:10D81000910554F08B5590408A35910538F484EB8E
:10D8200090E08E1B9F0BFC0141E00DC0CF01855B9A
:10D8300090408A35910518F4E45BF04003C02E1B3C
:10D840003F0BF9014FEFEE0FFF1FEC54F74F2591FF
:10D8500034918C2F992787FD9095289FB001299F9F
:10D86000700D389F700D1124842F992787FD909596
:10D87000689FA001699F500D789F500D1124CA0127
:10D88000CF9108952AE530E0281B390BC9010E9489
:10D89000F66B08950895089508950895089580E019
:10D8A00090E008951092B7081092B6081092BB0845
:10D8B0001092BA081092B9081092B8081092BC08D9
:10D8C0008AE090E00E9496159093CC038093CB035E
:10D8D0000895CF93DF938091CB039091CC030E9466
:10D8E0009F15882309F4AFC08091CB039091CC039E
:10D8F0000A969093CC038093CB03E0E0F0E09F0185
:10D9000090E05FEFACEFB6E04BE0ED018B8187FF7D
:10D910000BC09F5F8D81E80FF11D8981280F311D9C
:10D920008E81851708F4582F4150189647FFEDCF88
:10D930005093BC08232B41F52091D1033091D203A1
:10D940004091D3035091D403BB27A52F942F832F4D
:10D950009093D0038093CF03AA27BB27281B390BB2
:10D960004A0B5B0BCF01AA27BB27280F391F4A1F81
:10D970005B1F2093D1033093D2034093D303509382
:10D98000D403E5E0F0E013C02091CF033091D00341
:10D990002E173F0718F4E21BF30B02C0E0E0F0E0A3
:10D9A000892F9927880F991FE80FF91F3596F09353
:10D9B000B708E093B608EF3FF10578F480911D01B8
:10D9C00090911E018E9F90018F9F300D9E9F300D74
:10D9D0001124C90164E670E013C0CF0196958795C4
:10D9E0009695879520911D0130911E01289FA001D9
:10D9F000299F500D389F500D1124CA0169E170E034
:10DA00000E94E7777093B9086093B8082091CD031E
:10DA10003091CE032E0F3F1F3093CE032093CD03C2
:10DA20005EE02131350778F08091BA089091BB080B
:10DA300001969093BB088093BA0820513E403093E2
:10DA4000CE032093CD03DF91CF91089508950895DB
:10DA5000002422273327442751E0BB27EE27FF2746
:10DA6000A0E1660F771F881F991F001C221F331F1C
:10DA7000441F660F771F881F991F001C221F331F2A
:10DA8000441F2AF4050E2B1F3E1F4F1F04C0051A0A
:10DA90002B0B3E0B4F0B550FBB1FEE1F587F5560D6
:10DAA00047FD5250AA95E9F6E695B7955795E69544
:10DAB000B7955795852F9B2F08952227332741E04F
:10DAC000552768E0880F991F221F331F880F991F61
:10DAD000221F331F1AF4240F351F02C0241B350BDD
:10DAE000440F551F487F456037FD42506A9551F7F6
:10DAF0005695479556954795842F0895AA2797FFE1
:10DB000004C0809590958A1F9A1F77FF04C0609586
:10DB100070956A1F7A1F669F9001779FA001679F8B
:10DB2000300D411D5A1F300D411D5A1F889FF001B5
:10DB3000999F2E0F3F1F401D511D899F300D411D84
:10DB40005A1F300D411D5A1FCA01B901112480CF3F
:10DB50004FB720E430E0F8948091C9008F7780932C
:10DB6000C9008091C9008F7B8093C9008091C90052
:10DB70008F7D8093C9005A9A52985B9A539A832F4B
:10DB800099278093CD002093CC008091C8008260BB
:10DB90008093C80088E18093C9008091CA008F7784
:10DBA0008093CA008091CA008F7B8093CA008091C5
:10DBB000CA008F7D8093CA008091CA008F7E8093B7
:10DBC000CA008091CA00877F8093CA008091C900F3
:10DBD0008B7F8093C9008091CA0084608093CA00C3
:10DBE0008091CA0082608093CA008091C80087FF3C
:10DBF00003C08091CE00F9CF8091C90080688093E6
:10DC0000C9004FBF08950F931F93CF93DF93482F01
:10DC10004F5F893108F08BC080915C07841720F436
:10DC20004F5F40935C074150CB0183539B4268E1B7
:10DC300070E00E94FB77A42FBB27FD01EA0FFB1FBA
:10DC4000E35AF84F808191819B01281B390BC90150
:10DC500037FF03C0909581959F4F069794F480916C
:10DC6000D902883C30F48091D902865F8093D90232
:10DC700008C088EC8093D90280916F008F7D8093DB
:10DC80006F00FD01EA0FFB1FE35AF84F808191817D
:10DC90009C01220F331F280F391F260F371F37FF14
:10DCA00002C02D5F3F4FE901D595C795D595C79522
:10DCB000CB0101968C179D0714F4219706C0615083
:10DCC0007040C617D7070CF421968091D902843B87
:10DCD000D8F08D010A0F1B1FF801E35AF84F80811D
:10DCE0009181FE01E81BF90BCF0163E070E00E9417
:10DCF000FB77CB01880F991F860F971F0F56184F80
:10DD0000F8019183808307C0AA0FBB1FAF56B84F9D
:10DD100011961C921E92E42FFF27EE0FFF1FE35A6D
:10DD2000F84FD183C083443011F410924001DF9149
:10DD3000CF911F910F910895CF93DF932091BD084C
:10DD4000822F9927807F9070409709F06CC02F3107
:10DD500009F046C08091BE088093D9032091C00885
:10DD60002093DB038091C1088093DA03822F9927E7
:10DD700090935E0780935D07222309F054C0809141
:10DD80002B06282F3327220F331FF901EF56F84FA8
:10DD90001182108280912C06A82FBB27AA0FBB1FCF
:10DDA000FD01EF56F84F1182108280912E06E82F68
:10DDB000FF27EE0FFF1FCF018F56984FEC011982FE
:10DDC0001882235A384FE90119821882A35AB84F92
:10DDD00011961C921E92E35AF84F1182108223C0B2
:10DDE000C22FCF70CA30F8F48091BE088093E70844
:10DDF0008091BF088093E6088091C0088093E9086D
:10DE00008091C1088093E8086091E6087091E70866
:10DE10008C2F0E94036E6091E8087091E9088C2FA6
:10DE20008F5F0E94036EDF91CF910895CF93C82F2B
:10DE30008F3F49F48091DC038F3F29F41092DE0379
:10DE40001092DD0332C02091DE03222339F4CF315A
:10DE500011F485E001C084E08093DF038091DF034B
:10DE60009091DD038217A0F4892F80958093DD03C4
:10DE70008F3F19F48EEF8093DD038091DD03C81787
:10DE800011F40E949C6E1092DE031092DD030BC011
:10DE9000E22FFF27E354F74FC0832F5F2093DE0369
:10DEA0009C0F9093DD03C093DC03CF910895909174
:10DEB000D803933240F4E92FFF27ED53F74F8083C7
:10DEC0009F5F9093D8030895833218F48D5F8093F9
:10DED000D803089590E2E6ECF8E08FE19193815049
:10DEE00087FFFCCF0895CF93CFB723E031E0F894BC
:10DEF0008091C9008F778093C9008091C9008F7B82
:10DF00008093C9008091C9008F7D8093C9005A9A7F
:10DF100052985B9A539A832F99278093CD00209330
:10DF2000CC008091C80082608093C80088E1809313
:10DF3000C9008091CA008F778093CA008091CA007F
:10DF40008F7B8093CA008091CA0080628093CA0050
:10DF50008091CA0080618093CA008091CA00886065
:10DF60008093CA008091C90084608093C900809129
:10DF7000CA0084608093CA008091CA008260809346
:10DF8000CA008091C80087FF03C08091CE00F9CFFE
:10DF90008091C90080688093C9008091C900806425
:10DFA0008093C9000E946A6FCFBFCF910895282F38
:10DFB00099278F709070892B31F420958091D70329
:10DFC000822B8093D70308958091A201882309F4BE
:10DFD0004BC08091A10285FD04C08091A6018823D9
:10DFE00081F082E98093C30883E28093C408809122
:10DFF000A601882309F485E58093C5081092A6013F
:10E0000002C08093C3088091A3018F3071F4809186
:10E01000D7030E944F6C882341F081E98093C308A5
:10E020008093C40881E38093C5081092A201809177
:10E03000C80085FFFCCF8091C9008F7E8093C90006
:10E040008091C9008E7F8093C9008091C308882386
:10E0500011F48EEF01C08EE78093CE008091D7033C
:10E060008093A3011092D70308951F920F920FB6C9
:10E070000F9211248F939F93EF93FF939091A2019E
:10E08000992309F040C08091E003882361F48091D6
:10E09000C308882311F483E003C0813999F481E037
:10E0A0008093E0030FC0833099F48091C3088823E4
:10E0B00049F09093C3088091C9008E7F8093C90076
:10E0C0008EEF1EC08091C90081608093C9000EC090
:10E0D000833261F48091C9008E7F8093C9008FEFF5
:10E0E0008093CE0081E08093A20114C08091E00370
:10E0F000E82FFF27ED53F74F8F5F8093E003808178
:10E100008093CE0007C01092E0038091C900806127
:10E110008093C900FF91EF919F918F910F900FBE57
:10E120000F901F901895EF92FF920F931F93CF932C
:10E13000DF937C018B01EA01452B39F0F8018191D5
:10E140008F01F70109952197C9F7E6E0CDB7DEB752
:10E150000C947378EF92FF920F931F93CF93DF93FA
:10E160007C018B01EA01452B41F0F8010F5F1F4F45
:10E170008491F70109952197C1F7E6E0CDB7DEB7A5
:10E180000C9473780F931F93CF938C01C62F1616A0
:10E1900034F480E2F8010995C1501C16D4F3CF91F4
:10E1A0001F910F9108950F931F93CF938C01C62F4A
:10E1B000161634F480E3F8010995C1501C16D4F307
:10E1C000CF911F910F910895A5E3B0E0EAEEF0E73B
:10E1D0000C944B782E96EEADFFAD2E9788249924A3
:10E1E00054018091D603882321F42C961FAE1EAED5
:10E1F0002C975EE4452E512C4C0E5D1E6F01B6012E
:10E2000005C0153239F00894C11CD11CF6011491D7
:10E210001123B9F7A601461B570B31F02C968EAD92
:10E220009FAD2C970E94AA70112309F46AC208942A
:10E23000C11CD11CFF24FDA6FCA64FEFE42EF9A6BD
:10E24000F6010894C11CD11C1491153721F0812FBF
:10E2500080628837B1F4F0FE0AC0F20124E030E0B9
:10E26000420E531E80809180A280B3800AC0F201CA
:10E2700042E050E0440E551E808191814C01AA2459
:10E28000BB24103221F489A58823D1F61DC0133296
:10E2900019F458E0F52AD4CF1A3211F01D3291F456
:10E2A0001A3259F4F20182E090E0480E591EE081E2
:10E2B000ECA7EE232CF6E195ECA790E1F92AAFED5F
:10E2C000FA22BECF1B3211F419A7BACF1E32C1F504
:10E2D000F6010894C11CD11C14911A3279F4F20190
:10E2E00022E030E0420E531E408151813FEF4F3F0C
:10E2F000530714F44FEF5FEFE42EA2CF40E050E05D
:10E30000812F80538A30A0F4CA0133E0880F991F0F
:10E310003A95E1F7840F951F480F591F410F511D82
:10E3200040535040F6010894C11CD11C1491E8CF11
:10E330008FEF4F3F580714F44FEF5FEFE42E85CF78
:10E34000103329F4F4FC7CCF90E2F92A79CF812FA5
:10E3500081538930D8F440E050E0CA0123E0880FAF
:10E36000991F2A95E1F7840F951F480F591F410FF8
:10E37000511D40535040F6010894C11CD11C14910A
:10E38000812F80538A3048F34CA75FCF183619F499
:10E39000A4E0FA2A55CF1C3619F4B1E0FB2A50CF7D
:10E3A000133661F43E010894611C711CF20122E0F5
:10E3B00030E0420E531E808189833CC1143421F029
:10E3C000143611F0193651F5143411F431E0F32AF2
:10E3D000F0FE0AC0F20144E050E0440E551E808079
:10E3E0009180A280B3800CC0F20182E090E0480EE0
:10E3F000591E808191814C01AA2497FCA094BA2CCB
:10E40000B7FE0AC0B094A09490948094811C911C93
:10E41000A11CB11C8DE289A70AE06FC01F3411F066
:10E420001F3631F41F3411F491E0F92A08E064C07A
:10E43000103779F4F201A2E0B0E04A0E5B1E808151
:10E4400091814C01AA24BB2400E1B0E4FB2A18E727
:10E4500053C01337C1F5F20122E030E0420E531EE3
:10E46000608071806114710489F43E010894611C1C
:10E47000711C88E289838EE6F301818385E78B83B3
:10E480008CE68C838D8389E28E831F82E7FC13C028
:10E490008E2D992787FD9095AC0160E070E0C30157
:10E4A0000E941876009729F0382E3618E3140CF0E5
:10E4B000C3C03E2CC1C0F30101900020E9F73197A1
:10E4C0003E2E3618B9C0153511F0153731F4153513
:10E4D00011F4F1E0FF2A0AE00FC0183519F01837DF
:10E4E00009F0A0C000E1F3FE07C081149104A1046B
:10E4F000B10411F020E4F22A19A6EDA6E7FC02C04F
:10E500003FEDF32289E2682E712C6C0E7D1E811482
:10E510009104A104B10421F44DA5442309F47BC066
:10E52000802F9927AA27BB278EA79FA7A8ABB9AB97
:10E53000202E332490E0891690E0990691E0A906F8
:10E5400090E0B90648F0C501B4012EA53FA548A941
:10E5500059A90E940E7817C0AFEF8A169104A10442
:10E56000B10449F040F0C401B1010E94E7779B017A
:10E570004427552708C0882D602F0E94DB77282F5D
:10E580003327442755272AAB3BAB4CAB5DAB0A3056
:10E5900059F48AA9880F880F880F9AA9990F890FB3
:10E5A000382D381B832F10C0003139F48AA9829589
:10E5B000807F482D481B842F07C08AA9880F880FA9
:10E5C000880F582D581B852F90E02EA53FA548A9F0
:10E5D00059A982169306A406B50608F091E08AA808
:10E5E0009BA8ACA8BDA88A3010F4805D04C0895AED
:10E5F000183509F48F7DD3018E933D01992309F0DD
:10E6000099CF083041F4F3FE06C0803321F080E357
:10E61000FD0182933F01CE010196382E3618F8E2B3
:10E620003F0E0BC0112309F46CC03E010894611C1D
:10E63000711C1983B1E03B2E19A6032D2DA42318BC
:10E6400027FC222489A5882311F00F5F02C0F6FC65
:10E650000E5F020DEF2CFF24C70180739070892B91
:10E6600049F48CA5801B682F2C968EAD9FAD2C97FE
:10E670000E94C27089A5882331F041E050E0BE01BC
:10E68000675D7F4F0AC0E6FE0EC080E38AA71BA726
:10E6900042E050E0BE01665D7F4F2C968EAD9FAD8F
:10E6A0002C970E949370C70180739070809749F4F3
:10E6B0008CA5801B682F2C968EAD9FAD2C970E9449
:10E6C000D370622D2C968EAD9FAD2C970E94D37087
:10E6D000832D992787FD9095AC01B3012C968EADC3
:10E6E0009FAD2C970E949370E4FE89CD2CA5201B32
:10E6F0002CA7622F2C968EAD9FAD2C970E94C270D6
:10E700007ECDE2E1CB5C0C9467782FB740E0F894C3
:10E71000E0E0F0E081E2809357009491E2E0F0E0E5
:10E72000809357003491E4E0F0E0809357008491A7
:10E730002FBF9E3199F4363941F4893011F441E00C
:10E740000DC08A3059F442E009C0373939F48630B7
:10E7500011F443E003C0853009F444E0842F992785
:10E7600008959FB7F8948091C900877F8093C9006E
:10E770008091C9008F7E8093C9008091C9008F77F6
:10E780008093C9008091C9008F7B8093C9008091DC
:10E79000C9008F7D8093C90052985A9A53985B9A0A
:10E7A0009FBF08951F93CF93DF93182F8091D603B7
:10E7B000882309F4A5C08091A101181709F4A0C00D
:10E7C0008091D503882321F40E9485738093D5031B
:10E7D00082ED91E090933F0180933E0189E09AE0C1
:10E7E0009F938F93C7E8D1E1DF93CF93E091E40348
:10E7F000F091E50309950F900F900F900F90812FE6
:10E80000992784309105F1F0853091051CF4892B0E
:10E8100051F00CC086309105D9F086309105ACF0EE
:10E82000089741F12AC085E09AE002C08CEF99E098
:10E830009F938F93DF93CF93E091E403F091E503EF
:10E84000099527C087EF99E0F3CF8FEE99E0F0CFDD
:10E8500087EE99E09F938F93DF93CF93E091E4034A
:10E86000F091E503099588ED91E090933F01809345
:10E870003E010FC082EE99E0DBCF86E19AE09F93E4
:10E880008F93DF93CF93E091E403F091E503099533
:10E8900010E00F900F900F900F908091D50384306F
:10E8A00011F08230C1F40E94B173812F8150833006
:10E8B00018F40E944A6922C0143019F40E94736F40
:10E8C0001DC0153019F40E94A86D18C01830B1F49D
:10E8D0000E94266D13C0112389F08CE29AE09F9369
:10E8E0008F9387E891E19F938F93E091E403F091F8
:10E8F000E50309950F900F900F900F901093A101D1
:10E90000DF91CF911F9108950F931F9381E0809322
:10E91000D6034091A001E2E9F9E020E030E05FE4B5
:10E92000849199272F5F3F4F829FB001839F700D85
:10E93000929F700D112446275150319657FFF0CF0A
:10E940004093A001EAE6F9E020E030E057E284914C
:10E9500099272F5F3F4F829FB001839F700D929F39
:10E96000700D112446275150319657FFF0CF409338
:10E97000A0018091D503882321F40E9485738093A0
:10E98000D5038091A001833459F088E190E029E219
:10E990000FB6F894A895809360000FBE2093600096
:10E9A00084EE90E79093E5038093E4030E9486054C
:10E9B00085E690E09F938F9388E590E09F938F93F7
:10E9C0001F921F92809101016AE00E94DB77892FDC
:10E9D00099279F938F93809101010E94DB7799275C
:10E9E0009F938F9387E49AE09F938F9307E811E1B9
:10E9F0001F930F93E091E403F091E503099582E9F9
:10EA000099E09F938F931F930F93E091E403F0910C
:10EA1000E50309958AE699E09F938F931F930F93DF
:10EA2000E091E403F091E50309950E94860583ECEB
:10EA30008093810080916F00806280936F008DB71A
:10EA40009EB746968DBF1F910F91089580919006B5
:10EA50008D3338F08091310887FD03C08CE38093BB
:10EA6000900680914006882331F08055853618F055
:10EA70008FE7809340060895CF938091D603882333
:10EA800009F472C08091E10381508093E1038823EF
:10EA900009F053C089E18093E103809190068E33A1
:10EAA00038F08091310887FD03C08DE38093900694
:10EAB0008091D902823820F58091A2029091A30220
:10EAC000885E934020F08091BC08843620F4109238
:10EAD000E3031092E2038091E2039091E303009735
:10EAE00039F101979093E3038093E203419728F172
:10EAF0008091310884FF21C08091A00284601BC0F6
:10EB00008091D902853BC8F09091900684E1989F4E
:10EB1000C001112440962091E2033091E3032817AD
:10EB2000390730F42F5F3F4F3093E3032093E20324
:10EB30008091A0028B7F8093A002C091A401CC237E
:10EB400021F0C150C093A4010FC086E98093A401B5
:10EB50008091A101843011F40E94E46F8091A001A2
:10EB6000833411F0C093D603CF9108951F920F9272
:10EB70000FB60F9211242F933F934F935F936F9390
:10EB80007F938F939F93AF93BF93EF93FF932091C6
:10EB9000CE008091B0018823B1F02093C60080910F
:10EBA000B001823059F52F3F49F58FEF94E3ACE087
:10EBB000B0E0C297A109B109B7FFFBCF809127044C
:10EBC0008093CE001BC09091A101892F815083308A
:10EBD00020F4822F0E94A56911C0943021F4822F65
:10EBE0000E94D76F0BC0953021F4822F0E94166FC0
:10EBF00005C0983019F4822F0E94276DFF91EF9184
:10EC0000BF91AF919F918F917F916F915F914F9144
:10EC10003F912F910F900FBE0F901F901895FB0101
:10EC2000DC0102C005900D9241505040D8F7089584
:10EC3000FC014150504030F001900616D1F7319759
:10EC4000CF010895882799270895A0E0B0E0EBE26E
:10EC5000F6E70C9453786C017B01EA015901219786
:10EC60008FEFCF3FD80789F086010894C11CD11CD3
:10EC7000C7010894E11CF11CF5010995F801808396
:10EC80002197FFEFCF3FDF0779F7EAE0CDB7DEB797
:10EC90000C946F78CF92DF92EF92FF920F931F93B5
:10ECA0007C016B01FB010995082FC7010196F60154
:10ECB0000995182FC8011F910F91FF90EF90DF90D9
:10ECC000CF900895A0E0B0E0E8E6F6E70C94557820
:10ECD0008C017B01EA01690121978FEFCF3FD807B3
:10ECE00071F0F70121917F01C8010F5F1F4F622F63
:10ECF000F60109952197FFEFCF3FDF0791F7E8E095
:10ED0000CDB7DEB70C947178CF92DF92EF92FF927D
:10ED10000F931F936C018B017A01FA010995812FE2
:10ED20009927682FC6010196F70109951F910F9148
:10ED3000FF90EF90DF90CF9008955058BB27AA27FF
:10ED40000ED0E0C0D1D030F0D6D020F031F49F3FCB
:10ED500011F41EF4C6C00EF4E095E7FBBCC0E92F29
:10ED6000E2D080F3BA17620773078407950718F09B
:10ED700071F49EF5FAC00EF4E0950B2EBA2FA02D7B
:10ED80000B01B90190010C01CA01A0011124FF2758
:10ED9000591B99F0593F50F4503E68F11A16F04053
:10EDA000A22F232F342F4427585FF3CF4695379552
:10EDB0002795A795F0405395C9F77EF41F16BA0B17
:10EDC000620B730B840BBAF09150A1F0FF0FBB1FC5
:10EDD000661F771F881FC2F70EC0BA0F621F731F0E
:10EDE000841F48F4879577956795B795F7959E3F6B
:10EDF00008F0B3CF9395880F08F09927EE0F9795F9
:10EE00008795089598D088F09F5790F0B92F99274B
:10EE1000B751A0F0D1F0660F771F881F991F1AF025
:10EE2000BA95C9F712C0B13081F09FD0B1E0089512
:10EE30009CC0672F782F8827B85F39F0B93FCCF393
:10EE4000869577956795B395D9F73EF4909580951B
:10EE5000709561957F4F8F4F9F4F0895E89409C03B
:10EE600097FB3EF490958095709561957F4F8F4FFD
:10EE70009F4F9923A9F0F92F96E9BB279395F69513
:10EE8000879577956795B795F111F8CFFAF4BB0F91
:10EE900011F460FF1BC06F5F7F4F8F4F9F4F16C0F5
:10EEA000882311F096E911C0772321F09EE8872F7F
:10EEB000762F05C0662371F096E8862F70E060E03B
:10EEC0002AF09A95660F771F881FDAF7880F9695B4
:10EED000879597F9089597F99F6780E870E060E05B
:10EEE00008959FEF80EC089500240A9416161706E3
:10EEF00018060906089500240A941216130614062B
:10EF000005060895092E0394000C11F4882352F08D
:10EF1000BB0F40F4BF2B11F460FF04C06F5F7F4F45
:10EF20008F4F9F4F089557FD9058440F551F59F02C
:10EF30005F3F71F04795880F97FB991F61F09F3FE6
:10EF400079F087950895121613061406551FF2CF0F
:10EF50004695F1DF08C0161617061806991FF1CF5F
:10EF600086957105610508940895E894BB27662786
:10EF70007727CB0197F90895629FD001739FF00125
:10EF8000829FE00DF11D649FE00DF11D929FF00D39
:10EF9000839FF00D749FF00D659FF00D9927729F70
:10EFA000B00DE11DF91F639FB00DE11DF91FBD01FB
:10EFB000CF0111240895991B79E004C0991F961779
:10EFC00008F0961B881F7A95C9F780950895AA1BAB
:10EFD000BB1B51E107C0AA1FBB1FA617B70710F044
:10EFE000A61BB70B881F991F5A95A9F78095909576
:10EFF000BC01CD01089597FB092E07260AD077FDA5
:10F0000004D0E5DF06D000201AF4709561957F4F9B
:10F010000895F6F7909581959F4F0895A1E21A2ED5
:10F02000AA1BBB1BFD010DC0AA1FBB1FEE1FFF1FAC
:10F03000A217B307E407F50720F0A21BB30BE40BFC
:10F04000F50B661F771F881F991F1A9469F7609543
:10F050007095809590959B01AC01BD01CF010895FD
:10F0600097FB092E05260ED057FD04D0D7DF0AD016
:10F07000001C38F450954095309521953F4F4F4FE7
:10F080005F4F0895F6F790958095709561957F4F45
:10F090008F4F9F4F08952F923F924F925F926F92A2
:10F0A0007F928F929F92AF92BF92CF92DF92EF9218
:10F0B000FF920F931F93CF93DF93CDB7DEB7CA1B99
:10F0C000DB0B0FB6F894DEBF0FBECDBF09942A88C4
:10F0D000398848885F846E847D848C849B84AA846C
:10F0E000B984C884DF80EE80FD800C811B81AA81F9
:10F0F000B981CE0FD11D0FB6F894DEBF0FBECDBFC4
:10F10000ED010895EE0FFF1F0590F491E02D099495
:02F11000FFCF2F
:10F112005E0A010164FF01FFFFC01FC01F01010160
:10F12200737373FF03007D0000C409C409640010F7
:10F132004661737400004E6F726D616C0000456130
:10F142007379000051756164726F00006400D2012E
:10F1520001200B050000ECFF000204060708080866
:10F162000706040200FEFCFAF9F8F8F8F9FAFCFEC8
:10F17200000204060708086440415A4664640A0211
:10F18200969696960840403A10FB30380132FF03BB
:10F19200780090D0030090D0030032002064FFFF7B
:10F1A20064200B0A0D0B0C0E0B0F10FA200101014B
:06F1B20070FF010F640074
:00000001FF
